:100000000C944E090C947F090C947F090C947F0981
:100010000C947F090C947F090C947F090C947F0940
:100020000C947F090C947F090C947F090C947F0930
:100030000C947F090C947F090C947F090C94DD4685
:100040000C947F090C947F090C947F090C947F0910
:100050000C947F090C947F090C947F090C94996788
:100060000C947F090C9462600C9438600C947F09A6
:100070000C947F090C947F090C947F090C947F09E0
:100080000C947F090C947F090C947F090C947F09D0
:100090000C9428610C9498600C94DF600C94F547E4
:1000A0000C947F090C947F090C947F090C947F09B0
:1000B0000C947F090C947F090C947F090C947F09A0
:1000C0000C947F090C947F090C947F090C940260B6
:1000D0000C94D85F0C947F090C947F090C947F09D1
:1000E0000C947F09720B2A0C470D7A0D7A0D5B0D6B
:1000F000200C7A0D7A0D7A0D350C350C350C7A0DF5
:100100007A0D6B0BE00B820B8F0BE00BE00B070CF7
:10011000170C8F0B070CE00BAA0C940C940CAA0C78
:10012000AA0CB70CC20C8B0CAA0CAA0C25102A1016
:100130002F1039104310BC104D1055105D10671072
:1001400071107B108A109410BC109E10A810B21071
:10015000A2167D16BD16BD16BD16BD16BD16BD1662
:10016000BD16BD16BD16E212DA15FB15F415E51520
:10017000BD16BD16BD16BD16BD16BD16BD16911613
:10018000F01CE41CE41CF01CF01CCB1CD81CD81C7C
:10019000F01CF01C9C289F28B728CE2817292A2954
:1001A0004A29A24D914D944D9C4D9C4D944D914D9D
:1001B0009C4D9C4D9C4D914D914D914D9C4D9C4D18
:1001C000A24D865083508350865086508850885068
:1001D0004950865086500A530A530A530A5307530C
:1001E00007530E530E530E530E530E530E530E530E
:1001F0000E53075307530E530E530E530E530E5305
:100200000C530A5332643564246428642E646C648D
:1002100039643D64436447644B6451645564596474
:100220006C645F646364676407634236B79BD8A7F6
:100230001A39685618AEBAAB558C1D3CB7CC57630B
:10024000BD6DEDFD753EF6177231BF000000803FB9
:1002500008000000BE922449123EABAAAA2ABECDD5
:10026000CCCC4C3E00000080BEABAAAAAA3E000047
:100270000000BF000000803F00000000000841783F
:10028000D3BB4387D1133D190E3CC3BD4282AD2B76
:100290003E68EC8276BED98FE1A93E4C80EFFFBE6E
:1002A00001C4FF7F3F00000000000C9482700C949A
:1002B00087270C943D640C949C340C940A530C9442
:1002C0003D420C9459640C945E5E0C949A260C94F6
:1002D000944D0C946B400C949F280C943F260C94E6
:1002E0002A100C9428640C9422260C9432640C94EA
:1002F0001C440C942B400C94F04C0C94685D0C94B2
:100300008C410C942F100C94E41C0C9488500C9489
:10031000E2120C94815E0C9488400C94F4150C94B9
:10032000820B0C947A0D0C9447640C9465410C94E8
:1003300071100C940C530C94E72F0C94CE280C9451
:100340007C1D0C948F0B0C942A0C0C944A290C9451
:100350001B5D0C94720B0C9477450C9443640C94C5
:1003600058330C9425100C9413260C94C4400C9410
:10037000E5150C9445330C9494100C942A290C9494
:100380005B0D0C9467100C9491160C9446350C94EC
:1003900052450C940F420C94BD160C9439640C9485
:1003A00074400C9443100C9486500C94CB330C94F2
:1003B0006C640C942E640C94914D0C94070C0C946A
:1003C000A2160C947D160C948C430C9424640C940B
:1003D00049500C94FC2B0C945F640C94FB150C940A
:1003E0009C4D0C9459270C94DA340C94DA210C941B
:1003F0005D100C9445450C94F01C0C947F400C94BB
:100400008B0C0C94B7280C9463640C94B70C0C946C
:10041000DD380C9417290C9475440C94F3430C9418
:10042000A22A0C9453400C946B0B0C94B2100C94B5
:100430006D330C949E100C9472400C9497270C947E
:100440005B400C9423490C94A8100C9487400C94A6
:10045000765D0C945D450C9439100C949B4A0C9479
:100460006A270C944D100C944B640C94545D0C94BE
:1004700035640C94940C0C94350C0C943D400C9405
:10048000E0440C9483500C949C280C9436430C94B8
:10049000AA0C0C94AC260C9407530C94A24D0C940B
:1004A0001D410C94D81C0C94BC100C942C4A0C9438
:1004B000DA150C9455640C949E400C94E4270C942B
:1004C00048450C947B100C9483410C94455D0C942E
:1004D000B85D0C940E530C94C20C0C945C5E0C949E
:1004E000470D0C945A350C94200C0C94DD410C945F
:1004F0003C410C9451640C94E00B0C94055E0C94FC
:10050000D4260C94845F0C946F260C944F330C9477
:100510009C4A0C94974A0C94170C0C94002C0C9445
:100520008A100C944B450C9457400C9469410C94E0
:1005300081090C94E8330C9444430C94DB260C940E
:1005400055100C94CB1C0C9461260C946764636466
:10055000696E6F70737578585B003D0056432300D9
:1005600020636D643D003D0056435F686561742300
:10057000003D0050696E3A003D0050696E3A00201F
:1005800048616C7465640A003D00526573746F7253
:1005900065643A20003A204E6F2073746F72656470
:1005A0002076616C756573202D2064656661756CBD
:1005B000740A00466F7263652057686974650A00A3
:1005C000416C7265616479204163746976650A00E3
:1005D0005475726E696E6720584F4E0A00416C72F6
:1005E000656164792048616C7465640A00416C72CD
:1005F0006561647920496E6163746976650A0041BA
:100600006C7265616479204163746976650A00548F
:1006100075726E696E6720584F4E0A00584F4646F5
:1006200020736B69707065642E205072657620634C
:100630006D643A005475726E6564206F666620665C
:10064000726F6D3A00526573746F726564206672E2
:100650006F6D3A00536B6970204772700029003E3D
:10066000003C00205061723D280020436D643D0035
:1006700020537566663D00205375623D0020497425
:10068000656D3D0052414D3D00476F74204950203B
:10069000616464726573733A00276970205B6970E6
:1006A0005B2C646E735B2C67775B2C7375626E6575
:1006B000745D5D5D5D27202D20736574207374610A
:1006C0007469632049500A004661696C656420744E
:1006D0006F20636F6E666967757265204574686523
:1006E000726E6574207573696E6720444843502E9E
:1006F00020596F752063616E2073657420697020C6
:100700006D616E75616C6C792100537461727469EE
:100710006E67206C616E00246E6F646573002466E2
:100720006F726D6174002464617461747970650026
:10073000302D31303000696E746567657200687302
:100740007600636F6C6F72004F4E2C4F46462C48FC
:10075000414C542C524553542C584F4E2C584F4614
:10076000462C544F47474C4500656E756D00666CCE
:100770006F617400322E312E300024686F6D696510
:1007800000757074696D652C667265656865617069
:1007900000393335366661375F323031392D3130CB
:1007A0002D3136004C696768744875622000246EEC
:1007B000616D6500726561647900207472792061F1
:1007C0006761696E20696E2035207365636F6E64A2
:1007D00073006661696C65642C2072633D0041772B
:1007E000616974696E6720666F72207265746169F1
:1007F0006E656420746F7069637300636F6E6E65FD
:10080000637465642061732000202E2E2E002075F5
:100810007365723A003A000A417474656D707469C8
:100820006E67204D51545420636F6E6E656374691A
:100830006F6E20746F2000247374617465006469A6
:1008400073636F6E6E6563746564005573696E677C
:10085000204D5154542070617373776F7264206619
:10086000726F6D20636F6E666967004465766963B9
:1008700065204E616D653A00526562696E64207351
:100880007563636573732E204950206164647265DB
:1008900073733A004572726F723A20726562696EC4
:1008A00064206661696C0052656E657765642073CB
:1008B0007563636573732E204950206164647265AB
:1008C00073733A004572726F723A2072656E657783
:1008D0006564206661696C004E6F206C696E6B0008
:1008E000416363657074696E6720636F6D6D616EDF
:1008F00064732E2E2E0A003E3E3E004E6F204D4168
:100900004320636F6E666967757265643A2073652C
:1009100074206669726D776172652773204D41435B
:100920000A004D6F6462757320706F6C6C696E673E
:10093000206572726F723D002D0020504920566173
:100940006C203A004D6F6462757320706F6C6C6937
:100950006E67206572726F723D002D0020464D203B
:1009600056616C203A004D6F6462757320706F6C35
:100970006C696E67206572726F723D002056616C03
:100980003A20004D423A20004E6F7420737570700B
:100990006F727465642072656720747970650A00EF
:1009A000496C6C6567616C20617267756D656E740A
:1009B000730A00757074696D6500667265656865B7
:1009C00061700024737461747300200020000A5267
:1009D000414D3D00202D746172676574207A6F6E01
:1009E000652D00204F464600204F4E00204F4646C2
:1009F0000020636D643A00204375723A002053650D
:100A0000743A0020457870697265640A002F0049C5
:100A10006E3A20003D00494E3A0066616E006D6FEF
:100A2000646500536574436D643A00536574466CA5
:100A300061673A00436C72466C61673A0020566108
:100A40006C3D002053746F7265200052474200488D
:100A50005356004C4F57004D454449554D004849A9
:100A6000474800444543524541534500494E43528F
:100A7000454153450044495341424C454400454E8D
:100A800041424C45440046414C5345005452554563
:100A9000004452590046414E5F4F4E4C5900584F4A
:100AA000464600584F4E0048414C5400544F47476B
:100AB0004C4500524553540054787432436D643AA7
:100AC000002B002D00485454502F312E3120256921
:100AD0000020485454502F312E310D0A486F737442
:100AE0003A2025730D0A4163636570743A202A2FFA
:100AF0002A0D0A436F6E6E656374696F6E3A2063E8
:100B00006C6F73650D0A0025730020000D0A004705
:100B10004554006661696C656420746F20636F6E74
:100B20006E6563740A004552524F523A2053657203
:100B30007665722072657475726E65642000446F0C
:100B40006E652E0A004170706C79696E672E0A001E
:100B5000436F6E6669672070617273696E672066A5
:100B600061696C65640A00676F7420436F6E666923
:100B7000670A00436F6E666967205552493A2068DC
:100B80007474703A2F2F002044656661756C742070
:100B9000636F6E6669672073657276657220757320
:100BA00065643A20006C617A79686F6D652E7275A4
:100BB00000205361766564000A282D29524553545C
:100BC0004152545F4C414E5F4F4E5F4D5154545F04
:100BD0004552524F5253000A282D2948415244523F
:100BE000455345542C207573696E6720736F667486
:100BF000000A282D29434F554E544552000A282DEE
:100C000029444854000A282D294F57495245000AC3
:100C1000282B294D4F44425553000A282B29444D77
:100C200058000A282B2957697A4E657435353030BB
:100C3000000A282B294453323438322D3130300009
:100C40000A282B294672656552616D207072696EA3
:100C500074696E670064653A61643A62653A656614
:100C60003A66653A6564000A4669726D7761726535
:100C7000204D4143204164647265737320006C61B0
:100C80007A79686F6D652E7275000A436F6E6669BA
:100C900067207365727665723A000A282B295741DE
:100CA000544348444F47003230313130334C0020F8
:100CB000432B2B2076657273696F6E3A003933359A
:100CC000366661375F323031392D31302D313600A3
:100CD0000A4C617A79686F6D652E7275204C696770
:100CE000687448756220636F6E74726F6C6C6572A5
:100CF0002000000020002300260029002C002F00E7
:100D00003200000100000301060109013D00494EC7
:100D10003A0043757272656E74204C414E20636FC9
:100D20006E6669672869702C646E732C67772C7304
:100D300075626E6574293A000A557365207468659A
:100D4000736520636F6D6D616E64733A202768650B
:100D50006C7027202D207468697320746578740A7C
:100D6000276D61632064653A61643A62653A65663D
:100D70003A66653A3030272073657420616E6420CE
:100D800073746F7265204D41432D616464726573A5
:100D90007320696E20454550524F4D0A27697020D7
:100DA0005B69705B2C646E735B2C67775B2C73756F
:100DB000626E65745D5D5D5D27202D207365742016
:100DC0007374617469632049500A277361766527DB
:100DD000202D207361766520636F6E6669672069D8
:100DE0006E204E5652414D0A2767657427205B637B
:100DF0006F6E66696720616464725D27202D2067CD
:100E0000657420636F6E6669672066726F6D20700F
:100E100072652D636F6E66696775726564205552E1
:100E20004C20616E642073746F726520616464721B
:100E30000A276C6F616427202D206C6F616420632A
:100E40006F6E6669672066726F6D204E5652414D17
:100E50000A2770776427202D20646566696E6520F7
:100E60004D5154542070617373776F72640A276B0D
:100E7000696C6C27202D207465737420776174630E
:100E800068646F670A27636C65617227202D206391
:100E90006C65617220454550524F4D0A277265625C
:100EA0006F6F7427202D207265626F6F7420636FDF
:100EB0006E74726F6C6C657200536F66742072652D
:100EC000626F6F74696E672E2E2E00444D58696EE6
:100ED0002042756666657220616C6C6F6320657276
:100EE0007200496E697420696E2063683A0052414D
:100EF0004D3D000A6D71747420000A6D6F64627557
:100F00007320000A696E7075747320000A69746535
:100F10006D7320000A436F6E666967757265643A87
:100F2000002C003D0050696E3A002C003D4C4F579C
:100F300000546865726D6F3A00444D58206F7574A7
:100F400020737461727465642E204368616E6E65EF
:100F50006C733A2000444D5820696E20737461729E
:100F60007465642E204368616E6E656C733A004C44
:100F70006F61646564006C6F6164206661696C65B3
:100F800064004E6F2073746F72656420636F6E66C9
:100F90006967004C6F6164696E6720436F6E6669B4
:100FA000672066726F6D20454550524F4D000A72A2
:100FB000657175657374204D51545420436F6E668E
:100FC000696700536176656420746F20454550520F
:100FD0004F4D00536176696E6720636F6E66696777
:100FE00020746F20454550524F4D2E2E0053617690
:100FF00065640A005365742064796E616D696320CD
:1010000049500A00454550524F4D20636C6561724E
:1010100065640A0050617373776F72642075706441
:10102000617465640A00636F756C64206E6F742070
:1010300070617273653A2000557064617465640A6A
:10104000002C20002E00696E00735F6F7574006DB8
:1010500079686F6D65002076616C75652069732015
:101060000020756E6B6E6F776E0A0020696E61638B
:10107000746976650A00206163746976650A0020E8
:101080004772703A0020696E6163746976650A0080
:10109000206163746976650A0020696E76616C6907
:1010A00064004D6F64627573206F70206661696CB7
:1010B00065640A002D3E005075623A2000636D643D
:1010C00000434F4F4C0048454154004155544F0098
:1010D0002D3E005075623A2000736574002D3E006D
:1010E0005075623A20002D3E005075623A2000553E
:1010F0006E6B6E6F776E20636D64200A004F4646FC
:10110000004F4E00537461747573206465666665A4
:101110007265640A004E6F7420737570706F72741C
:1011200065642072656720747970650A00293A0049
:1011300028543A003D3E00206973200044656C65E8
:1011400074696E6720636F6E662E2052414D207762
:1011500061733A00536B697070696E672E2E004F91
:101160004F4D21005D20000A5B003A004D41433A9B
:10117000005265747279696E6720434D440A003EDF
:101180003E2000496E76616C696420636F6D6D610D
:101190006E640000002100240027002A002D00308A
:1011A00000330001010000040107010A01000022D0
:1011B00000250028002B002E003100340002010021
:1011C00000050108010B01050505050705080808CC
:1011D00008020202020A0A080804040404010101C8
:1011E00001010101010303030303030303040707D0
:1011F000070C0C0C0C0C0C0C0C020202020606066E
:1012000006060606060B0B0B0B0B0B0B0B01021055
:101210002020080810204010204080020102010810
:1012200004020101020408102040808040201008C0
:101230000402018004020180402010080402010819
:101240000402010102040810204080010204081079
:1012500020408000000A0B02090C0D0E0807030451
:10126000010000000000000000000000000000007D
:10127000000000000000000000000000000000125C
:10128000111000000000000000000000000000003D
:1012900000000000000000000000827011241FBE4A
:1012A000CFEFD1E2DEBFCDBF00E00CBF15E0A0E084
:1012B000B2E0EAE7F3E001E00BBF02C007900D9255
:1012C000AA38B107D9F72BE0AAE8B5E001C01D9212
:1012D000A333B207E1F719E0CEE4D9E000E006C09D
:1012E00021970109802FFE010E94877CCD34D10710
:1012F00080E00807A9F70E94E3670C94BB810C9477
:1013000000002F923F924F925F926F927F928F9246
:101310009F92AF92BF92CF92DF92EF92FF920F9384
:101320001F93CF93DF93CDB7DEB76D970FB6F894C9
:10133000DEBF0FBECDBF5C011B015B8B4A8B490139
:10134000102FFD8AEC8ADF8ACE8ADC011296ED919D
:10135000FC911397E080F1800E94104A2B013C0120
:1013600064E876E086E398E00E94A35E2AE0B30199
:10137000A20186E398E00E94DC5E6DE776E086E3FA
:1013800098E00E94A35EB70186E398E00E94CA5FDE
:1013900067E776E086E398E00E94A35E6E897F8926
:1013A00086E398E00E94CA5F60E776E086E398E013
:1013B0000E94A35E4AE050E06C897D8986E398E054
:1013C0000E946D5F6AE676E086E398E00E94A35E85
:1013D0004AE050E0B10186E398E00E946D5F63E669
:1013E00076E086E398E00E94A35EF5018281938116
:1013F000892B11F40C94E6111D861C861F861E860F
:10140000198A188A8114910479F164017E01FCE043
:10141000EF0EF11C612C712C2A893B896216730630
:101420001CF533E063167104F9F0D6014D905D9020
:101430006D01F701419251927F0161E676E086E30A
:1014400098E00E94A35E4AE050E0B20186E398E093
:101450000E946D5F6FE576E086E398E00E94A35EF0
:10146000FFEF6F1A7F0AD8CF6DE576E086E398E04C
:101470000E94A35E86E398E00E94C65FD50118969D
:101480008C91873069F411110BC064E576E086E336
:1014900098E00E94A35E86E398E00E94C65F96C72C
:1014A00060E070E0C5010E94C7222C01C5010E94C6
:1014B000D94F7C01B4E02B16310451F0E7E02E1631
:1014C000310469F1F3E02F16310409F05AC005C068
:1014D000181619060CF452C01EC0D50118968C912E
:1014E000873009F44EC0C5010E94AB23853009F056
:1014F0007DC765E476E086E398E00E94A35E4AE05B
:1015000050E065E070E086E398E00E946D5F86E35E
:1015100098E00E94C65F22242394312C32C0F5014A
:101520008085873071F1C5010E94AB23C82ED12C74
:10153000863091F464E376E086E398E00E94A35E4F
:101540004AE050E0B60186E398E00E946D5F86E3D2
:1015500098E00E94C65F12C06CE176E086E398E0F6
:101560000E94A35E4AE050E0B60186E398E00E9444
:101570006D5F86E398E00E94C65F38C7A2E02A2E1E
:10158000312CD50119966D907C901A9761147104D5
:1015900009F495C0B5E02B16310409F444C034F4C5
:1015A000F2E02F16310409F459C075C026E0221666
:1015B0003104C9F03FE02316310409F06CC0D301B7
:1015C000ED91FC910488F589E02DCE88DF88EC88C8
:1015D000FD88012F94014A895B896FE070E0C301A7
:1015E00019950C94A112EF2809F0FAC66FE076E085
:1015F00086E398E00E94A35EF50181859285DC0177
:10160000ED91FC910488F589E02DCE88DF88EC8887
:10161000FD88012F94014A895B8961E070E019958A
:101620008C0166E0D8C61E141F04ACF4D301ED9102
:10163000FC910488F589E02DCE88DF88EC88FD8850
:10164000012F94014A895B8962E070E0C30119951A
:101650008C0165E0C0C66DEE75E0C4C6C5010E9490
:10166000AB238530A9F0D301ED91FC910488F58975
:10167000E02DCE88DF88EC88FD88012F94014A890F
:101680005B8962E070E0C30119958C0162E0A3C63A
:101690006DED75E0A7C6D301ED91FC910488F58945
:1016A000E02DCE88DF88EC88FD88012F94014A89DF
:1016B0005B89B101C30119958C01622D8CC6B0E123
:1016C0002B16310408F016C2F1018827EE58FF4F9F
:1016D0008F4F0C94877C882483941E141F0424F05D
:1016E000812C02C088248394F501808590E08A30A3
:1016F000910508F09CC0FC018827EE57FF4F8F4FE3
:101700000C94877C8E859F85892B49F42A893B8997
:101710002330310521F48FE7D50118968C93C5014C
:101720000E94AD22D62E972EC82E092FEA89FB895A
:10173000E230F105D1F0E330F10531F1319761F597
:101740004C855D85D42E97FF27C09F778C879D871A
:10175000272F30E03F872E87CA019927998B888BE6
:1017600023E030E03B8B2A8B17C0CC840D850F77AC
:101770009078092B9E8470E0798B688B006883E0F9
:1017800090E09B8B8A8B08C0CC840D850F77907876
:10179000092B9E84D88800684D2D592D6C2D702FF3
:1017A000C5010E947522882061F11E141F041CF4DB
:1017B000D11024C017C0EF2809F5DD20F9F01AC0B8
:1017C0004C855D85052E000C660B770BC5010E94CC
:1017D00075228820B1F01E141F0434F48C859D8579
:1017E000892B61F462E007C0EF2841F48C859D8568
:1017F000892B21F061E0C5010E947F2360E07BE03E
:1018000022C660E07AE0C5010E94F34C12C04C850C
:101810005D85052E000C660B770BC5010E947522B5
:10182000112329F060E07AE0C5010E94F34C811099
:1018300061C1D50118968C91873009F0C9C55AC18C
:10184000E114F10409F0D5C560ED75E086E398E098
:101850000E94A35EF5018085813039F4C5010E94A4
:10186000AB23813011F41111CFC5622DC5010E9447
:101870007F231E141F0444F4112331F060E071E053
:10188000C5010E94F34CA4C5C5010E94AD22DC0134
:10189000CB01D82E992ECA2E0B2FF501208523308F
:1018A00018F4213018F010C02430E9F44997A1054C
:1018B000B1052CF4F2E3DF2E912CC12C00E04D2D6C
:1018C000592D6C2D702F0CC00097A105B10529F082
:1018D000F8E1F81710F0E2E3DE2E4D2D592FBD018F
:1018E000C5010E9475224D2D592D6C2D702F41156B
:1018F00051056105710509F449C0D50118968C910F
:1019000090E08A309105F0F5FC018827E457FF4FFD
:101910008F4F0C94877C112309F4ECC0C5010E9401
:10192000D94F892B49F193C50F77CC860D87892D27
:1019300090E09F878E878D2D90E0998B888B112367
:1019400029F060E073E0C5010E94F34C73E0672E5C
:10195000712C6EC05D874C87112329F060E073E025
:10196000C5010E94F34C66246394712C61C05D87AD
:101970004C87112309F429C560E071E0C5010E947C
:10198000F34C65C5112309F462C5F6CF2AE030E0B7
:1019900040E050E0BA0186E398E00E94255F65E9E7
:1019A00075E086E398E00E94A35EF50180858530AE
:1019B000C9F0A0F48150823078F584E690E09D87EC
:1019C0008C871F861E86998B888B007844E650E0B2
:1019D00064E6702FC5010E947522B1CF863059F0A0
:1019E0008830D1F484E190E09D878C8744E150E019
:1019F00060E070E019C084E690E09D878C8744E643
:101A000050E060E070E0C5010E947522112309F4E6
:101A1000AACF60E071E0A4CF84E690E09D878C8738
:101A200044E650E060E070E0C5010E94752294CF6A
:101A30006E01FCE0CF0ED11CE12CF12CD6018D9073
:101A40009D906D016AE875E086E398E00E94A35ED0
:101A50004AE050E0B70186E398E00E946D5F68E8D5
:101A600075E086E398E00E94A35E4AE050E0B4018E
:101A700086E398E00E946D5F86E398E00E94C65F6F
:101A8000BFEFEB1AFB0A6E147F04C1F6E0C4C50178
:101A90000E94AB23853071F11D861C861F861E8631
:101AA000198A188A62E0C5010E947F23112311F16F
:101AB00060E071E0C8C41E141F04E4F41D861C8697
:101AC0001F861E86198A188AC5010E94AB2386309C
:101AD00011F462E001C065E0C5010E947F2360E06F
:101AE00071E0C5010E94F34C6FE775E086E398E072
:101AF0000E94A35ECE84DF84C6010D2C000CAA0BCD
:101B0000BB0B8A8F9B8FAC8FBD8FA889B989B98F8A
:101B1000A88F2FEF30E00E949E7C54E6652E712C3A
:101B2000812C912CA40193010E94467C7901F5013E
:101B30008085843009F4A8C158F4813009F443C089
:101B4000C8F0823009F4B3C0833009F416C23DC432
:101B5000883009F4D0C338F4863009F4C8C187301E
:101B600009F498C132C4893009F42EC38F3709F4BF
:101B70006CC12BC4141415040CF027C4AC85BD85AE
:101B80002FEF30E00E949E7CA40193010E94467CCE
:101B9000622FC20157C1C6010D2C000CAA0BBB0B52
:101BA0008A8F9B8FAC8FBD8FA889B989B98FA88F79
:101BB0002FEF30E00E949E7C24E630E040E050E0D1
:101BC0000E94467C7901F2E3CF16D1040CF051C09B
:101BD000141415040CF058C182E390E08C199D098F
:101BE000288D398D829FD001839FB00D929FB00DBB
:101BF00011242FEF30E00E949E7C28E833E140E082
:101C000050E00E94467C622FC20103960E94C947A1
:101C10000E851F852EEF31E0D8010E949E7C42E3A5
:101C2000C42ED12CE12CF12CA70196010E94467CF8
:101C3000A889B9890E94967C24E630E040E050E013
:101C40000E94467C49015A019801A5E6BFEF0E9417
:101C5000967CA70196010E94467C0FEF020F74014B
:101C60003FEF8316910489F184F1EE24EA94F12C7C
:101C70002CC0141415040CF007C12A8D3B8D4C8D1B
:101C80005D8D2253310941095109ABE9B0E00E9451
:101C9000657C22E330E040E050E00E94467C04E6B0
:101CA000020F60E0C20103960E94C9470EC01414DF
:101CB00015040CF0E9C02FEF30E0D6010E949E7CA5
:101CC000A40193010E94467C022FAC85BD852FEFB5
:101CD00030E00E949E7C2DE631E040E050E00E9422
:101CE000467C322F122F1F71110F110F812F880F79
:101CF00015E5682F619F060E60E0611D1124922F8B
:101D00009074207237FD24C091110CC0211104C0C1
:101D1000862F8095F62E14C025E5F22EF60E10E0E3
:101D20006BEA36C021110FC0182F3AEA139F010E3B
:101D300010E0111D11248BEA811B9AEAF92EF60E90
:101D4000682F10E025C080E0F62EF094162F0FC00B
:101D5000911112C021110DC0182F2AEA129F010EF5
:101D600010E0111D11243BEAF32EF11A1B5A60E01A
:101D70000FC0162F10950BC0211104C085E5860FEA
:101D80001BEA03C08AEA860F90E0161B682FF12C2D
:101D90000F3F09F425C00023F9F0662321F0609F6E
:101DA000060E60E0611DFF2031F03F2D309F030ED5
:101DB00030E0311DF32E112321F0109F010E10E0B1
:101DC000111D11240095009F000E00E0011D11243B
:101DD000600FF00E100F04C01FEFFF24FA946FEF96
:101DE0008FEFE81609F423C020E03E2D332321F0C5
:101DF000339F212D09F02F5F2223B1F0662321F0BC
:101E0000629F060E60E0611DFF2031F03F2D329F82
:101E1000030E30E0311DF32E112321F0129F010E2D
:101E200010E0111D112403C010E0F12C60E0C2018C
:101E30000E94C9476F2DC20101960E94C947612FB8
:101E4000C20102960E94C947C0C214141504E4F4EA
:101E500060E0C2010E94C94760E0C20101960E9491
:101E6000C94760E0C20102960E94C947A889B989A2
:101E70002FEF30E00E949E7CA40193010E94467CDB
:101E8000622FC2010396DECF6C857D85C5010E945D
:101E90001E4F9BC20480F581E02D8085853009F0BE
:101EA00094C2A680B780A114B10409F48EC2F501D2
:101EB00061857285CE0101960E946D54CE88DF88BF
:101EC000EC88FD88012F9E01245F3F4F4A895B8982
:101ED000B101CE0101960E948109D5011296AD9003
:101EE000BC901397CE0101960E942F51DCCF411474
:101EF000510409F46AC257FE06C051944194510836
:101F000001E010E002C000E010E0F42C61E0842D5C
:101F10000E949C64012B69F0B1E02B16310429F07A
:101F200061E0E6E02E16310409F460E0062F10E0CF
:101F300011C0F1E02F16310451F091E080E026E06D
:101F40002216310409F090E0092F182F02C001E099
:101F500010E0602F8F2D0E946D646AE775E086E3C4
:101F600098E00E94A35E4AE050E0B20186E398E068
:101F70000E946D5F68E775E017C14114510409F4D0
:101F800023C157FE06C051944194510801E010E06E
:101F900002C000E010E0F42C61E0842D0E949C64FB
:101FA0008091A100887F8093A10080919100887F1B
:101FB000809391008091A10082608093A100809124
:101FC0009100826080939100AC85BD85012B99F0D2
:101FD000CD01BB0FAA0BBB0B9C01AD0124563109EF
:101FE00041095109AFEFB0E00E94657C2CE93FEF59
:101FF0004FEF5FEF08C02FEF30E00E949E7C24E699
:1020000030E040E050E00E94467C890161E08F2D85
:102010000E949C640115110509F4B1C00F3F110520
:1020200009F4AFC0F201FF27ED5AFD4EE4918E2F67
:1020300090E0FC013197E231F10508F09DC088275E
:10204000EA56FF4F8F4F0C94877C84B5806884BD1F
:1020500007BD9BC084B5806284BD08BD96C08091D9
:10206000800080688093800010938900009388002E
:102070008CC08091800080628093800010938B00E0
:1020800000938A0082C080918000886080938000E5
:1020900010938D0000938C0078C08091B000806810
:1020A0008093B0000093B30070C08091B000806254
:1020B0008093B0000093B40068C080919000806865
:1020C0008093900010939900009398005EC08091D7
:1020D000900080628093900010939B0000939A0080
:1020E00054C08091900088608093900010939D0070
:1020F00000939C004AC08091A00080688093A0005B
:102100008091A0008F7B8093A0001093A900009382
:10211000A8003BC08091A00080628093A000109333
:10212000AB000093AA0031C08091A000886080932A
:10213000A0001093AD000093AC0027C08091200157
:1021400080688093200110932901009328011DC00D
:102150008091200180628093200110932B010093D5
:102160002A0113C080912001886080932001109380
:102170002D0100932C0109C00038110514F460E012
:1021800001C061E08F2D0E946D6463E775E086E316
:1021900098E00E94A35E4AE050E0B20186E398E036
:1021A0000E946D5F61E775E086E398E00E94A35EA0
:1021B0004AE050E0B80186E398E00E946D5F86E354
:1021C00098E00E94C65F01C11C8560E070E0C50117
:1021D0000E94C722082FF92E6CE575E086E398E08F
:1021E0000E94A35E4AE050E0602F7F2D86E398E0D6
:1021F0000E946D5F6AE575E086E398E00E94A35E49
:10220000612F012E000C770B4AE050E086E398E046
:102210000E946D5F86E398E00E94C65F80918E0504
:1022200090918F05892B81F0622DC5010E947F233B
:10223000412F110F550B660B770BC5010E947522BC
:10224000C5010E940E4FC1C081E090E090938F05C0
:1022500080938E0526E040E855E260E070E089E971
:1022600097E00E94FA5300938C0989E997E09093D4
:102270008B0980938A091092970A1092990A1092FA
:10228000980A80ED97E09093120A8093110A1092B9
:10229000140A1092130A112339F085E090E090930C
:1022A000160A8093150A04C01092160A1092150A95
:1022B00086E00E94435162E370E080E090E00E947B
:1022C000D86482ED97E09093120A8093110A1092DD
:1022D000140A1092130A34E61302A0011124509339
:1022E000160A4093150A86E00E94435110928F050A
:1022F00010928E056AC00480F581E02D618572859B
:10230000CE0101960E946D54CE0101960E94682272
:10231000882309F456C08985893009F052C0122DEE
:10232000EC8460E070E0CE0101960E94C722082F85
:10233000F92E68E675E086E398E00E94A35E4AE025
:1023400050E0602F7F2D86E398E00E946D5F66E687
:1023500075E086E398E00E94A35E6E2D0E2C000CC3
:10236000770B4AE050E086E398E00E946D5F60E6FC
:1023700075E086E398E00E94A35E4AE050E0622D9B
:10238000022C000C770B86E398E00E946D5F86E3D9
:1023900098E00E94C65F80918E0590918F05892BF1
:1023A00009F464C0622DC5010E947F234E2DEE0CFE
:1023B000550B660B770BC5010E947522C5010E9463
:1023C0000E4FCE0101960E942F51BBC08FEF0FC060
:1023D00081E090E0B6C0C5010E947F23C801B1C072
:1023E0006FEF75E086E398E00E94A35E8DEF9FEFAC
:1023F000A8C060EC75E086E398E00E94A35EF5015A
:102400008085873099F726CA63EB75E086E398E00C
:102410000E94A35E8FE7D50118968C931F861E86B7
:1024200084E690E0998B888BCC847D857F7744E629
:1024300050E06C2DC5010E947522622DC5010E94DD
:102440007F2360E073E0C5010E94F34C53CBF5019C
:102450008085813009F04ECBCE84DF84C114D10455
:1024600009F099CB8FE7F501808744CB81E090E0BC
:1024700090938F0580938E0526E040E855E260E05A
:1024800070E089E997E00E94FA5300938C0989E98A
:1024900097E090938B0980938A091092970A109283
:1024A000990A1092980A1230A1F1153091F16E2D0F
:1024B000EE0C770B880B990B0E94C17D22E538EB5F
:1024C00042E152E40E94A67C20E030E040E251E488
:1024D0000E94767E2DEE3EE94CE35EE30E94177D7E
:1024E0006B017C0120E030E0A9010E94717E20E0B8
:1024F00030E040E05FE387FD05C0C701B6010E9400
:10250000A67C04C0C701B6010E94A57C0E94897DFB
:1025100002C060E070E083ED97E09093120A809330
:10252000110A1092140A1092130A7093160A6093FB
:10253000150A86E00E94435110928F0510928E0575
:1025400040CF6D960FB6F894DEBF0FBECDBFDF91C2
:10255000CF911F910F91FF90EF90DF90CF90BF90A0
:10256000AF909F908F907F906F905F904F903F9033
:102570002F9008954F925F926F927F928F929F92C9
:10258000AF92BF92CF92DF92EF92FF920F931F9381
:10259000CF93DF93CDB7DEB7C55AD1400FB6F894CD
:1025A000DEBF0FBECDBFE0919205F09193053B9643
:1025B000E831F10508F0E1C38827E855FF4F8F4F58
:1025C0000C94877C0E9412650091E0061091E10650
:1025D0002091E2063091E30606171707280739070E
:1025E00008F0CBC30DE613E0CF56DE4F1983088306
:1025F000C159D140CD56DE4F188219821A821B82F2
:10260000C359D140CF57DE4F19830883C158D140F9
:10261000CD57DE4F188219821A821B82C358D140CF
:10262000CF59DE4F19830883C156D140CD59DE4FB3
:10263000188219821A821B82C356D140CF5BDE4FAB
:1026400019830883C154D140CD5BDE4F18821982B3
:102650001A821B82C354D1406AE077E086E398E097
:102660000E94A35E86E398E00E94C65FBE016F569B
:102670007E4F86E090E00E94B9637C01892B09F4CB
:1026800067C165E773E086E398E00E94CA5F1A833A
:102690000983CD56DE4F88819981AA81BB81C359B8
:1026A000D1408B839C83AD83BE83CE0101960E9473
:1026B000313FBE016F577E4F8AE090E00E94B963C0
:1026C000892B09F42EC16BE873E086E398E00E9441
:1026D000CA5F1A830983CD57DE4F88819981AA8109
:1026E000BB81C358D1408B839C83AD83BE83CE0115
:1026F00001960E94313FBE016F597E4F8EE090E0FF
:102700000E94B963892B09F4DFC061E973E086E3B5
:1027100098E00E94CA5F1A830983CD59DE4F8881F1
:102720009981AA81BB81C356D1408B839C83AD83A1
:10273000BE83CE0101960E94313FBE016F5B7E4F8A
:1027400082E190E00E94B963892B09F477C066E9C1
:1027500073E086E398E00E94CA5F1A830983CD5B29
:10276000DE4F88819981AA81BB81C354D1408B837C
:102770009C83AD83BE83CE0101960E94313F1A83B4
:102780000983CD5BDE4F88819981AA81BB81C354C7
:10279000D1408B839C83AD83BE83CF57DF4F19839A
:1027A0000883C158D040CD59DE4F88819981AA81D4
:1027B000BB81C356D140CD57DF4F88839983AA830D
:1027C000BB83C358D040CF53DF4F19830883C15C0C
:1027D000D040CD57DE4F88819981AA81BB81C358F3
:1027E000D140CD53DF4F88839983AA83BB83C35CD9
:1027F000D040CF5FDE4F19830883C150D140CD5602
:10280000DE4F88819981AA81BB81C359D140CD5FB8
:10281000DE4F88839983AA83BB83C350D1409E0136
:102820002F5F3F4FAE014F575F4FBE016F537F4F3A
:10283000CE018F5F9E4F0E94495985C01A8309833C
:10284000CD59DE4F88819981AA81BB81C356D14081
:102850008B839C83AD83BE83CF57DF4F198308835F
:10286000C158D040CD57DE4F88819981AA81BB8164
:10287000C358D140CD57DF4F88839983AA83BB8348
:10288000C358D040CF53DF4F19830883C15CD04079
:10289000CD56DE4F88819981AA81BB81C359D14031
:1028A000CD53DF4F88839983AA83BB83C35CD04019
:1028B000AE014F5F5F4FBE016F577F4FCE018F5309
:1028C0009F4F0E94E5623FC01A830983CD57DE4FB8
:1028D00088819981AA81BB81C358D1408B839C8315
:1028E000AD83BE83CF57DF4F19830883C158D040D3
:1028F000CD56DE4F88819981AA81BB81C359D140D1
:10290000CD57DF4F88839983AA83BB83C358D040B8
:10291000BE016F5F7F4FCE018F579F4F0E9437637D
:1029200012C01A830983CD56DE4F88819981AA810E
:10293000BB81C359D1408B839C83AD83BE83CE01C1
:1029400001960E94826386E398E00E94C65F2FC1D1
:102950006DE973E086E398E00E94CA5F0FB6F894D1
:10296000A89580916000886180936000109260005B
:102970000FBE8091E6089091E708009711F00E9441
:102980006D7286E690E00E94D5718C0186E6D801D2
:102990001D928A95E9F7C801855B9F4F0E945B44B1
:1029A0001093E7080093E6088091E8088093DB081D
:1029B00080910502882319F00E945B2B06C069EB09
:1029C00073E086E398E00E94D73C26E030E045E7DC
:1029D00057E064E089E090E00E94CA428DE693E00F
:1029E0009A8389831B821C821D821E82CE010396DC
:1029F0000E94C54660E08EE290E00E94A84280FFFF
:102A000090C08091E6089091E708FC0116A217A2F9
:102A100010A611A612A613A614A615A616A617A6EA
:102A200010AA11AA12AE13AE14AE15AEFE9640EE69
:102A30005EE260E070E0408351836283738334968A
:102A400040EA5FE060E070E040835183628373831B
:102A5000F49724E1DF011D922A95E9F726E0E5E7E6
:102A6000F7E0DC01189601900D922A95E1F7FC0140
:102A7000E65BFF4F10820E94925B7C01019709F098
:102A800050C06091E6087091E708625F7F4FCE0109
:102A900001960E94CC5FCE0103960E94C5466091CC
:102AA000E6087091E708665E7F4FCE0101960E94AE
:102AB000CC5FCE0103960E94D5466091E6087091E6
:102AC000E7086A5E7F4FCE0101960E94CC5FCE017F
:102AD00003960E94CD466091E6087091E7086E5D0E
:102AE0007F4FCE0101960E94CC5F8B819C81AD818E
:102AF000BE818093DE089093DF08A093E008B09336
:102B0000E108E091E608F091E708828993899093C3
:102B1000E3088093E208848995899093E50880937F
:102B2000E40899E288E10FB6F894A89580936000D4
:102B30000FBE90936000A895EF2819F568EC76E039
:102B400086E398E00E94A35E69E976E086E398E078
:102B50000E94A35E86EF9FEF90939305809392056A
:102B60000E941265DC01CB01805A9541AF4FBF4FE7
:102B70008093E0069093E106A093E206B093E3060B
:102B8000FCC069E876E086E398E00E94A35E8DE6EB
:102B900093E09A8389831B821C821D821E82CE0150
:102BA00003960E94873FCE0101960E94313F81E04B
:102BB00090E0DFC080918A0581111AC060E070E06A
:102BC00080E090E00E94F330D4C00E941265009132
:102BD000E0061091E1062091E2063091E306061727
:102BE000170728073907D0F10E9414558111C5C075
:102BF00082E090E0BEC0A895CF55DE4F1882C15A42
:102C0000D140FE01EF56FE4F119211928EE0DF018E
:102C10001D928A95E9F70091F4061091F5060115C9
:102C2000110529F0C8010E945F5481118AC20E94D7
:102C300014558111A2C00091F4061091F5060115FA
:102C4000110509F49AC0C8010E945F54E82EF12CC6
:102C5000B2E0EB16F1040CF091C28FC020E030E03E
:102C600043E050E060E48E010F5F1F4FC8010E94F7
:102C70007F4966EC73E0C8010E94C680F8010190AC
:102C80000020E9F7CF01801B910B08968138910550
:102C900038F50E941455882319F180916F0990919D
:102CA0007009019611F481E090E09093700980938F
:102CB0006F0980916F09909170099093F408809347
:102CC000F50847E050E06FEE78E0C8010E948B54B1
:102CD000AC01455051096FEE78E082EA0E94AB5496
:102CE00083E090E0909393058093920560EE78E006
:102CF00086E398E00E94A35E40C00E9412650091A6
:102D0000E0061091E1062091E2063091E3060617F5
:102D100017072807390788F5109293051092920536
:102D20002CC00E9412650091E0061091E1062091EE
:102D3000E2063091E306061717072807390708F45B
:102D400057CF1BC00E947A38892B09F051CF0E94BF
:102D50001265DC01CB0188579C4EAF4FBF4F80936B
:102D6000E0069093E106A093E206B093E30686EFB7
:102D70009FEF90939305809392050FB6F894A895D2
:102D800080916000886180936000109260000FBEA7
:102D90008091920590919305181619060CF0ABC11D
:102DA00060E08EE290E00E94A84280FF51C1009155
:102DB000E6081091E7080115110509F49CC10E946D
:102DC00012654B015C01F80182AD93ADA4ADB5ADC8
:102DD00098012A5B3F4F7901892B8A2B8B2B09F4B1
:102DE000AEC0F90180819181A281B381A5019401D6
:102DF000281B390B4A0B5B0BCA01B90157FD64C094
:102E000028EE33E040E050E00E94467CCE55DE4F95
:102E1000688379838A839B83C25AD1402401350118
:102E200088EE480E83E0581E611C711CCE55DE4FA3
:102E300088819981AA81BB81C25AD140481A590A16
:102E40006A0A7B0AD7014D925D926D927C9213972C
:102E5000BA01A9014F5F5F4F6F4F7F4FF80182A901
:102E600093A9A4A9B5A96A017B01CC0CDD1CEE1CB9
:102E7000FF1C8C159D05AE05BF052CF412AA13AAE4
:102E800014AA15AA09C0841B950BA60BB70BF80151
:102E900082AB93ABA4ABB5ABF80186A997A9A0AD63
:102EA000B1AD8C159D05AE05BF052CF416AA17AA69
:102EB00010AE11AE09C0841B950BA60BB70BF80121
:102EC00086AB97ABA0AFB1AF6801FAE4CF0ED11CCF
:102ED000D6018C91833099F4F80182A993A9A4A911
:102EE000B5A9181619061A061B064CF084E0D6017F
:102EF0008C93C8010E94925B01967C0102C0E12C78
:102F0000F12CF6018081833011F0811125C0F80188
:102F100086A997A9A0ADB1AD181619061A061B0609
:102F2000DCF0D6011C9284E13E96DF011D928A9569
:102F3000E9F7C8010E94925B03967C010DC0D501A0
:102F4000C40188519C4FAF4FBF4FF90180839183DB
:102F5000A283B383E12CF12CD801DA968D929D9255
:102F6000AD92BC92DD97B2E0EB16F10429F0E4E0FB
:102F7000EE16F10409F050C06091E6087091E70880
:102F8000625F7F4FCE0101960E94CC5FCE01039617
:102F90000E94C5466091E6087091E708665E7F4F23
:102FA000CE0101960E94CC5FCE0103960E94D546C9
:102FB0006091E6087091E7086A5E7F4FCE01019646
:102FC0000E94CC5FCE0103960E94CD466091E60838
:102FD0007091E7086E5D7F4FCE0101960E94CC5F35
:102FE0008B819C81AD81BE818093DE089093DF0848
:102FF000A093E008B093E108E091E608F091E708BB
:10300000828993899093E3088093E2088489958963
:103010009093E5088093E408F3E0EF16F10409F4D7
:1030200051C064F431E0E316F10451F142E0E416DA
:10303000F10409F060C067EA78E049C054E0E516A1
:10304000F10409F442C085E0E816F10409F053C028
:1030500068ED78E086E398E00E94A35E86E398E05E
:103060000E94C65F0E94145581110E948F3F0E94EA
:103070001265DC01CB01805D9A48AF4FBF4F13C092
:1030800064EC78E086E398E00E94A35E0E94145509
:1030900081110E948F3F0E941265DC01CB01885193
:1030A0009C4FAF4FBF4F8093E0069093E106A093F3
:1030B000E206B093E30686EF9FEF9093930580932B
:1030C000920519C064E978E0DDCF68E778E086E32F
:1030D00098E00E94A35E8DE693E09A8389831B8229
:1030E0001C821D821E82CE0103960E94873FCE0164
:1030F00001960E94313F99E288E10FB6F894A895B5
:10310000809360000FBE9093600080919205909133
:103110009305CB55DE4F0FB6F894DEBF0FBECDBF83
:10312000DF91CF911F910F91FF90EF90DF90CF90A3
:10313000BF90AF909F908F907F906F905F904F90D7
:10314000089560E0C8010E948C67DC0119960D911A
:103150001C911A971093FD060093FC066BE678E02D
:1031600086E398E00E94A35EB80186E398E00E949F
:10317000CA5F86E398E00E94C65F59CD61E0C8014E
:103180000E948C67FC0161847284F2E0EF16F10406
:10319000A9F062E0C8010E948C67FC0181849284DE
:1031A000F3E0EF16F10471F063E0C8010E948C6750
:1031B000DC0119960D911C911A9707C08BE5882E9A
:1031C00087E0982E8E010F551E4F40E150E0BE0162
:1031D0006F567E4F86E390E00E947A30892B51F43F
:1031E000B5E0EB16F1040CF01CC3FE01EF56FE4FE8
:1031F0007F0104C09E012F563E4F790170928309D2
:103200006092820990928509809284098CE99AE4FF
:1032100090937B0980937A095E013FE7A31A3EEF02
:10322000B30A40E150E06EE378E0C5010E94FA7411
:103230006E014FE9C41A4EEFD40A20E030E041E0BD
:1032400050E060E2C6010E947F4940E250E067E33F
:1032500078E0C6010E94DC7467E178E086E398E0DC
:103260000E94A35EB30186E398E00E94CA5F65E115
:1032700078E086E398E00E94A35E4AE050E0B40163
:1032800086E398E00E946D5F6EE078E086E398E068
:103290000E94A35EB80186E398E00E94CA5F69E0DD
:1032A00078E086E398E00E94A35ED8018C918111BA
:1032B00004C0E12CF12C00E010E08090FC0690901E
:1032C000FD060E94145581113BC1609182097091E5
:1032D00083098091ED089091EE0840918409509106
:1032E0008509DC01ED91FC916115710521F00088E3
:1032F000F189E02D16C00684F785E02D2DE633E038
:103300003A83298340907E0950907F09609080091C
:10331000709081094B825C826D827E82BE016F5FFC
:103320007F4F19958130910509F003C19093700981
:1033300080936F0987E0E3E1F2E0DE0111960190EE
:103340000D928A95E1F7FE013196A4EFB8E0CE0127
:10335000089621912D93E817F907D9F70115110562
:1033600029F0E114F10421F086EF03C086E301C0E7
:1033700086EB8093FB081092FC088FE08093FD0899
:10338000F40101900020E9F7CF01881999094096CE
:103390008138910508F0C1C04FE050E06FEE78E051
:1033A000C4010E948B54F60101900020E9F7319787
:1033B000EC19FD09E80FF91F3296E138F10508F024
:1033C000ACC0AC016FEE78E0C6010E948B54F501F1
:1033D00001900020E9F73197EA19FB09E80FF91F7E
:1033E0003296E138F10508F098C0AC016FEE78E054
:1033F000C5010E948B540115110579F1F801019066
:103400000020E9F73197E01BF10B9C012E5F3F4F45
:10341000E20FF31FE138F10508F07FC0AC016FEE59
:1034200078E0C8010E948B54E114F104B1F0F70177
:1034300001900020E9F73197EE19FF099C012E5FFA
:103440003F4FE20FF31FE138F10508F066C0AC0111
:103450006FEE78E0C7010E948B54AC0145505109D2
:103460006FEE78E080E10E94AB540E941265609399
:103470007109709372098093730990937409609332
:1034800075097093760980937709909378098091F4
:10349000ED089091EE08DC01ED91FC910084F1853E
:1034A000E02D1995892BC1F40E94126500917509D0
:1034B000109176092091770930917809DC01CB01D0
:1034C000801B910BA20BB30B88399A43A105B10560
:1034D000F0F28CEF9FEF1DC0CE018F579F4F0E94DF
:1034E000E93C0497D1F48091F208811111C00E9447
:1034F00012656093750970937609809377099093AC
:10350000780910927909109289091092880918C0D7
:1035100090E090938909809388098091ED089091BB
:10352000EE08DC01ED91FC910488F589E02D1995F8
:103530008BC18EEF9FEF909389098093880984C196
:103540000091FC061091FD066BEF77E086E398E0B2
:103550000E94A35EB80186E398E00E94CA5F86E3FA
:1035600098E00E94C65F81E080938A0520E030E009
:1035700043E050E060E4CE018F5F9E4F0E947F49A0
:1035800066EC73E0CE018F5F9E4F0E94C680CE0135
:103590008F5F9E4F0E94095920E030E042E050E0EA
:1035A00060E4CE018F5F9E4F0E947F496AEC73E01A
:1035B000CE018F5F9E4F0E94C680BE016F5F7E4F1F
:1035C00086E398E00E94D73CCE018F5F9E4F0E9419
:1035D000095920E030E041E050E060E4CE018F5F27
:1035E0009E4F0E947F496AEC73E0CE018F5F9E4F31
:1035F0000E94C680BE016F5F7E4F86E398E00E9406
:10360000D73CCE018F5F9E4F0E940959FE01EF53B8
:10361000FF4F119211921EE3DF01212F1D922A9577
:10362000E9F71A821982FE0133968EE7DF011D92B7
:103630008A95E9F720E030E041E050E060E4CE0117
:103640008F539F4F0E947F4940E450E067E378E04A
:10365000CE018F539F4F0E94DC7440E850E064EB32
:1036600077E0CE0101960E94FA74BE016F5F7F4F32
:10367000CE018F539F4F0E949D5520E030E041E0E6
:1036800050E060E4CE018F539F4F0E947F4940E499
:1036900050E06EEA77E0CE018F539F4F0E94DC74BA
:1036A00040E850E064EA77E0CE0101960E94FA74A7
:1036B00040E850E061E977E0CE0101960E94DC74B9
:1036C000BE016F5F7F4FCE018F539F4F0E949D556C
:1036D00020E030E041E050E060E4CE018F539F4FA6
:1036E0000E947F4940E450E063EC79E0CE018F53C3
:1036F0009F4F0E94DC7440E850E061E877E0CE0123
:1037000001960E94FA74BE016F5F7F4FCE018F5306
:103710009F4F0E949D5520E030E041E050E060E482
:10372000CE018F539F4F0E947F4940E450E06AE7EB
:1037300077E0CE018F539F4F0E94DC7440E850E049
:1037400064E777E0CE0101960E94FA74BE016F5FD4
:103750007F4FCE018F539F4F0E949D55A0917307BD
:10376000B0917407109709F443C080911A029091A8
:103770001B02AE014F5B5E4FFA01819391932EE1E4
:1037800011922A95E9F79E012F573F4FF901819336
:10379000919311921A95E9F716960D911C9117972E
:1037A000E0907307F0907407E114F10471F00115D3
:1037B000110559F0D80118968C918530A9F7C801E8
:1037C0000E945F54882381F36DC020E030E041E027
:1037D00050E060E4CE018F539F4F0E947F4940E448
:1037E00050E067E177E0CE018F539F4F0E94DC7479
:1037F00084E090E090939305809392050E94126577
:10380000DC01CB0188579C4EAF4FBF4F8093E00641
:103810009093E106A093E206B093E3066EED77E0A5
:1038200067CA64E08091F4069091F5060E948C6767
:10383000DC011996ED90FC901A976BE478E086E332
:1038400098E00E94A35EDACC009188091091890962
:1038500062ED77E086E398E00E94A35E4AE050E0E4
:10386000B80186E398E00E946D5F6AEB77E086E33B
:1038700098E00E94A35E86E398E00E94C65F0E94E3
:103880001265DC01CB0188579C4EAF4FBF4F809330
:10389000E0069093E106A093E206B093E3068CE085
:1038A00090E067CA60E0C8010E948C67FC018185D6
:1038B0009285A385B4858A30910508F463C020E021
:1038C00030E041E050E060E4CE018F539F4F0E9412
:1038D0007F49F8016081718140E450E0CE018F534F
:1038E0009F4F0E94EC806CEC73E0CE018F539F4F92
:1038F0000E94C68040E450E066E277E0CE018F533C
:103900009F4F0E94DC74BE016F5B7E4FCE018F53D0
:103910009F4F0E949D55CF57DF4F8881C158D0409F
:10392000882361F120E030E041E050E060E4CE0126
:103930008F539F4F0E947F49D8016D917C9140E445
:1039400050E0CE018F539F4F0E94EC806CEC73E0EF
:10395000CE018F539F4F0E94C68040E450E06EE13D
:1039600077E0CE018F539F4F0E94DC74BE016F57EA
:103970007F4FCE018F539F4F0E949D55F8010281CA
:1039800013810ECFFC0140E250E08827E054FF4F46
:103990008F4F0C94877C6EE677E0CE018F5B9E4F55
:1039A0000E94FA74CF57DF4F1882C158D04087CF9A
:1039B00069E677E0CE018F5B9E4F0E94FA7440E487
:1039C00050E068E477E017C062E477E0CE018F5BF7
:1039D0009E4F0E94FA7440E450E06EE377E00BC023
:1039E00066E377E0CE018F5B9E4F0E94FA7440E45D
:1039F00050E060E377E0CE018F579F4F0E94FA744A
:103A00005ECFBC018230910508F40895613E8EE1DD
:103A1000780748F49B0195E0369527959A95E1F74C
:103A200048E0420F01C04FEF91E0242F30E0290F12
:103A3000311D35952795229FF001239FF00DF00D44
:103A400011246E177F0718F44FEF420F04C02F3F69
:103A500039F091E0920F491740F78FEF890F0895E1
:103A60008FEF0895CF93DF93009709F440C0FC01D6
:103A700020812223E1F1EC0169ED70E10E94CC7418
:103A8000892B31F16DEB70E1CE010E94CC74892B52
:103A900011F16EE17AE0CE010E94CC74892BF1F035
:103AA0006FE47AE0CE010E94CC74892BD1F06BE4F4
:103AB0007AE0CE010E94CC74892BB1F06AE17AE001
:103AC000CE010E94CC74892B91F485E090E011C066
:103AD00082E090E00EC081E090E00BC086E090E0D4
:103AE00008C083E090E005C084E090E002C080E080
:103AF00090E0DF91CF9108952F923F924F925F9285
:103B00006F927F928F929F92AF92BF92CF92DF92ED
:103B1000EF92FF920F931F93CF93DF93CDB7DEB752
:103B20002F970FB6F894DEBF0FBECDBF4C018B01AF
:103B30004C876901672B09F46AC32115310509F126
:103B4000D9018C918823E9F06FE270E0C9010E94ED
:103B50001981009751F0FC011192CF010E94321D92
:103B60007C015FE0652E712C10C0C6010E94321DE1
:103B70007C014FE0642E712C892B39F0C12CD12CA3
:103B800004C0612C712CE12CF12C5801D5018C91D1
:103B9000882349F0082E000C990B0E947280F501D1
:103BA00081935F01F3CFD801BC90BDE2BB1609F44D
:103BB000CAC080ED8B0D8A3008F4C5C061E071E1A8
:103BC000C8010E94CC74892B09F4E8C06DEF70E144
:103BD000C8010E94CC74892B09F4E4C063EB7AE03D
:103BE000C8010E94CC74892B09F4B0C06CEA7AE059
:103BF000C8010E94CC74892B09F4ACC067EA7AE052
:103C0000C8010E94CC74892B09F4A8C063EA7AE049
:103C1000C8010E94CC74892B09F4A4C06EE97AE033
:103C2000C8010E94CC74892B09F4A0C066EC70E135
:103C3000C8010E94CC74892B09F49CC061EC70E12E
:103C4000C8010E94CC74892B09F498C06BEC70E118
:103C5000C8010E94CC74892B09F494C065E97AE00C
:103C6000C8010E94CC74892B09F490C061E97AE004
:103C7000C8010E94CC74892B09F48CC06CE87AE0EE
:103C8000C8010E94CC74892B09F488C066E87AE0E8
:103C9000C8010E94CC74892B09F484C06EE77AE0D5
:103CA000C8010E94CC74892B09F478C065E77AE0DA
:103CB000C8010E94CC74892B09F474C06CE67AE0C8
:103CC000C8010E94CC74892B09F470C063E67AE0C5
:103CD000C8010E94CC74892B09F46CC06EE57AE0AF
:103CE000C8010E94CC74892B09F468C067E57AE0AA
:103CF000C8010E94CC74892B09F464C063E57AE0A2
:103D0000C8010E94CC74892B09F460C0EBE7BE1691
:103D100009F460C0F3E2BF1609F461C043E050E06B
:103D20006FE47AE0C8010E94EC74892B09F45CC04E
:103D300043E050E06BE47AE0C8010E94EC74892B08
:103D400009F057C04CC0A12CB12C56C033E0A32EB3
:103D5000B12C52C024E0A22EB12C4EC095E0A92E69
:103D6000B12C4AC086E0A82EB12C46C0B7E0AB2EDD
:103D7000B12C42C0AAE0AA2EB12C3EC0FBE0AF2E6F
:103D8000B12C3AC0ECE0AE2EB12C36C07DE0A72EAF
:103D9000B12C32C06EE0A62EB12C2EC0AA24A39462
:103DA000B12C2AC042E0A42EB12C26C038E0A32EAC
:103DB000B12C22C029E0A22EB12C1EC090E1A92E68
:103DC000B12C1AC081E1A82EB12C16C0B2E1AB2EE5
:103DD000B12C12C0AEEFAA2EBB24BA940DC0FDEFD9
:103DE000AF2EBB24BA9408C0ECEFAE2EBB24BA941D
:103DF00003C0AA24AA94BA2C68EB7AE086E398E080
:103E00000E94A35E4AE050E0B50186E398E00E947C
:103E10006D5F86E398E00E94C65F2FEFA216B206A0
:103E200009F094F43EEFA3163FEFB3060CF0EEC199
:103E30008CEFA8168FEFB80659F09DEFA9169FEFEB
:103E4000B90609F458C0D5C1A114B10421F0D1C1FB
:103E500063E0E62EF12CDE011196BB87AA87A12C28
:103E6000B12CBA85BE87EB85EF8725012FEF421A6B
:103E7000520A5201D8018C918823E9F0F8013E2EB4
:103E80001F2F8191882329F08D3219F080538A30B9
:103E9000B0F7832D912F0E94A574282E9D876CE288
:103EA00070E0832D912F0E94D1808C01892B31F0FD
:103EB0000F5F1F4F03C080E090E002C0822D9D8500
:103EC000EA85FB8581939193FB87EA8701151105AC
:103ED00039F0F3E04F16510441F653E0A52EB12C12
:103EE000D401ED91FC910190F081E02D0C852E859F
:103EF0003F85A5017AC1CE0107969E01275F3F4FFE
:103F00003F932F93215031093F932F939F938F938A
:103F10008DE494E09F938F931F930F930E94908161
:103F20000FB6F894DEBF0FBECDBF039709F06EC188
:103F30001F81B8840985812FB11608F48B2DA02E1E
:103F4000801708F4A82E1A19BA180A199A2D9095F4
:103F50009F3F39F080E090950E94011D80958A87EF
:103F600002C0FFEFFA878B2D90E0810F911D800F2B
:103F7000911D892B29F4FA84F0941A8600E0FDC083
:103F80002A852F3FF1F0211102C031E03A878A855E
:103F9000282F30E040E050E06FEF7FEF80E090E0CE
:103FA0000E94467CA12FB0E00E94657C172FAB2DAC
:103FB000B0E00E94657CB72EA02FB0E00E94657C27
:103FC000072FEB2CF12CE10EF11CE00EF11C9FEF02
:103FD000E916F104FCF4E114F10419F4EE24E3947D
:103FE000F12C970140E050E06FEF7FEF80E090E030
:103FF0000E94467CA12FB0E00E94657C172FAB2D5C
:10400000B0E00E94657CB72EA02FB0E00E94657CD6
:10401000072F05C0AFEFEA16F10409F06CF42A2D62
:104020003E2D230F08F42FEF922F2F3F29F080E031
:104030000E94011DF82E02C0FF24FA94802F011760
:1040400008F4812F8B1508F48B2D81132FC0B1102C
:104050000DC0082F20E8021B08F400E020E6029FB4
:10406000000E00E0011D1124005386C02B2D30E00E
:10407000482F50E0421B530B2417350744F40B2DF7
:1040800020E6029F000E00E0011D112475C006E528
:104090000B0D081B24E0021B08F400E020E6029F41
:1040A000000E00E0011D1124005E66C08B1139C0B6
:1040B00001111BC03BEA032F011B08F400E0202F75
:1040C0004FE2249F020E20E0211D1124482F431BA4
:1040D00008F440E0042F30E6039F000E00E0011DCD
:1040E0001124020F0695005C47C0202F30E090E0BD
:1040F000821B930B2817390744F420E6029F000E19
:1041000000E0011D1124005A37C025E5021B08F408
:1041100000E020E3029F000E00E0011D1124005882
:104120002BC011110CC020E8021B08F400E020E3B2
:10413000029F000E00E0011D112408571DC0212F11
:1041400030E0802F90E0821B930B012F2817390756
:1041500044F420E6029F000E00E0011D11240056E9
:104160000BC025E5021B08F400E020E6029F000ECC
:1041700000E0011D112400540F5F202F30E0ADE658
:10418000B1E00E94787C212C312C21012A94A201DB
:1041900091010E94467C3A8329838A85282F30E04A
:1041A000A4E6B0E00E94787CA20191010E94467CC6
:1041B0003C832B832F2D30E0A4E6B0E00E94787C76
:1041C000A20191010E94467C3E832D83D401ED9192
:1041D000FC910190F081E02D33E0E32EF12C0C8571
:1041E0009E012F5F3F4F43E050E0B301C40119959A
:1041F00010C0D401ED91FC910190F081E02D0C856F
:1042000020E030E040E050E0B501F0CF02C080E0B7
:1042100090E02F960FB6F894DEBF0FBECDBFDF91B2
:10422000CF911F910F91FF90EF90DF90CF90BF90B3
:10423000AF909F908F907F906F905F904F903F9046
:104240002F9008958F929F92AF92BF92CF92DF925C
:10425000EF92FF920F931F93CF93DF93E091730739
:10426000F0917407309709F468C0812EC02F932E07
:10427000C22EA52ED42EB72ED62FBC01CF010E9460
:10428000BD508C01009709F45BC0DC0118968C913D
:10429000853009F055C060E0C8010E948C677C0140
:1042A00061E0C8010E948C67FC0101851285D7017D
:1042B00019962D913C911A972130310569F02CF413
:1042C000232BF1F56C2FC80118C02230310549F0BD
:1042D00027303105A9F034C06C2FC80103960E9425
:1042E000C9476D2FC8010E94C9476D2DC8010196AD
:1042F0000E94C9476C2DC80102960E94C94720C080
:10430000892BF1F080858530D9F4E680F780E114BF
:10431000F104B1F00C2F182D2C2D392D4D2D5A2DC7
:104320006D2F7B2DF701818592850E942221D70177
:104330001296ED90FC901397EACF80E090E002C0D7
:1043400081E090E0DF91CF911F910F91FF90EF906E
:10435000DF90CF90BF90AF909F908F900895CF92B5
:10436000DF92EF92FF920F931F93CF93DF93E09131
:10437000F806F091F9063097A1F09085953089F410
:1043800069017A01EB01682FCF010E948C67FC0163
:1043900081859285009729F09601A701BE010E94B0
:1043A0002221DF91CF911F910F91FF90EF90DF902D
:1043B000CF900895AF92BF92CF92DF92EF92FF928B
:1043C0000F931F93CF93DF938091F1069091F206A4
:1043D000892B09F472C0E1E0F0E0C0E0D0E0CC2429
:1043E000C394D12CB6010C2E02C0660F771F0A941D
:1043F000E2F74091DD055091DE057F0184E0E80E93
:10440000F11CCF01B12C9C01A0910702B0910802D0
:10441000A817B90720F42091070230910802A09153
:104420008C07B0918D07A20FB31FAC90A091F1063D
:10443000B091F2069C0121503109A20FB31F0A2D41
:1044400010E02C9130E00217130729F0462B572B70
:10445000AC92BB24B3940196E816F906A1F65093EA
:10446000DE054093DD05BB2011F18091F1069091AE
:10447000F206E80FF91F028110E0218130E040814F
:1044800050E03197608170E0CE010E94AF210E9420
:104490001265DC01CB01845D9E4FAF4FBF4F80930F
:1044A000D9059093DA05A093DB05B093DC0521963E
:1044B000F701C430D10509F095CFDF91CF911F915D
:1044C0000F91FF90EF90DF90CF90BF90AF90089545
:1044D000DC011296ED91FC911397309721F081E069
:1044E0009085953009F080E00895CF92DF92EF92A9
:1044F000FF92CF93DF93DC011696ED91FC91179715
:10450000309721F12085223009F56A017B01EC0109
:1045100063E47AE086E398E00E94A35E6DE37AE0CC
:1045200086E398E00E94A35E2AE030E0B701A6018E
:1045300086E398E00E94255F86E398E00E94C65FCC
:10454000EE81FF81C186D286E386F486DF91CF912A
:10455000FF90EF90DF90CF900895FC0186819781C6
:10456000009789F0FC012085223041F0253059F474
:1045700060E00E948C67009731F0FC0161857285D4
:1045800083859485089560E070E0CB0108950F93D2
:104590001F93CF93DF93FC01C481D581209791F0C5
:1045A0008885823029F4672B69F489859A8514C03F
:1045B000853041F48B01CE010E945F5490E00817D2
:1045C00019071CF080E090E007C0602FCE010E9428
:1045D0008C67FC0181859285DF91CF911F910F91AE
:1045E00008950F931F93CF93DF93EB0163E0FC01DA
:1045F000828193810E948C67009759F1AE014095AA
:1046000050954F6F506F052E000C660B770BFC0119
:10461000018512852385348540235123622373232A
:10462000418752876387748764E37AE086E398E082
:104630000E94A35E4AE050E0BE0186E398E00E943B
:104640006D5F86E398E0DF91CF911F910F910C94FD
:10465000C65FDF91CF911F910F9108950F931F9324
:10466000CF93DF93EB0163E0FC01828193810E9491
:104670008C67009749F1AE0144275F70052E000C4E
:10468000660B770BFC010185128523853485402B51
:10469000512B622B732B41875287638774876BE2A0
:1046A0007AE086E398E00E94A35E4AE050E0BE0113
:1046B00086E398E00E946D5F86E398E0DF91CF91FA
:1046C0001F910F910C94C65FDF91CF911F910F91B5
:1046D0000895CF93DF93EB0163E0FC018281938126
:1046E0000E948C67009741F0FC01818592858827A4
:1046F0009F708C239D2300C0DF91CF910895CF93AD
:10470000C62F63E0FC01828193810E948C67009731
:1047100001F1FC01418552856385748544275F70F2
:10472000662777274C2B418752876387748763E21C
:104730007AE086E398E00E94A35E4AE050E06C2FA6
:1047400086E398E00E94745F86E398E0CF910C9432
:10475000C65FCF91089563E0FC01828193810E943E
:104760008C67009719F0FC01818508958FEF0895FB
:10477000BF92CF92DF92EF92FF920F931F93CF934E
:10478000DF93EC010E946822882309F441C08A81EA
:104790009B810E945F54082F10E0C801880F991F69
:1047A0009C012A593D4F790132E0B32E04301105A6
:1047B000D4F4F701C190D1907F010E946F2A009735
:1047C00051F0FC01B086A601DD0C660B770B41872A
:1047D000528763877487BC018A819B810E94D8506D
:1047E0000F5F1F4FE3CF0A811B8160E0C8010E9469
:1047F0008C67FC018185888761E0C8010E948C6715
:104800009D838C8362E0C8010E948C679F838E83A6
:10481000DF91CF911F910F91FF90EF90DF90CF909C
:10482000BF900895CF93DF93EC01FB012481358184
:1048300040815181628173810E94255FCE01DF91A9
:10484000CF9108958F929F92AF92BF92CF92DF92B5
:10485000EF92FF920F931F93CF93DF93CDB7DEB705
:10486000C054D1090FB6F894DEBF0FBECDBF8C0186
:104870005B01FC01F38066E17AE086E398E00E9448
:10488000A35E4AE050E06F2D86E398E00E94745FDB
:1048900064E17AE086E398E00E94A35E4AE050E09B
:1048A000B50186E398E00E946D5F86E398E00E9480
:1048B000C65FF801C080D18068E574E0C6010E943F
:1048C000BD504C016DE574E0C6010E94BD508C01E5
:1048D00062E674E0C6010E94BD507C0167E674E0A8
:1048E000C6010E94BD506C010097D1F0FC016185AA
:1048F000728540E450E0CE0101960E940A810E9438
:104900001455882369F080918D05882309F452C0DD
:1049100007C0F80161857285FB01808181116EC03D
:104920008114910409F46FC0F40161857285CE0190
:1049300001960E946D54CE0101960E946822882340
:10494000A1F1AB2889F00115110561F4C12CD12C1E
:10495000E12CF12C01E020E030E040E050E061E0AB
:1049600070E010C0F80114C0E114F10481F4C12C0E
:10497000D12CE12CF12C01E020E030E040E050E0CF
:1049800062E070E0CE0101960E9481090EC0F7013D
:1049900061857285FB018081882339F020E030E059
:1049A00041E0CE0101960E947C1DCE0101960E943D
:1049B0002F5129C06FE270E0CE0101960E94D18094
:1049C000892B51F4F6012185328543E050E060E403
:1049D000CE0101960E947F49A114B10439F001155E
:1049E000110509F096CF6CE674E008C0E114F104FB
:1049F00019F46FE674E002C0F7018CCFCE01019686
:104A00000E949D558DCFC05CDF4F0FB6F894DEBF7E
:104A10000FBECDBFDF91CF911F910F91FF90EF900F
:104A2000DF90CF90BF90AF909F908F900895FF92AE
:104A30000F931F93CF93DF93EC011D821C821A8288
:104A40001B82088119810115110509F456C0F8016E
:104A50008085863009F051C08091E4069091E5068A
:104A6000892B09F44AC063E774E0C8010E94BD5075
:104A7000009719F0FC0181858A83F801808191817A
:104A80000E94A574F82E8B8365E774E0C8010E942C
:104A9000BD50009779F51A816FE07AE086E398E0DF
:104AA0000E94A35E4AE050E06F2D86E398E00E94EA
:104AB000745F6DE07AE086E398E00E94A35E4AE0CE
:104AC00050E0612F86E398E00E94745F86E398E0EF
:104AD0000E94C65F40E050E065E774E088819981FC
:104AE0000E94F55065E774E0888199810E94BD506D
:104AF000009719F009969D838C83DF91CF911F91C8
:104B00000F91FF900895EF92FF920F931F93CF9311
:104B1000DF938091DD059091DE05C4E0D0E021E0D7
:104B200030E0AC0142235323452B29F0A9014095E5
:104B3000509584239523220F331F219791F790934B
:104B4000DE058093DD050E9412650091D905109164
:104B5000DA052091DB053091DC05601771078207CB
:104B6000930708F459C0012B022B032B09F454C0FE
:104B70001092D9051092DA051092DB051092DC052F
:104B8000E12CF12CE091F106F091F206EC0FFD1F03
:104B9000038110E0228130E0418150E0608170E0CB
:104BA000C7010E94AF218FEFE81AF80A249684E02B
:104BB000E816F10439F7C1E0D0E080910702909146
:104BC00008028C179D0728F4809107029091080233
:104BD00001C0CE0120918C0730918D07F901E80FBB
:104BE000F91F4AE050E0608186E398E00E94745F1C
:104BF00067E774E086E398E00E94CA5F2196C131BE
:104C0000D105D9F686E398E0DF91CF911F910F91FE
:104C1000FF90EF900C94C65FDF91CF911F910F91A1
:104C2000FF90EF900895CF93DF93EC01E881F98135
:104C30000284F385E02DCE0119950196B9F7DF9135
:104C4000CF910895FC01A285B3851097A9F08685C0
:104C50009785029788F0CD010196938782876C93A0
:104C6000868597850197978786870284F385E02D4F
:104C7000108281E090E0089580E090E00895FC01CA
:104C8000868197818F3F2FEF920729F02FEF3FEF1B
:104C9000378326830895A085B185109789F02485F0
:104CA00035852115310561F0CD0101969187808709
:104CB0008C912150310935872487082E000C990BDF
:104CC0000895FC0186819781019639F481E024855D
:104CD0003585232B19F480E0089581E00895CF9263
:104CE000DF92EF92FF920F931F93CF93DF937C019C
:104CF0006A018B01C0E0D0E0CC15DD0589F0D70159
:104D0000ED91FC910284F385E02DC70119958F3F49
:104D1000BFEF9B0729F0F80181938F012196ECCF1B
:104D2000CE01DF91CF911F910F91FF90EF90DF9017
:104D3000CF900895CF93C62FDC01ED91FC910088B0
:104D4000F189E02D1995DC01ED91FC910190F08144
:104D5000E02D6C2FCF911994CF93DF93EC018E81CE
:104D60009F810196D9F4288539858A859B85820F94
:104D7000931F81159041A0F4E881F9810284F385A5
:104D8000E02DCE011995813291056CF3E881F9810E
:104D90000684F785E02D682FCE01199581E001C0CA
:104DA00080E0DF91CF910895062E000C770BFC0177
:104DB000778366830895CF93DF93EC018E819F8183
:104DC000019611F5E881F9810088F189E02DCE0185
:104DD0001995DC01ED91FC910084F185E02D199588
:104DE000892BA1F0E881F9810284F385E02DCE01C1
:104DF00019958132910534F3E881F9810684F785AC
:104E0000E02D682FCE01199581E001C080E0DF918F
:104E1000CF9108950F931F93CF93DF93EC018B01F4
:104E200069E774E00E94CA5F01151105B9F1F80144
:104E300061918F01662391F1603220F0623211F0AE
:104E40006C3541F56CE5CE010E949C5EF80131970E
:104E500080818C30D1F044F48930D9F08A30B9F0B7
:104E6000883029F762E616C0823259F024F48D307A
:104E7000F1F662E70FC08F3231F08C35C1F66CE588
:104E800009C062E207C06FE205C066E603C06EE6D5
:104E900001C064E7CE010E949C5EC9CF62E2CE01F0
:104EA0000E949C5E80E090E0DF91CF911F910F9176
:104EB0000895FC012085318582859385AC014F5F83
:104EC0005F4F53874287820F931F0E94067C81E0C9
:104ED00090E00895FC01868197818F3F2FEF920724
:104EE00029F02FEF3FEF3783268308952085318502
:104EF00082859385AC014F5F5F4F53874287820F56
:104F0000931F0E94FE7B082E000C990B0895FC0154
:104F1000868197818F3F2FEF920729F02FEF3FEF88
:104F2000378326830895808591850C949E75CF9252
:104F3000DF92EF92FF92CF93DF93EC018E819F81FE
:104F40008F3F2FEF920759F02FEF3FEF3F832E83D4
:104F5000DF91CF91FF90EF90DF90CF9008950E9466
:104F600012656B017C01A4EFCA0EA1E0DA1EE11C00
:104F7000F11CE881F9810088F189E02DCE011995B5
:104F8000DC01ED91FC910084F185E02D1995892BD0
:104F900039F40E9412656C157D058E059F0548F356
:104FA000E881F9810088F189E02DCE011995DC01B5
:104FB000ED91FC910284F385E02DDF91CF91FF907C
:104FC000EF90DF90CF901994EF92FF920F931F9381
:104FD000CF93DF93009719F48FEF9FEF82C0FC010E
:104FE000E484F584D7010D911C91D801ED91FC91D9
:104FF0000688F789E02DC8011995882369F3D8013F
:10500000ED91FC910084F185E02DC8011995D8013E
:10501000ED91FC91892B61F30284F385E02DC801A9
:105020001995EC010196C1F2F8018589882339F0C0
:105030004AE050E06C2F86E398E00E94745FD7014D
:1050400012968C91882309F44BC0C532D10509F022
:1050500047C0D801ED91FC910084F185E02DC80195
:10506000199502975CF0D801ED91FC910688F789BB
:10507000E02DC80119958111ECCFAECFD1E0C0E091
:10508000D801ED91FC910284F385E02DC8011995BA
:105090008F3FBFEF9B0709F49FCF9C01215431093B
:1050A0002A31310530F09C01215631092A31310570
:1050B00038F48D2F8295807F829FC00D11240AC005
:1050C000C0978A30910530F49D2F9295907F989FDC
:1050D000C00D1124D150A0F68C2FCC0F990B01C01C
:1050E000CE01DF91CF911F910F91FF90EF90089526
:1050F0008F929F92AF92BF92CF92DF92EF92FF92E8
:105100000F931F93CF93DF936115710509F4FFC0CF
:10511000FB010085002E000C110B220B330B073016
:10512000110508F0F4C0DB01EC01F8018827E65313
:10513000FF4F8F4F0C94877C6BE774E006C0199685
:105140008C91882389F060E874E0CE01DF91CF91E3
:105150001F910F91FF90EF90DF90CF90BF90AF9095
:105160009F908F900C94C75E65E874E0EECF19961F
:105170004D915D916D917C911C972AE030E0CE01BC
:10518000DF91CF911F910F91FF90EF90DF90CF9023
:10519000BF90AF909F908F900C94255F1996CD9003
:1051A000DD90ED90FC901C9720E030E0A901C70154
:1051B000B6010E94127D87FF09C06BE874E0CE0142
:1051C0000E94CA5FF7FAF094F7F8F094C701B601AD
:1051D0000E94907D4B015C012AE0AB01BC01CE0135
:1051E0000E94DC5E6DE874E0CE010E94CA5FC501DA
:1051F000B4010E94BF7D9B01AC01C701B6010E94B2
:10520000A57C2DEC3CEC4CE45DE30E94A67C20E008
:1052100030E040E251E40E94767E0E94907DAB0136
:1052200060E070E02AE0CE010E94DC5E70C019965A
:105230006D917C911A97CE01DF91CF911F910F91C3
:10524000FF90EF90DF90CF90BF90AF909F908F90A6
:105250000C940A2716960D911C9117976BE5CE01B9
:105260000E949C5E019619F48FEF9FEF52C00115CA
:10527000110571F0B801CE010E9478280196A1F3C2
:10528000F801028113810115110589F36CE2E7CF62
:105290006DE52FC016960D911C9117976BE7CE0107
:1052A0000E949C5E019601F30115110509F1F801B8
:1052B00060817181CE010E940A270196A9F26AE3FA
:1052C000CE010E949C5E019679F2B801CE010E9447
:1052D0007828019649F2F801028113810115110520
:1052E00019F36CE2CE010E949C5E0196E9F6BCCFF8
:1052F0006DE7CE010E949C5E21E030E0019611F046
:1053000020E030E088279927821B930B02C080E0C1
:1053100090E0DF91CF911F910F91FF90EF90DF9080
:10532000CF90BF90AF909F908F900895CF93DF93D1
:10533000EC01E881F9810284F385E02DCE01199515
:105340008F3F2FEF920771F0E881F981813291054B
:1053500094F30684F785E02D682FCE01199580E03F
:1053600090E002C08FEF9FEFDF91CF910895EF9211
:10537000FF920F931F93CF93DF938C017B01DC018E
:10538000ED91FC910284F385E02D1995829709F047
:1053900078C084E0F701808786E090E00E94D571B4
:1053A000EC01892B09F46DC0E0EEF5E0F983E883A8
:1053B00080E091E0DF019C011D9221503040E1F737
:1053C0009B838A831D821C82D801ED91FC9102840B
:1053D000F385E02DC80119958F3FBFEF9B0709F4B6
:1053E0004DC08232910509F44FC0803291050CF412
:1053F0004BC08C35910511F0BE013DC0D801ED9137
:10540000FC910284F385E02DC80119958F3FBFEF11
:105410009B07A1F18236910531F15CF48F32910541
:10542000F9F08C359105C9F0829771F6BE0182E2E0
:1054300022C08E369105D1F034F48636910521F6DE
:10544000BE018CE018C08237910599F08437910530
:1054500009F0BACFBE0189E00EC0BE018CE50BC0D9
:10546000BE018FE208C0BE0188E005C0BE018AE02F
:1054700002C0BE018DE00E947162A6CFCE010E94E3
:105480006D728FEF9FEF24C08C819D81009749F052
:10549000E881F9818E0F9F1FFC013197808188235D
:1054A00021F0BE0180E00E9471628C819D810E948A
:1054B000D5718C01009739F060EE75E00E94E580AF
:1054C000CE010E946D72F7011287018780E090E0A3
:1054D000DF91CF911F910F91FF90EF9008958DE094
:1054E00090E00E94D571009729F02DE0FC01119207
:1054F0002A95E9F708950F931F93CF93DF930097B1
:10550000E1F0EC010C851D850115110579F0D8013C
:105510008D919C91009739F0DC01ED91FC9104880C
:10552000F589E02D1995C8010E946D72CE01DF91B9
:10553000CF911F910F910C943C75DF91CF911F91EA
:105540000F910895AF92BF92CF92DF92EF92FF92A8
:105550000F931F93CF93DF9300D01F92CDB7DEB789
:105560006115710509F496C06B01182FDB011C96BB
:10557000AD90BC901D97F501E080F180D701ED91D1
:10558000FC910688F789E02DC7011995811104C0A7
:10559000C6010E947B2A7EC0F5019281911114C040
:1055A000D701ED91FC910190F081E02D612FC701B1
:1055B0001995F7018589882309F469C0612F86E36D
:1055C00098E00E949C5E63C0812F8F7D81548A3158
:1055D00038F380ED810F8A3018F383ED810F82302C
:1055E000F8F21F35E9F21E37D9F21132B1F086EC2C
:1055F000810F823090F08AED810F873070F01D337B
:1056000061F0812F8F7E8F3241F08DED810F8230DE
:1056100020F01B3511F01D3511F491FFC1CF198217
:105620001A821B821C82812F012E000C990B9F93E2
:105630001F938FE894E09F938F938E010F5F1F4F0E
:105640001F930F930E9461816E01F4E0CF0ED11C75
:105650000F900F900F900F900F900F90D701ED913A
:10566000FC910190F081E02DD8016C91C701199552
:10567000F7018589882331F0D8016C9186E398E0A1
:105680000E949C5E0F5F1F4F0C151D0539F780E0CF
:1056900090E002C08FEF9FEF0F900F900F900F9050
:1056A000DF91CF911F910F91FF90EF90DF90CF90FE
:1056B000BF90AF900895CF93DF931092050260EDF5
:1056C00077E080E090E00E94D86461E08091DB08A0
:1056D0000E949C64CFB7F8948091DF05811127C0A8
:1056E000ECEFF1E18491E2E4F2E19491E82FF0E053
:1056F000EE0FFF1FED56FE4EA591B491EC91E923FC
:1057000021F461E085E30E946D6461E085E30E941D
:105710009C648CB580618CBD8CB580648CBD61E06F
:1057200084E30E949C6461E083E30E949C64809116
:10573000DF058F5F8093DF05CFBF60E080E090E002
:105740000E94A842482F406864E080E090E00E94F8
:10575000FC42C0E0DC2FD295DD0FD07ED45F42E06A
:105760006D2F8EE190E00E94FC4242E06D2F8FE1B0
:1057700090E00E94FC42CF5FC83061F7DF91CF918B
:105780000895DF92EF92FF920F931F93CF93DF93D1
:105790004115510539F18901EA01F62ED92EE82E7D
:1057A0008091D9089091DA080E94A5420E94664231
:1057B0008D2D0E949E428E2D0E949E428F2D0E9412
:1057C0009E427E01E00EF11ECE15DF0529F080E03D
:1057D0000E949E428993F8CF0E9461420E949D429E
:1057E000C80102C080E090E0DF91CF911F910F913E
:1057F000FF90EF90DF90089560E08DE00C946D6471
:1058000061E08DE00C946D642F923F924F925F9215
:105810006F927F928F929F92AF92BF92CF92DF92C0
:10582000EF92FF920F931F93CF93DF93CDB7DEB725
:10583000CD55D1090FB6F894DEBF0FBECDBF009194
:10584000E6061091E7060115110509F4A6C30E94AA
:105850001265C090EC06D090ED06E090EE06F09058
:10586000EF06C616D706E806F90608F054C0F80198
:105870000680F781E02D6D96FFAFEEAF6D979E012C
:105880002F5B3F4F69963FAF2EAF69976D964EAD38
:105890005FAD6D974115510579F1FA01808586302C
:1058A000F9F463965FAF4EAF6397CE018F5A9F4F67
:1058B0000E9417256596EFAC6597EE2089F06796F4
:1058C0008EAD9FAD6797892B09F05DC009C06496C6
:1058D0002FAD649720FFDAC14817590709F4CCC1EE
:1058E0006D96EEADFFAD6D970280F381E02D6D9664
:1058F000FFAFEEAF6D97CACF0E941265DC01CB01FE
:10590000C296A11DB11D8093EC069093ED06A09365
:10591000EE06B093EF060E9412650091E806109122
:10592000E9062091EA063091EB06061717072807CB
:10593000390708F032C3E091E606F091E7060681E8
:1059400017810115110571F0F8018085863031F459
:105950001A830983CE0101960E941725F80102815E
:105960001381EFCF0E941265DC01CB0188579C4E5A
:10597000AF4FBF4F8093E8069093E906A093EA06E5
:10598000B093EB060AC36496FFAC6497F0E4FF1291
:1059900022C165E974E063968EAD9FAD63970E9466
:1059A000BD508C01F1FC02C062E001C060E08E2DB0
:1059B0000E949C6465968FAD6597863308F0865388
:1059C00090917B00282F2870977F922B90937B00DB
:1059D0008770806480937C0080917A0080648093DB
:1059E0007A0080917A0086FDFCCF8091780020912A
:1059F000790090E0AC01522B6B965FAF4EAF6B9786
:105A00000115110509F4D1C0F8018085853009F030
:105A1000CCC0C8010E945F546E968FAF6E978430E1
:105A200008F45DC063E0C8010E948C67FC018185B9
:105A300092854AE0C42EC89E7001C99EF00C1124C4
:105A400062E0C8010E948C67FC0181859285C89E36
:105A50001001C99E300C11244101032C000CAA082E
:105A6000BB0861E0C8010E948C676C0160E0C8015E
:105A70000E948C67FC0141845284638474846B9619
:105A80002EAD3FAD6B97C901330FAA0BBB0B9C0129
:105A9000AD012419350946095709C7010F2C000C1F
:105AA000AA0BBB0BBC01CD01681979098A099B09B6
:105AB0000E94147CF6012185328543855485241982
:105AC0003509460957090E94467C820E931EA41E82
:105AD000B51E6E96FFAD6E97F530A1F416C08AE044
:105AE0006B962EAD3FAD6B97829F4001839F900CCC
:105AF0001124092C000CAA08BB08212C312CE12C04
:105B000038E2F32E81E090E007C064E0C8010E9413
:105B10008C67FC0181859285A7010F2C000C660B18
:105B2000770B84169506A606B70614F4B501A401F2
:105B30004101032C000CAA08BB0884169506A60692
:105B4000B70614F44A015B016E96FFAD6E97F23012
:105B500009F0CDC06B962EAD3FAD6B976901330F49
:105B6000EE08FF0860E0C8010E948C67FC01818597
:105B70009285A385B485C816D906EA06FB060CF4FF
:105B800096C061E0C8010E948C67FC018185928506
:105B9000A385B4858C159D05AE05BF050CF0A0CE80
:105BA000C12CD12C7601C39485C08AE06B962EADB2
:105BB0003FAD6B97829F4001839F900C1124092C6D
:105BC000000CAA08BB08212C312CE12C28E2F22E73
:105BD00081E090E08CC0FF1508F464C023E02F152D
:105BE00008F47ECEF1FC03C010E062E002C011E0D8
:105BF00060E08E2D0E949C6465962FAD659730E025
:105C0000F901ED5AFD4E8491F901E35FFD4E0491D7
:105C1000F901E953FE4EF490FF20A1F081110E949A
:105C20001764EF2DF0E0EE0FFF1FEE50F34FA5913C
:105C3000B491EC910E2331E020E009F430E0832FA1
:105C4000922F02C080E090E0412F50E031E04817F1
:105C5000590709F030E0632F70E06796EEADFFADB5
:105C60006797A281B3816A177B07C9F0218122233C
:105C700009F42DCE215014C081E09081911180E073
:105C8000808373836283682F70E003C030837383E3
:105C90006283CE018F5A9F4F0E94222421CE23E09F
:105CA00021831ECE32E4F31609F473CE19CEC12C33
:105CB000D12C76016796EEADFFAD67978281938117
:105CC000092E000CAA0BBB0B8C159D05AE05BF055C
:105CD00009F406CEB601CE018F5A9F4F0E942224AE
:105CE0006796EEADFFAD6797D382C282F9CD679616
:105CF000EEADFFAD6797428153816B962EAD3FAD00
:105D00006B97241B350B37FF03C031952195310963
:105D10008217930714F4118205C08181863014F430
:105D20008F5F8183818185309CF0C101330CAA0B88
:105D3000BB0B88159905AA05BB0551F0C701FF0CDF
:105D4000AA0BBB0B88159905AA05BB0509F0C8CDA0
:105D50006B968EAD9FAD6B974817590709F4C0CD70
:105D6000C501B4010E94C17D20E030E040E251E471
:105D70000E94177D6B017C0165961FAD65976EE0F3
:105D80007DE086E398E00E94A35E4AE050E0612F48
:105D900086E398E00E94745F6CE07DE086E398E023
:105DA0000E94A35E22E0B701A60186E398E00E946C
:105DB000A85586E398E00E94C65F63960EAD1FADBE
:105DC000639768E574E0C8010E94BD505C0167E616
:105DD00074E0C8010E94BD508C01009709F48AC08C
:105DE000FC016185728540E450E0CE0101960E947D
:105DF0000A816FE270E0CE0101960E94D180892B6A
:105E000051F4F8012185328543E050E060E4CE0191
:105E100001960E947F49C701B6010E94897D1B013E
:105E20003F926F932EE635E03F932F9369965FADD7
:105E300069975F9368968FAD68978F930E94618191
:105E40000F900F900F900F900F900F9020E030E088
:105E5000A901C701B6010E94717E260137011816FB
:105E600024F077FA709477F870946996EEADFFADF0
:105E7000699701900020E9F731978F0169962EAD5F
:105E80003FAD6997021B130B8EE2808392E4892E4B
:105E9000912C8C0E9D1E800E911EB10137FE03C009
:105EA000719561957109072E000C880B990B0E9462
:105EB000C17D9B01AC01C301B2010E94A57C20E021
:105EC00030E040E251E40E94767E0E94897D605D70
:105ED000F4016083E3E4F0E0EC0FFD1FE00FF11F3D
:105EE00010820E941455882329F080918D05882303
:105EF00009F44BC0A114B104E9F120E030E0A9019C
:105F0000C701B6010E94717E20E030E040E05FE30F
:105F100087FD05C0C701B6010E94A67C04C0C70169
:105F2000B6010E94A57C0E94897D23967FAF6EAF4B
:105F30002397F50161857285CE0101960E946D540B
:105F4000CE0101960E946822882381F0C12CD12CB9
:105F5000E12CF12C01E09E012F5B3F4F41E050E02E
:105F600060E070E0CE0101960E948109CE010196A9
:105F70000E942F516796EEADFFAD67976B962EADE1
:105F80003FAD6B9733832283ABCCBE016F5B7F4FFA
:105F9000CE0101960E949D55ADCFC35ADF4F0FB67B
:105FA000F894DEBF0FBECDBFDF91CF911F910F914F
:105FB000FF90EF90DF90CF90BF90AF909F908F9029
:105FC0007F906F905F904F903F902F900895A8958D
:105FD0000E94BA12029724F00E94DF3D0E94042C16
:105FE0000C94832580918D058F5F80938D05A895F6
:105FF0000E94042C80918D05815080938D05089519
:1060000060ED7CE086E398E00E94A35E6DEB7CE0AF
:1060100086E398E00E94A35E6FEA7CE086E398E066
:106020000E94A35E67EA7CE086E398E00E94A35E9C
:1060300086E398E00E94C65F6AE97CE086E398E028
:106040000E94A35E6AE87CE086E398E00E94A35E7B
:106050006EE77CE086E398E00E94A35E67E67CE062
:1060600086E398E00E94A35E65E57CE086E398E025
:106070000E94A35E60E47CE086E398E00E94A35E59
:1060800061E37CE086E398E00E94A35E62E27CE04C
:1060900086E398E00E94A35E6AE17CE086E398E0F4
:1060A0000E94A35E6FE07CE086E398E00E94A35E1E
:1060B00065E07CE086E398E00E94A35E6DEF7BE004
:1060C00086E398E00E94A35E61EF7BE086E398E0C0
:1060D0000E94A35E67ED7BE086E398E00E94A35EEA
:1060E00068EB7BE086E398E00E94A35E86E398E09D
:1060F0000C94C65FAF92BF92CF92DF92EF92FF9265
:106100000F931F93CF93DF936C017B018A010E9451
:10611000FE7B81508E3FA0F45701C0E0D0E00150DB
:106120001109C017D1077CF4C6018C0F9D1F0E9476
:10613000FE7BF50181935F01882329F02196F1CF41
:1061400080E090E005C0CE0DDF1D188281E090E078
:10615000DF91CF911F910F91FF90EF90DF90CF9043
:10616000BF90AF900895CF92DF92EF92FF920F937E
:106170001F93CF93DF936C01EB0109900020E9F7A7
:106180002197C61BD70BC032D10514F0CFE1D0E068
:106190008B01E12CF12CEC16FD0664F4F801619101
:1061A0008F01C7018C0D9D1D0E94067CFFEFEF1A29
:1061B000FF0AF1CF60E0C6018C0F9D1FDF91CF91E8
:1061C0001F910F91FF90EF90DF90CF900C94067C81
:1061D000882319F061EC7AE002C063EC7AE086E390
:1061E00098E00C94A35EAF92BF92CF92DF92EF92B1
:1061F000FF920F931F93CF93DF93CDB7DEB7C058B5
:10620000D1090FB6F894DEBF0FBECDBF8E010F5B74
:106210001F4FD8011D921C92FE01ED5BFF4F2EE136
:10622000DF011D922A95E9F70297CCF0FB0162810C
:1062300073814FE150E0C8010E940A81B80186E1F4
:1062400090E00E94B330B80186E398E00E94CA5FF4
:1062500061EB7BE086E398E00E94A35E1BC040E216
:1062600050E0B80186E190E00E947A30892BB1F4C9
:1062700040E250E065EA7BE0C8010E94FA7467E8FA
:106280007BE086E398E00E94A35EB80186E398E095
:106290000E94CA5F86E398E00E94C65F80917A07F9
:1062A0001F928F93809179071F928F938091780727
:1062B0001F928F93809177071F928F93809176071B
:1062C0001F928F93809175071F928F9389E994E0B5
:1062D0009F938F931F9280E48F93CE0101966C0160
:1062E0009F938F930E94248163E77BE086E398E08D
:1062F0000E94A35EB80186E398E00E94CA5FB601DF
:1063000086E398E00E94CA5F86E398E00E94C65F39
:106310000FB6F894A8958091600088618093600022
:10632000109260000FBE7E0191E6E90EF11CD701CC
:1063300013961C921E92129788EE93E0A0E0B0E0B4
:10634000F70184839583A683B78388E084878BE4F1
:1063500093E09183808316870587108A178680E5EE
:1063600090E0928B818B158A64EE77E282EA9AE262
:106370000E9453758C010FB6F894DEBF0FBECDBFDF
:10638000892BE1F183E090E00E94D571D8011D9640
:106390009C938E931C97FC01F182E0821282C701CC
:1063A0000E943D42882319F0C7010E944443D7014F
:1063B0001F966D917C9150975196AD90BC905297DD
:1063C0006115710569F0CE0189589F4F0E94CC5F1D
:1063D000A501BE0169587F4FC7010E94774507C0DC
:1063E000F70165857685A501C7010E942C4A18161C
:1063F00019060CF498C0C8010E947B2A00E010E046
:10640000F701E388F48899E288E10FB6F894A8953B
:10641000809360000FBE909360000115110509F490
:1064200069C0F8ECEF16F10409F056C067E67BE0AE
:1064300086E398E00E94A35EEB961FAE1EAEEB973C
:10644000ED961FAE1EAEED978FEF9FEFEF969FAFCD
:106450008EAFEF9782E792E0E9969FAF8EAFE99714
:10646000C158DF4F19830883CF57D040F8940E945A
:10647000944CCE0189589F4F0E949C3C9093E50616
:106480008093E4067894C8010E947B2A8091E406F8
:106490009091E506892B79F460E57BE086E398E04E
:1064A0000E94A35E0E941265DC01CB018856954CC8
:1064B000AF4FBF4F2DC065E47BE086E398E00E94BC
:1064C000A35E0E94B3356EE37BE086E398E00E9412
:1064D000A35E82E090E0C7C066E27BE086E398E0DE
:1064E0000E94A35E4AE050E0B70186E398E00E9474
:1064F0006D5F06C063E17BE086E398E00E94A35EE7
:106500000E941265DC01CB0188579C4EAF4FBF4FF4
:106510008093E0069093E106A093E206B093E30631
:1065200085EF9FEFA0C0D7011D96BC901D971E96CA
:10653000AC90DF92CF928FE09BE09F938F931F935D
:106540000F930E94DC75DF92CF928AE09BE09F93CD
:106550008F931F930F930E94DC75D8011C96ED91C9
:10656000FC911D9781E08283DF92CF9287E09BE0D0
:106570009F938F931F930F930E94DC75D8011C96F5
:10658000ED91FC911D971282AF92BF9281ED9AE03E
:106590009F938F931F930F930E94DC758CE09BE079
:1065A0009F938F931F930F930E94DC75F701148ABA
:1065B000138AD8011C96ED91FC911D97A080B180A3
:1065C0000FB6F894DEBF0FBECDBF83E3C82ED12C2B
:1065D000D501ED91FC910084F185E02DC50119955F
:1065E00041975CF4B1E0CB1AD10839F064E170E076
:1065F00080E090E00E94D864EBCF6E01F7E7CF0E09
:10660000D11CDF92CF9285EC9AE09F938F931F93DA
:106610000F930E94F9750F900F900F900F900F90AD
:106620000F90019709F0ECCEF60180819181D7019E
:1066300054969C938E935397D12C80E08A3039F4F2
:10664000BAE0DB1609F4DCCE9AE0D92E03C08D3017
:1066500009F0D82EC8010E949E758F3F79F7C801B6
:106660000E947B2ACDCEC058DF4F0FB6F894DEBF14
:106670000FBECDBFDF91CF911F910F91FF90EF9093
:10668000DF90CF90BF90AF9008950E94F330909329
:1066900093058093920584EA9AE00C94444369EB55
:1066A0007EE086E398E00E94A35EE0E0F0E01994CB
:1066B000CF93DF93C0E0D0E060E0CE010E94067C83
:1066C0002196C11582E0D807B9F764E070E186E34E
:1066D00098E0DF91CF910C94A35E0F931F93CF931B
:1066E000DF93EB018AE797E09F938F9389E797E029
:1066F0009F938F9388E797E09F938F9387E797E027
:106700009F938F9386E797E09F938F9385E797E01A
:106710009F938F9388EC94E09F938F938B818F93BB
:106720008A818F930E9490812DB73EB7205F3F4FA3
:106730000FB6F8943EBF0FBE2DBF069794F40A80A3
:10674000DB81C02D66E270E186E398E00E94A35EE3
:10675000BE0186E398E0DF91CF911F910F910C94D9
:10676000CA5F0E94414C05E717E0C0E0D0E0F801A5
:1067700061918F01CE010E94067C2196C630D10521
:10678000B1F768E370E186E398E0DF91CF911F9164
:106790000F910C94A35ECF93DF931F92CDB7DEB71A
:1067A0001982892B21F0FB016281738103C0BE0134
:1067B0006F5F7F4F86E390E00E94B33064E170E149
:1067C00086E398E00E94A35E0F90DF91CF91089539
:1067D000EF92FF920F931F93CF93DF93CDB7DEB766
:1067E0002C970FB6F894DEBF0FBECDBF8C017B0196
:1067F0008DE693E09A8389831B821C821D821E8210
:1068000098878F8319861A861B861C86053011058A
:106810005CF0BE01695F7F4FF701808591850E9422
:106820001164892B09F052C0BE016F5F7F4F82E176
:1068300090E00E94F263043011050CF44FC0BE01D9
:10684000695F7F4FF701868197810E941164892BD0
:1068500009F444C0BE01695F7F4F8EE090E00E9462
:10686000F263BE01695F7F4FF701848195810E94C9
:106870001164892BF1F1BE01695F7F4F8AE090E0DE
:106880000E94F263BE01695F7F4FF70182819381AD
:106890000E941164892BC1F1BE01695F7F4F86E0C0
:1068A00090E00E94F2636DEE7FE086E398E00E9444
:1068B000A35E2C960FB6F894DEBF0FBECDBFDF915E
:1068C000CF911F910F91FF90EF900895BE01695FE6
:1068D0007F4F82E190E00E94F263B1CFBE016F5F13
:1068E0007F4F8EE090E00E94F263033011050CF0C0
:1068F000B8CFBE016F5F7F4F8AE090E00E94F263E5
:10690000023011050CF0BECFBE016F5F7F4F86E0F5
:1069100090E00E94F2630130110529F6BE016F5F1D
:106920007F4F86E090E00E94F26364EF7FE086E3B1
:1069300098E00E94A35EB7CFCF93DF93CDB7DEB7C9
:106940002C970FB6F894DEBF0FBECDBF1C821B8202
:106950001E821D828FEF9FEF98878F8389E992E0D7
:106960009A83898388E490E09A8789871C861B86AE
:1069700063ED7FE086E398E00E94A35E6091E40609
:106980007091E506CE0101960E9478286FEFCE0146
:1069900001960E94592763EC7FE086E398E00E940D
:1069A000A35E2C960FB6F894DEBF0FBECDBFDF916D
:1069B000CF9108950F931F93CF93DF93CDB7DEB799
:1069C00069970FB6F894DEBF0FBECDBF8FE290E09F
:1069D0009A838983FE01339687E1DF011D928A95B0
:1069E000E9F76EEA7FE086E398E00E94A35E25E780
:1069F00037E0DE011196AE01435F5F4F8D01F90173
:106A000061919F01862F90E074E0959587957A9526
:106A1000E1F78C579D4FFC01808111968C93119763
:106A2000E62FEF70F0E0EC57FD4F808112968C93CB
:106A300012971296A417B50711F71E866CED74E035
:106A4000C8010E94C680B80186E398E00E94CA5F30
:106A5000C8010E9409591E8664EE74E0C8010E94B4
:106A6000C680B80186E398E00E94CA5F6EEE74E0CB
:106A7000C8010E94663C69960FB6F894DEBF0FBE4F
:106A8000CDBFDF91CF911F910F910895CF93C1E0BA
:106A900068EE73E080E090E00E94D8644AE050E045
:106AA0006C2F86E398E00E94745FCF5FC43181F75A
:106AB000CF9108950F931F93CF93DF9300D000D011
:106AC000CDB7DEB70E94003062E17DE086E398E05A
:106AD0000E94A35E0DE613E01A8309831B821C82C9
:106AE0001D821E82CE0103960E94873FCE01019631
:106AF0000E94313F1A8309831B821C821D821E82E1
:106B000024E030E0AE014D5F5F4F60E081E090E057
:106B10000E94C12BCE0101960E94313F1A83098346
:106B20001B821C821D821E8224E030E0AE014D5F7C
:106B30005F4F60E085E090E00E94C12BCE0101969E
:106B40000E94313F68E37DE086E398E00E94A35E07
:106B500026960FB6F894DEBF0FBECDBFDF91CF9162
:106B60001F910F9108957F928F929F92AF92BF9243
:106B7000CF92DF92EF92FF920F931F93CF93DF9309
:106B8000CDB7DEB72B970FB6F894DEBF0FBECDBFE3
:106B90008091E4069091E506009709F497C260EFB2
:106BA00074E00E94BD509093F9068093F806009718
:106BB00009F4A9C00E945F54082F10E001151105C7
:106BC00009F4A1C0000F111F000F111F8091F106E1
:106BD0009091F206892B09F085C0C8010E94D571F9
:106BE0009093F2068093F10610928907109288071D
:106BF0001092FB061092FA061092870710928B07EC
:106C000010928A077801013082E018071CF0E12C0D
:106C100032E0F32EC70101960E94D57190938D0743
:106C200080938C0790938607809385078E0D9F1D18
:106C30009093800780937F070E941265609381077D
:106C400070938207809383079093840780E090E09D
:106C5000E0918C07F0918D07E80FF91F10820196E3
:106C6000E816F906ACF782E090E0909389078093EC
:106C7000880780E98093C9001092C8001092CD0067
:106C800083E08093CC008EE08093CA00F0920802EB
:106C9000E092070220918C0730918D0780910702C6
:106CA00090910802820F931F9093800780937F0733
:106CB000232B09F426C162EE7EE086E398E00E9471
:106CC000A35E4AE050E0B80186E398E00E946D5F61
:106CD00086E398E00E94C65F8AED91E290937E077A
:106CE00080937D0765E57FE086E398E00E94A35EE0
:106CF0004AE050E0B80186E398E00E946D5F86E3C9
:106D000098E00E94C65F66EF74E08091E40690917F
:106D1000E5060E94BD508C010097B1F00E945F54BF
:106D20008111F6C011C069E37FE086E398E00E941C
:106D3000A35E4AE050E0B70186E398E00E946D5FF1
:106D400086E398E00E94C65FE090E406F090E506D6
:106D50006AEF74E0C7010E94BD509093F7068093DC
:106D6000F60661E075E0C7010E94BD508C0190936A
:106D700074078093730767E075E0C7010E94BD50F8
:106D80009093FF068093FE06109291051092900555
:106D90000115110521F1D8011696CD90DC901797B9
:106DA00027EDA22E22E0B22E0091730710917407F6
:106DB0000115110569F0C114D10451F0F601808567
:106DC0008530B1F7C6010E945F54823088F3CCC091
:106DD000F801868197819093910580939005E090CA
:106DE000E406F090E50663EF74E0C7010E94BD5031
:106DF0008C019093E7068093E6066EE075E0C7018C
:106E00000E94BD509093F5068093F406011511057C
:106E1000C1F0D80116960D911C9117970115110517
:106E200081F0F8018085863031F41A830983CE0120
:106E300001960E941725D80112960D911C91139767
:106E4000EDCF64E17FE086E398E00E94A35E6CE012
:106E50007FE086E398E00E94A35E81E020917307C3
:106E600030917407232B09F480E00E94E83063E03E
:106E70007FE086E398E00E94A35E81E02091E60631
:106E80003091E706232B09F480E00E94E8306AEF96
:106E90007EE086E398E00E94A35E81E02091F60602
:106EA0003091F706232B09F480E00E94E83063EF6D
:106EB0007EE086E398E00E94A35E81E02091F406E4
:106EC0003091F506232B09F480E00E94E83086E338
:106ED00098E00E94C65F0E94104A6B017C016EEE32
:106EE0007EE086E398E00E94A35E2AE0B701A60157
:106EF00086E398E00E94DC5E86E398E00E94C65F2D
:106F0000E5C06BEC7EE086E398E00E94A35EE0CEF5
:106F100061E0C8010E948C67FC01E184F2849091D9
:106F20000007992359F0809170008E7F8093700044
:106F300010920007109202021092010282E18093E7
:106F4000000291110E946B47C7010E94934701E024
:106F500010E0E016F1060CF4E6CE60E0C8010E94F5
:106F6000C9470F5F1F4FF5CFBA82A982DC82CB825F
:106F70001B861A86CE0101960E94B823CE01019687
:106F80000E9468228823D1F18A859B850097E1F0D1
:106F9000DC01ED91FC910484F585E02D1995892B98
:106FA00049F08A859B85DC01ED91FC910284F38593
:106FB000E02D19958A859B85DC01ED91FC91068079
:106FC000F781E02D19951AC060E070E0CE010196BE
:106FD0000E94C7228C0197FF76C011950195110977
:106FE00088248394912CCE0101960E94AB23E82E35
:106FF000F12C8985853061F0863079F1D6011296C1
:10700000CD90DC901397CE0101960E942F51CCCEEB
:10701000EF2829F462E0CE0101960E947F2361E00F
:10702000802F0E949C6460E0802F0E946D6461E369
:107030007FE086E398E00E94A35E4AE050E0B8015A
:1070400086E398E00E946D5F6CE27FE086E398E063
:107050000E94A35E6AE27FE031C0702E61E0802F63
:107060000E949C6461E0892821F0EA94EF2829F4C9
:1070700003C0EA94EF2809F060E0E62EF12C872D9A
:107080000E946D6465E27FE086E398E00E94A35E63
:107090004AE050E0B80186E398E00E946D5F63E249
:1070A0007FE086E398E00E94A35E4AE050E0B701EB
:1070B00086E398E00E946D5F61E27FE086E398E0FE
:1070C0000E94A35E9BCF812C912C8DCF2B960FB667
:1070D000F894DEBF0FBECDBFDF91CF911F910F910E
:1070E000FF90EF90DF90CF90BF90AF909F908F90E8
:1070F0007F900895CF93DF93CDB7DEB72C970FB66F
:10710000F894DEBF0FBECDBF63E97FE086E398E071
:107110000E94A35E86E398E00E94C65F88E490E048
:107120000E94FE7B8B37A1F51C821B821E821D8272
:107130008FEF9FEF98878F8389E992E09A83898305
:1071400088E490E09A8789871C861B860E94944C6D
:10715000CE0101960E949C3C9093E5068093E40644
:10716000892B19F466E77FE015C06FE67FE086E3C0
:1071700098E00E94A35E86E398E00E94C65F0E94AA
:10718000B33584EA9AE00E94444381E090E00CC069
:1071900062E87FE086E398E00E94A35E86E398E0E1
:1071A0000E94C65F80E090E02C960FB6F894DEBF98
:1071B0000FBECDBFDF91CF9108950C947A382F92F6
:1071C0003F924F925F926F927F928F929F92AF9277
:1071D000BF92CF92DF92EF92FF920F931F93CF93C4
:1071E000DF93CDB7DEB728970FB6F894DEBF0FBE9A
:1071F000CDBF8C016B010E949629019609F4D3C280
:10720000D801ED91FC910284F385E02DC801199518
:107210007C018F3FBFEF9B0709F4C5C2D801ED91F8
:10722000FC910684F785E02D682FC8011995B2E21C
:10723000EB16F10429F4B601C8010E94B729B5C2C2
:10724000EDE2EE16F10429F0C701C0970A9708F0A5
:1072500044C1D801ED91FC910284F385E02DC80171
:1072600019957C018F3FBFEF9B0709F49CC28D9756
:1072700089F4D801ED91FC910284F385E02DC801D9
:1072800019957C01019609F48EC2EFEFFFEFF887A4
:10729000EF8304C021E030E038872F83C701C09717
:1072A000A12CB12C0A97C8F49AE0992E9A9CC0019F
:1072B0009B9C900D1124B701605371095B01A80ECE
:1072C000B91ED801ED91FC910284F385E02DC8012F
:1072D00019957C01C0970A9748F3BEE2EB16F104BA
:1072E000D1F0C7018F7D85349105A9F0EF81F88534
:1072F000AE9EC001AF9E900DBE9E900D1124092E32
:10730000000CAA0BBB0BF60181879287A387B48779
:1073100082E08087D8C0B501BB0C880B990B0E9416
:10732000C17D2B013C01FEE2EF16F104A1F5D8016D
:10733000ED91FC910284F385E02DC80119957C0143
:10734000212C312C20E030E040E251E4C301B201B5
:107350000E94767E4B015C01B70160537109072ED4
:10736000000C880B990B0E94C17DA50194010E941D
:10737000A67C2B013C01B1E02B1A3108D801ED911C
:10738000FC910284F385E02DC80119957C01C0971A
:107390000A97C0F202C0212C312CC7018F7D8534A1
:1073A000910509F042C0D801ED91FC910284F3856A
:1073B000E02DC80119957C018B32910559F4D80153
:1073C000ED91FC910284F385E02DC80119957C01B3
:1073D000B1E00CC08D9761F4D801ED91FC9102846D
:1073E000F385E02DC80119957C01BFEFBE8302C073
:1073F000E1E0EE83A12CB12C8AE0982EC701C09762
:107400008A309105B0F49A9C90019B9C300D112418
:107410005C01A20EB31ED801ED91FC910284F385AC
:10742000E02DC80119957C01E9CFB1E0BE83A12C04
:10743000B12CEF81F885BF01FF0F880B990B0E94DB
:10744000C17DA30192010E94767E2B013C01B50112
:10745000BB0C880B990B0E94C17D4B015C01FE8126
:107460006F2FFF0F770B880B990B0E94C17D9B013B
:10747000AC01C501B4010E94767E4B015C01B101F3
:10748000330C880B990B0E94C17D9B01AC01C50197
:10749000B4010E94A67C9B01AC0160E070E080E238
:1074A00091E40E94E37E9B01AC01C301B2010E9402
:1074B000767ED60119966D937D938D939C931C9740
:1074C00083E018968C93D801ED91FC910684F785A2
:1074D000E02D6E2DC801199522C0BBE5EB16F10415
:1074E00009F060C0D801ED91FC910284F385E02D94
:1074F000C80119958B35910509F055C185E0F60154
:107500008087C8010E949629D801ED91FC910284E0
:10751000F385E02DC80119958D35910519F480E0AA
:1075200090E043C1D801ED91FC910684F785E02DF0
:10753000682FC8011995BB24BA940E946F2A7C0158
:10754000009709F430C1BB2021F0F60197838683B0
:1075500008C0D40113969C938E931297FC019582D8
:107560008482C8010E949629B701C8010E94DF38B1
:10757000892B09F018C1C8010E949629D801ED9104
:10758000FC910284F385E02DC8011995B12C4701C7
:107590008C32910591F221E030E08D35910509F0B2
:1075A00089C086C0BBE7EB16F10409F088C0D8019A
:1075B000ED91FC910284F385E02DC80119958B377C
:1075C000910509F0F0C086E0F6018087C8010E94AD
:1075D0009629D801ED91FC910284F385E02DC80134
:1075E00019958D37910509F49ACFD801ED91FC9149
:1075F0000684F785E02D682FC801199599249A947F
:107600000E946F2A7C01009709F4CDC0992021F0D7
:10761000F6019783868308C0D50113969C938E93B9
:107620001297FC01B582A482C8010E949629B70175
:10763000C8010E94B729019609F4B5C0C8010E948B
:107640009629D70119968D919C911A9711969C9322
:107650008E931A961C921E921997D801ED91FC9167
:107660000284F385E02DC8011995CA9709F09BC0E3
:10767000C8010E949629B701C8010E94DF3801960F
:1076800009F491C0C8010E949629D801ED91FC919E
:107690000284F385E02DC8011995912C57018C3295
:1076A000910509F4ADCF21E030E08D37910511F45B
:1076B00020E030E088279927821B930B76C0BEE636
:1076C000EB16F10411F519821A821B821C82D80173
:1076D000ED91FC910484F585E02D44E050E0BE017D
:1076E0006F5F7F4FC8011995049709F05CC044E0B3
:1076F00050E06BE774E0CE0101960E94FC80009799
:1077000009F051C0F601108650C0F6E6EF16F104FC
:1077100021F59E012F5F3F4F790185E0D9011D9230
:107720008A95E9F7D801ED91FC910484F585E02D67
:1077300045E050E0B901C80119950597A1F545E06C
:1077400050E065E874E0C7010E94FC80009759F59D
:1077500021E0F6012087118628C0F4E7EF16F10436
:1077600011F519821A821B821C82D801ED91FC91BD
:107770000484F585E02D44E050E0BE016F5F7F4F4B
:10778000C8011995049779F444E050E060E874E08A
:10779000CE0101960E94FC80009729F421E0F601B9
:1077A0002087218702C08FEF9FEF28960FB6F894AD
:1077B000DEBF0FBECDBFDF91CF911F910F91FF9024
:1077C000EF90DF90CF90BF90AF909F908F907F9081
:1077D0006F905F904F903F902F900895CF92DF92DF
:1077E000EF92FF92CF93DF93EC010E9412656B0141
:1077F0007C018091ED089091EE08DC01ED91FC9107
:107800000084F185E02D1995892B79F40E94126589
:10781000DC01CB018C199D09AE09BF0988399A4357
:10782000A105B10530F380E00DC08091ED08909185
:10783000EE08DC01ED91FC910284F385E02D1995B1
:10784000888381E0DF91CF91FF90EF90DF90CF9020
:1078500008958F929F92AF92BF92EF92FF920F93F3
:107860001F93CF93DF938C017B0149015A010E9442
:107870006F2AEC01892BF9F083E0888789869A8644
:10788000AB86BC8688819981009711F00E946D7249
:10789000C7010E947A8099838883BE01C801DF9165
:1078A000CF911F910F91FF90EF90BF90AF909F905D
:1078B0008F900C94D850DF91CF911F910F91FF9032
:1078C000EF90BF90AF909F908F900895FB01019033
:1078D0000020E9F73197AF01461B570B20E00C94CD
:1078E0004D550F931F93CF93DF93EC012097F9F041
:1078F0000A811B81888587FD06C08E819F81009744
:1079000011F00E94713C8885843031F489859A8514
:10791000009711F00E946D7288819981009711F093
:107920000E946D72CE010E946D72E801DFCFDF917F
:10793000CF911F910F9108950F931F93CF93DF93D2
:10794000009791F08C010E946F2AEC01892B61F065
:10795000C8010E949629BE01C8010E94DF38019625
:1079600031F4CE010E94713C80E090E001C0CE0174
:10797000DF91CF911F910F910895FC01848588308C
:1079800021F063E070E00C946E4580E00895CF93A1
:10799000C82F462F61E070E00E94204361E070E054
:1079A0008C2F0E946E458111F9CFCF9108950F93CE
:1079B0001F93CF93DF93EC010E94C75E8C01CE0131
:1079C0000E94C65F800F911FDF91CF911F910F9191
:1079D00008954F925F926F927F928F929F92AF9293
:1079E000BF92CF92DF92EF92FF920F931F93CF93AC
:1079F000DF931F921F92CDB7DEB75C018FEE98E048
:107A00000E94EE3B81113AC036C08C01CE01019636
:107A10000E94EE3B882379F1C80101962981F70184
:107A200021937F01422F4F7750E0449DB001459D47
:107A3000700D549D700D1124C60ED71E47E0440CE6
:107A4000551C661C771C4A95D1F727FF27C0853047
:107A50009105D9F68FEF9FEF90938909809388095C
:107A60008091ED089091EE08DC01ED91FC91048885
:107A7000F589E02D199580E090E08EC09090EF0898
:107A8000198280EFE82E88E0F82E01E010E0C12C8A
:107A9000D12C412C512C32014394B8CFF92DF07FD9
:107AA000FA832FEF280FD5012C93F03319F581516C
:107AB000974F0E94EE3B8823F1F2C8018F50974FF9
:107AC0000E94EE3B8823B9F2C8010396D501EC91E0
:107AD000F0E0E751F74FE780F12CFE2CEE242085F3
:107AE000E20EF11C2091EF0821FF08C0B2E0EB0E7E
:107AF000F11C04C020E0E12CF12C01C022E0422E58
:107B0000512CFC01E751F74F4F018C01481A590ADB
:107B10002EEF622E77247A94C801840D951D8C1562
:107B20009D0578F5CE0101960E94EE3B882309F46D
:107B3000A2CF80918609909187090097B1F0FA81D0
:107B4000F03399F4D5012C91F301E21BF1099F0167
:107B5000200F311FE216F30640F4DC01ED91FC9199
:107B60000190F081E02D698119950038110518F414
:107B70008981F40186830F5F1F4FFFEF8F1A9F0AE1
:107B8000CBCF8091860990918709892B21F4013808
:107B9000110508F070CFC8010F900F90DF91CF91C1
:107BA0001F910F91FF90EF90DF90CF90BF90AF901B
:107BB0009F908F907F906F905F904F9008952F923D
:107BC0003F924F925F926F927F928F929F92AF926D
:107BD000BF92CF92DF92EF92FF920F931F93CF93BA
:107BE000DF931F92CDB7DEB70E941455382E88233D
:107BF00009F422C10E9412652B013C018091750994
:107C000090917609A0917709B0917809A30192012A
:107C1000281B390B4A0B5B0BDA01C90189399A43DE
:107C2000A105B105A8F48091710990917209A09104
:107C30007309B0917409A3019201281B390B4A0BF7
:107C40005B0BDA01C90189399A43A105B105C8F175
:107C5000209179098091ED089091EE08222371F02E
:107C60002CEF3FEF3093890920938809DC01ED91D7
:107C7000FC910488F589E02D1995DDC020EC209356
:107C8000EF081092F008DC01ED91FC910280F38185
:107C9000E02D42E050E06FEE78E0199540927109D6
:107CA000509272096092730970927409409275093A
:107CB00050927609609277097092780981E08093FA
:107CC00079098091ED089091EE08DC01ED91FC912D
:107CD0000084F185E02D1995892B09F4ADC0CE0102
:107CE00001960E94E93C5C01892B09F4A0C04092F6
:107CF000750950927609609277097092780980919F
:107D0000EF08807F803309F076C080917A099091E6
:107D10007B09892B09F490C0E980F12CF701E75128
:107D2000F74F078110E0102F00278085080F111DE5
:107D300097012F50374F4901B7016E50774FA80177
:107D4000C9010E94A180B8016E0D7F1DDB01A75102
:107D5000B74F18961C9218978091EF088670282EBE
:107D6000E0917A09F0917B0932E0831337C01996CC
:107D7000CC901997D12CDC2CCC241A968C91C80E5F
:107D8000D11C4BEF5FEF4E195F09401B510B4A0DA1
:107D90005B1D6C50774FC401199580E48093EF0808
:107DA0002092F008D092F108C092F2088091ED087C
:107DB0009091EE08DC01ED91FC910280F381E02DC1
:107DC00044E050E06FEE78E01995409271095092CE
:107DD000720960927309709274092EC04DEF5FEFC3
:107DE0004E195F09401B510B4A0D5B1D6E50774FBA
:107DF000C401199521C0803CA9F480ED8093EF085F
:107E00001092F0088091ED089091EE08DC01ED9160
:107E1000FC910280F381E02D42E050E06FEE78E0CB
:107E200019950AC0803D41F41092790905C00E945D
:107E30001455811101C0312C832D0F90DF91CF910A
:107E40001F910F91FF90EF90DF90CF90BF90AF9078
:107E50009F908F907F906F905F904F903F902F906A
:107E60000895AF92BF92CF92DF92EF92FF921F934D
:107E7000CF93DF9300D000D0CDB7DEB76C017C018B
:107E800010E08AE0A82EB12C1330A9F0F70182810E
:107E900090E0A0E0B0E089839A83AB83BC83BE828C
:107EA000AD82BE016F5F7F4F86E398E00E9412248F
:107EB00064E470E114C0F601858190E0A0E0B0E0D8
:107EC00089839A83AB83BC83BE82AD82BE016F5F20
:107ED0007F4F86E398E00E94122461E470E10E94E3
:107EE000A35E1F5FFFEFEF1AFF0A143069F62696B4
:107EF0000FB6F894DEBF0FBECDBFDF91CF911F91BB
:107F0000FF90EF90DF90CF90BF90AF90089524E066
:107F100030E0AC0160E08FE090E00C94C12BCF9397
:107F2000DF93C9EED8E080EE8E831F828C819D8125
:107F3000DC01ED91FC910280F381E02D42E050E004
:107F40006FEE78E019958FEF9FEF909389098093FA
:107F500088098C819D81DC01ED91FC910680F7817F
:107F6000E02D19958C819D81DC01ED91FC910488B7
:107F7000F589E02D19950E9412656093710970933F
:107F800072098093730990937409609375097093D3
:107F900076098093770990937809DF91CF910895BE
:107FA000CF92DF92EF92FF920F931F93CF93DF93C5
:107FB000D82E7B018A01C22E68E270E00E946E45D5
:107FC000D82F69E270E08D2D0E946E45CD2FD0E054
:107FD000DC2FCC27C80FD11D6D2D6295660F607EFA
:107FE000685E9801A701CE010E94C12BC1100EC08E
:107FF000C00FD11F4D2F68E270E08D2D0E942043ED
:108000004C2F69E270E08D2D0E942043DF91CF91CB
:108010001F910F91FF90EF90DF90CF900895FF9206
:108020000F931F93CF93DF93F82E00E010E08F2D76
:108030000E946B42EC01892B21F08F2D0E946B4234
:108040008C01C017D10799F7CE01DF91CF911F9115
:108050000F91FF900895CF93DF93EC01898D9A8D56
:10806000892B41F0E881F9810284F385E02DCE016E
:108070001995F4CFDF91CF910895CF93DF931F929D
:10808000CDB7DEB76983DC01ED91FC910280F3810D
:10809000E02D41E050E0BE016F5F7F4F19950F90DA
:1080A000DF91CF910895FC01818D928D0895FC019F
:1080B0008589968908952DE633E0FC01318320837C
:1080C000FB014189528963897489FC01428353838E
:1080D000648375830895DC01ED91FC91048CF58D2A
:1080E000E02D199480E00895FC019485FB018485BE
:1080F000981303C081E0983009F480E0089521E0EE
:10810000FC018485883009F420E0822F08950895C9
:10811000CF93DF931F92CDB7DEB76983DC01ED917A
:10812000FC910280F381E02D41E050E0BE016F5FE1
:108130007F4F19950F90DF91CF9108950F931F9363
:10814000CF93DF931F92CDB7DEB78C01DC01ED91A9
:10815000FC910084F185E02D1995892B69F021E0CF
:1081600041E050E0BE016F5F7F4FF80184850E94BF
:10817000D03F898190E002C08FEF9FEF0F90DF9199
:10818000CF911F910F910895CF93DF931F92CDB799
:10819000DEB7FC01218D328D232B61F021E041E01F
:1081A00050E0BE016F5F7F4F84850E94D03F898180
:1081B00090E002C08FEF9FEF0F90DF91CF91089575
:1081C000CF92DF92EF92FF921F93CF93DF93182FFE
:1081D0006B017A010E940F40EC01009799F463E073
:1081E00070E0812F0E946E458431F1F08823E1F028
:1081F000C1E0D0E08C3111F4C0E0D0E0D195C19560
:10820000D10912C0E816F9060CF4E7011C161D0688
:108210005CF420E0AE01B601812F0E94D03F60E403
:1082200070E0812F0E94C73CCE01DF91CF911F915A
:10823000FF90EF90DF90CF900895CF93DF93FC01F4
:10824000218D328D2115310519F48FEF9FEF11C06B
:10825000EC014217530708F0A9018C850E94E04009
:108260001816190694F7298D3A8D281B390B3A8F69
:10827000298FDF91CF9108950F931F93CF93DF93B1
:108280001F92CDB7DEB7FC01218D328D232B61F01B
:108290008C0141E050E0BE016F5F7F4F84850E94FA
:1082A000E040181619061CF08FEF9FEF08C0F80188
:1082B000818D928D0197928F818F898190E00F90AF
:1082C000DF91CF911F910F910895FC0184850C944B
:1082D000E040CF93DF931F92CDB7DEB741E050E08F
:1082E000BE016F5F7F4FFC0184850E94E04018163D
:1082F00019061CF4898190E002C08FEF9FEF0F9068
:10830000DF91CF910895FC018485883011F00C94A1
:108310000F4080E090E008950F931F93CF93DF9379
:10832000CDB7DEB728970FB6F894DEBF0FBECDBF2E
:108330008C01DC01ED91FC910680F781E02D19950F
:10834000F80184850E940F40892B51F148E050E0EC
:10835000BE016F5F7F4FD8011C968C910E94E04058
:1083600018161906FCF4D801519684E0FE013196E6
:1083700001900D928A95E1F78D8190E0982F8827E2
:108380002E81820F911DF801968B858B8F8190E055
:10839000982F88272885820F911D928F818F02C088
:1083A00080E090E028960FB6F894DEBF0FBECDBFF8
:1083B000DF91CF911F910F910895AF92BF92CF920D
:1083C000DF92FF920F931F93CF93DF938C015B019A
:1083D000EA01FC01C788D08CF4848F2D0E94BA5822
:1083E0008C179D0720F48F2D0E94BA58EC019E0136
:1083F000A501B6018F2D0E947B58F8018789908DC9
:108400008C0F9D1F908F878BCE01DF91CF911F9195
:108410000F91FF90DF90CF90BF90AF900895EF92B3
:10842000FF921F93CF93DF93FC012485283011F036
:1084300080E01DC07B01EC0110E063E070E0812F63
:108440000E946E45811102C01C8705C08831E1F38E
:108450001F5F183091F78C85883051F3FE86ED86CA
:108460001A8E198EA70162E00E94D65881E0DF9132
:10847000CF911F91FF90EF900895CF93DF93FC0170
:1084800024852830D1F0EC010E94BD3C843181F07C
:10849000882371F0883161F08C3161F4E881F981D1
:1084A0000084F185E02DCE01199521E0892B19F486
:1084B00020E001C021E0822F01C080E0DF91CF9158
:1084C000089561E08091DB080C946D6460E0809118
:1084D000DB080C946D641F93CF93DF93182F66E233
:1084E00070E00E946E45C82FD0E0DC2FCC2767E2F9
:1084F00070E0812F0E946E459E01280F311DC90139
:10850000DF91CF911F9108951F93CF93DF93182F81
:1085100060E270E00E946E45C82FD0E0DC2FCC27CF
:1085200061E270E0812F0E946E459E01280F311D8F
:10853000C901DF91CF911F91089508958EBD00006C
:108540000DB407FEFDCF8EB508958CBD9DBD089579
:108550001F93CF93DF93D82F192FC62F8091D9085F
:108560009091DA080E94A5420E946642812F0E94E3
:108570009E428D2F0E949E428C2F0E949E4280E040
:108580000E949E42C82F0E9461428C2FDF91CF91A2
:108590001F910895DF92EF92FF920F931F93CF9355
:1085A000DF93D82FD92EC62F7A0189018091D9085F
:1085B0009091DA080E94A5420E9466428D2D0E9489
:1085C0009E428D2F0E949E428C2F0E949E42E70168
:1085D000E00EF11ECE15DF0521F089910E949E422A
:1085E000F9CF0E946142C801DF91CF911F910F9195
:1085F000FF90EF90DF9008950F931F93CF93DF9339
:10860000182F092FD62FC42F8091D9089091DA08FE
:108610000E94A5420E946642802F0E949E42812FA6
:108620000E949E428D2F0E949E428C2F0E949E424D
:108630000E94614281E0DF91CF911F910F910895D7
:108640009B018295880F807E6CE0680FC9010C94B5
:10865000FC42CF93C82F60E170E00E94C73C4FEF0F
:1086600062E070E08C2FCF910C942043CF93DF9386
:10867000FC018485883029F0EF010E94294388E0BD
:108680008C87DF91CF910895CF92DF92EF92FF9286
:10869000CF93DF93EC018C858830B9F168E070E00E
:1086A0000E94C73C0E9412656B017C01CE010E94B2
:1086B000BD3C8823A1F00E941265DC01CB018C191E
:1086C0009D09AE09BF09883E9340A105B10538F464
:1086D00061E070E080E090E00E94D864E7CFCE01D6
:1086E0000E94BD3C882319F08C850E94294388E0B4
:1086F0008C8763E175E086E398E0DF91CF91FF908E
:10870000EF90DF90CF900C94D73CDF91CF91FF900A
:10871000EF90DF90CF9008958F929F92AF92BF928B
:10872000CF92DF92EF92FF920F931F93CF936C0142
:108730005B017A01FC01C485C83041F481E090E01E
:10874000F6019383828380E090E041C08A0141304A
:10875000584010F000E018E08C2F0E94BA584C01ED
:1087600063E070E08C2F0E946E45873111F08C31F0
:1087700021F48016910680F302C000E010E0980119
:10878000A50160E070E08C2F0E947B5860E270E0F1
:108790008C2F0E94C73C62E070E08C2F0E946E45D7
:1087A00084FD0BC063E070E08C2F0E946E45811148
:1087B000F2CF8C2F0E942943C1CF40E162E070E0EC
:1087C0008C2F0E942043012B09F4B8CFC701CF9111
:1087D0001F910F91FF90EF90DF90CF90BF90AF90DF
:1087E0009F908F900895CF93FC01C48560E270E064
:1087F0008C2F0E94C73C62E070E08C2F0E946E4577
:1088000084FD10C062E070E08C2F0E946E4583FFF3
:10881000F2CF48E162E070E08C2F0E94204380E0BC
:1088200090E008C040E162E070E08C2F0E9420439D
:1088300081E090E0CF9108951F93CF93DF93FB01E8
:10884000DC0158961C921E9257972281211109C073
:108850002381211106C02481211103C025812223F7
:1088600021F14115510509F1EA01DC011C961C9129
:10887000AF014E5F5F4F612F6295660F607E645F50
:1088800024E030E08CE090E00E94CA424D2F60E18D
:1088900070E0812F0E9420434C2F61E170E0812F16
:1088A0000E94204381E090E002C080E090E0DF91F0
:1088B000CF911F910895FC011382128288EE93E0FC
:1088C000A0E0B0E084839583A683B7838FEA92E02B
:1088D0009183808388E084878DE693E0908B8787FF
:1088E000118A128A138A148A0895AF92BF92CF9286
:1088F000DF92EF92FF920F931F93CF93DF93CDB749
:10890000DEB7AF970FB6F894DEBF0FBECDBF7C01C8
:108910005B016A010DE613E01A8309831B821C8246
:108920001D821E82CE0109960E945B441BA70AA7E6
:108930001CA61DA61EA61FA68091DE089091DF082A
:10894000A091E008B091E1088EA39FA3A8A7B9A7C2
:108950008B839C83AD83BE8318861F82AE01465DE8
:108960005F4FB501CE0101960E941E6581309105D1
:10897000B1F4D701ED91FC910488F589E02D1DA398
:108980000CA38CA59DA5AEA5BFA58EA39FA3A8A74C
:10899000B9A7A601BE016C5D7F4FC7011995AF96BF
:1089A0000FB6F894DEBF0FBECDBFDF91CF911F9100
:1089B0000F91FF90EF90DF90CF90BF90AF90089510
:1089C000DC01ED91FC91028CF38DE02D199591E085
:1089D00089270895CF93DF931F92CDB7DEB78983A0
:1089E00020916C073981E0916D07F0916E07822F1D
:1089F00090E080959095F8940080082200824BE0EA
:108A000000C05DE000005A95E9F700800822089454
:108A1000379508F4022A00824A9599F778940F90C6
:108A2000DF91CF91089585ED8093BC008091BC00CB
:108A300084FDFCCF10924607089540912207262F0F
:108A400030E0240F311D21323105DCF4209146073E
:108A50002430C9F4FC0180E090E0861758F430918E
:108A600022072191DC01AE5FB84FA30FB11D2C93FB
:108A70000196F3CF80912207680F6093220780E070
:108A8000089581E0089582E008958FEF9FEF0895A3
:108A90008FEF9FEF08958091010790E09195819568
:108AA00091090895CF93DF93CB01EA01642F0E94CF
:108AB0001D45CE01DF91CF910895CF93DF931F9293
:108AC000CDB7DEB7698361E0CE0101960E941D45F6
:108AD00081E090E00F90DF91CF9108959B01829506
:108AE000880F807E68E0680FC9010C94A8428F92BD
:108AF0009F92AF92BF92CF92DF92EF92FF920F932D
:108B00001F93CF93DF93EC018B017A016C85683062
:108B100069F04AE050E086E398E00E94745F6AE101
:108B200075E086E398E00E94D73C12C186E398E0A6
:108B30000E94C65FC12CD12CAC2C63E070E08C2D60
:108B40000E946E45B82E69E275E086E398E00E94C7
:108B5000CA5F40E150E0B60186E398E00E946D5F95
:108B60006DE275E086E398E00E94CA5F40E150E064
:108B70006B2D86E398E00E94745F86E398E00E9484
:108B8000C65FB11013C0AC8666E375E086E398E07B
:108B90000E94CA5F40E150E06C8586E398E00E9445
:108BA000745F86E398E00E94C65F0CC08B2D8B7FBC
:108BB000883149F38FEFC81AD80AE8E0CE16D104FD
:108BC00009F0BACF8C85883009F4C2C0C090030286
:108BD000D0900402FFEFCF1ADF0A0E941265DC0179
:108BE000CB019927AA27BB27B601680F791F61150A
:108BF00084E0780728F0709304026093030206C0B3
:108C000080E094E090930402809303024091030279
:108C10005091040261E08C850E94D6586801E2E020
:108C2000CE0ED11C46015801F6E0AF0EB11CF40186
:108C300061914F014AE050E086E398E00E94745F42
:108C40006DE874E086E398E00E94CA5FA814B90456
:108C500071F786E398E00E94C65FF80182818F3F3A
:108C600051F483818F3FA1F484818F3F89F4858102
:108C70008F3F71F46BC081110BC0F80183818111AA
:108C800007C08481811104C08581882309F45EC0F6
:108C9000E114F10409F45AC01C85612F6295660F36
:108CA000607E645F24E030E0A6018CE090E00E94EA
:108CB000CA424F2D60E170E0812F0E9420434E2D6B
:108CC00061E170E0812F0E94204364E070E0812F19
:108CD0000E94C73C0E9412654B015C016B017C0144
:108CE000F8E9CF0EFAE3DF1EE11CF11CCE010E9471
:108CF000BD3C873129F08C149D04AE04BF0420F0E4
:108D00000E94126597FD15C00E9412656C157D05C5
:108D10008E059F0570F06BE475E086E398E00E9495
:108D2000D73CE881F9810488F589E02DCE011995B9
:108D30000FC06AE070E080E090E00E94D8640E947A
:108D4000F22FCE010E94BD3C811105C088E08C87C6
:108D500080E090E00DC0CE010E94BD3C873131F62D
:108D60006FE375E086E398E00E94D73C81E090E0F5
:108D7000DF91CF911F910F91FF90EF90DF90CF90F7
:108D8000BF90AF909F908F90089524E030E0AC01A9
:108D900064E08FE090E00C94CA4224E030E0AC0143
:108DA00064E085E090E00C94CA4224E030E0AC013D
:108DB00064E081E090E00C94CA4278941F920F9294
:108DC0000FB60F9211240BB60F92CF92DF92EF9253
:108DD000FF920F931F932F933F934F935F936F9344
:108DE0007F938F939F93AF93BF93CF93DF93EF9333
:108DF000FF93809170008E7F809370000FE310E0EE
:108E00008BE1E82EF12C9BE2C92ED12CC0916F078B
:108E1000D09170072097F9F40332110508F43BC094
:108E200003521109E0916D07F0916E079081209136
:108E30006C07822F8095982390839BE0D701119730
:108E4000F1F79150D9F78081822B8083C601019779
:108E5000F1F780E00DC00B301105E8F00B5011095F
:108E6000E0917107F0917207EC0FFD1F319780813F
:108E70000E94EA442196D0937007C0936F078091B7
:108E80000102909102028C179D0708F0BFCF10924B
:108E9000700710926F07809170008160809370005E
:108EA000FF91EF91DF91CF91BF91AF919F918F9102
:108EB0007F916F915F914F913F912F911F910F91F2
:108EC000FF90EF90DF90CF900F900BBE0F900FBEF2
:108ED0000F901F90189581E0809300078091000209
:108EE000282F30E0F901E953FE4EE491F0E0EE0F57
:108EF000FF1FE355FE4E4591549150936E074093EA
:108F00006D07F901E35FFD4EE491E0936C0761E0CA
:108F10000E949C6483E08093B100E0E7F0E08081F0
:108F2000816080830895CF93DF931816190644F06B
:108F3000809170008E7F809370001092000719C09E
:108F4000EC0180917107909172070E946D72CE01C1
:108F5000C130D24014F080E092E0909302028093FE
:108F600001020E94D5719093720780937107892B3B
:108F700029F4109202021092010208C080910007A9
:108F8000811104C0DF91CF910C946B47DF91CF9199
:108F90000895FF920F931F93CF93DF938C01F62ECA
:108FA00080910007811102C00E946B47E801219760
:108FB000C11582E0D80798F48091010290910202D5
:108FC0008017910718F4C8010E9493478091710798
:108FD00090917207009719F0C80FD91FF882DF919E
:108FE000CF911F910F91FF9008951F920F920FB68E
:108FF0000F9211240BB60F922F933F934F935F93D1
:109000006F937F938F939F93AF93BF93EF93FF9350
:109010008091B900887F803609F49CC068F5883259
:1090200009F45BC090F4803109F454C038F488230B
:1090300009F4F2C0883009F44DC0F2C0883109F457
:109040004CC0803209F45DC0EBC0803409F468C0C4
:1090500048F4803309F455C0883309F0E1C08093A7
:109060004507D4C0803509F44FC0883509F45DC088
:10907000883409F0D5C0D2C0883909F4C3C0A8F437
:10908000883709F467C038F4883609F463C080373C
:1090900009F460C0C5C0883809F4B4C0803909F447
:1090A0005FC0803809F0BCC05BC0803B09F484C05D
:1090B00038F4803A09F466C0883A09F47DC0B0C03B
:1090C000803C09F4A3C0883C09F4A0C0883B09F4A3
:1090D00086C0A6C080916B0710C090916A078091EE
:1090E0006907981770F5E0916A0781E08E0F809309
:1090F0006A07F0E0E75BF84F80818093BB0085EC66
:1091000082C0809345078AC0E0916A0781E08E0F94
:1091100080936A078091BB00F0E0E75BF84F8083A3
:1091200090916A07809169076AC0E0916A0781E0BF
:109130008E0F80936A078091BB00F0E0E75BF84FE9
:10914000808380914807811169C081E0809347073F
:1091500084EA5DC083E08093460710924407CFCF36
:1091600080914407803208F04DC0E091440781E0CF
:109170008E0F809344078091BB00F0E0EC5DF84FC8
:109180008083BDCF85EC8093BC0010924607809110
:109190004407803230F4E0914407F0E0EC5DF84F92
:1091A00010826091440770E084E297E0E0E0F0E034
:1091B00019951092440734C084E0809346071092BA
:1091C000230710922207E0E0F0E019958091220732
:1091D000811105C081E08093220710920207E0917F
:1091E000230781E08E0F80932307F0E0EE5FF84FB6
:1091F00080818093BB00909123078091220798176C
:1092000008F47DCF85E88093BC000AC085EC80938C
:10921000BC001092460704C0109245070E941345F7
:10922000FF91EF91BF91AF919F918F917F916F913E
:109230005F914F913F912F910F900BBE0F900FBEFA
:109240000F901F90189508958F929F92AF92BF92A2
:10925000CF92DF92EF92FF920F931F93CF93DF9302
:10926000CDB7DEB72B970FB6F894DEBF0FBECDBFDC
:109270008C01CE0101967C016C018AE0882E912C34
:10928000A12CB12CC6018E199F094115510561050C
:10929000710581F0CB01BA01A50194010E94247CE3
:1092A000942F852F605DF60161936F01A901692FED
:1092B000782FE8CFFC013197EE0DFF1DD8019E01FC
:1092C0002150310940814D933197E217F307D1F7CF
:1092D000F801E80FF91F10822B960FB6F894DEBF45
:1092E0000FBECDBFDF91CF911F910F91FF90EF90F7
:1092F000DF90CF90BF90AF909F908F9008958F9206
:109300009F92AF92BF92CF92DF92EF92FF920F9314
:109310001F93CF93DF938C014A016901E090FE0611
:10932000F090FF06C62F660FDD0BE114F10449F142
:10933000F7018085863029F563E575E0C7010E9455
:10934000BD505C01F2E08F16910439F083E088167D
:10935000910451F46FE475E002C068E575E0C7015F
:109360000E94BD507C0102C0E12CF12CA114B1047B
:1093700051F0F50161857285AE01C8010E940A8134
:1093800008C0E12CF12CAE016FE470E1C8010E942D
:10939000FA74AE016CEC73E0C8010E94EC80E11439
:1093A000F10421F0F701618572850FC0F2E08F169C
:1093B0009104A1F083E08816910461F08A948928D1
:1093C00099F46091FC067091FD06AE01C8010E94FF
:1093D000EC800AC0AE0169E470E103C0AE0166E44E
:1093E00070E1C8010E94DC74AE016CEC73E0C8014E
:1093F0000E94EC80C114D10429F0AE01B601C8016D
:109400000E94EC80C801DF91CF911F910F91FF90D6
:10941000EF90DF90CF90BF90AF909F908F90089586
:10942000CF93DF931F921F92CDB7DEB78091270BAA
:109430009091280B009711F483E39BE0BE016F5FCE
:109440007F4F681B790B072E000C880B990B0F9030
:109450000F90DF91CF910895AF92BF92CF92DF929C
:10946000EF92FF920F931F93CF93DF93CDB7DEB7A9
:10947000AF970FB6F894DEBF0FBECDBF7C015B0186
:109480006A010DE613E01A8309831B821C821D8288
:109490001E82CE0109960E945B441BA70AA71CA648
:1094A0001DA61EA61FA68091DE089091DF08A09140
:1094B000E008B091E1088EA39FA3A8A7B9A78B836A
:1094C0009C83AD83BE8318861F82AE01465D5F4FCD
:1094D000B501CE0101960E941E6581309105B1F45F
:1094E000D701ED91FC910684F785E02D1DA30CA317
:1094F0008CA59DA5AEA5BFA58EA39FA3A8A7B9A720
:10950000A601BE016C5D7F4FC7011995AF960FB6DE
:10951000F894DEBF0FBECDBFDF91CF911F910F91A9
:10952000FF90EF90DF90CF90BF90AF900895FC0137
:109530008481958108950895AF92BF92CF92DF9272
:10954000EF92FF920F931F93CF93DF93CDB7DEB7C8
:10955000C154D1090FB6F894DEBF0FBECDBF5C0178
:109560006B018A0167E671E186E398E00E94A35EE1
:10957000B50186E398E00E94CA5F64E671E186E384
:1095800098E00E94A35EC114D10409F4A1C00C0D9F
:109590001D1DF80110820E94104A6A3F71051CF4DB
:1095A0006FE571E14DC07601E016F10641F0F7017B
:1095B00061917F0186E398E00E949C5EF5CF86E38F
:1095C00098E00E94C65F80919205909193059E015C
:1095D0002F5F3F4F790120E030E0049719F443E01A
:1095E00050E019C042E050E061E4C7010E947F49A9
:1095F000F70101900020E9F731978F010E191F093B
:10960000A801B701C5010E94FC800097A9F020E0E5
:1096100030E041E050E061E4C7010E947F49F7017A
:1096200001900020E9F731978F010E191F09A80159
:10963000B701C5010E94FC80892B39F064E571E116
:1096400086E398E00E94A35E43C00A0D1B1D6DE5F2
:1096500075E0C8010E94DC80892B69F4F601019055
:109660000020E9F73197EC19FD09329720F0C60187
:109670000E94F8612DC06FE270E0C8010E94D180A5
:109680005C01009741F0FC0110828181843201F17C
:10969000FFEFAF1ABF0AF80180818432C9F0B80128
:1096A000C7010E946D54C7010E946822882369F097
:1096B00041E08091920590919305049709F440E070
:1096C0009501B601C7010E947C1DC7010E942F5160
:1096D000CF5BDF4F0FB6F894DEBF0FBECDBFDF917B
:1096E000CF911F910F91FF90EF90DF90CF90BF909F
:1096F000AF9008958F929F92AF92BF92CF92DF92D8
:10970000EF92FF920F931F93CF93DF93CDB7DEB706
:109710002C970FB6F894DEBF0FBECDBFF82EE92E02
:109720006B015A01490181E090E090938F0580938D
:109730008E0526E240E855E260E070E089E997E0B6
:109740000E94FA53F0928C0989E997E090938B0973
:1097500080938A091092970A1092990A1092980A97
:109760008114910439F08A94892829F4102F002754
:109770000F6F01C01F6FC801A0E0B0E089839A831A
:10978000AB83BC8380E190E09E838D83A60160E083
:1097900070E04F83588769877A879C878B874AE078
:1097A00050E06F2D7E2D86E398E00E946D5F64E3AC
:1097B00071E186E398E00E94A35EBE01695F7F4F7E
:1097C00086E398E00E9412247C0160E371E10E942C
:1097D000A35E4AE050E0B501C7010E946D5F6DE2F3
:1097E00071E1C7010E94A35EBE016F5F7F4FC70199
:1097F0000E9412240E94C65FA114B10491F082E07D
:10980000A816B10409F5D092120AC092110A10925A
:10981000140A1092130A1093160A0093150A86E090
:1098200010C0D092120AC092110A011103C080E048
:1098300090E002C080E09FEF9093140A8093130A97
:1098400085E00E94435106C065E171E186E398E03E
:109850000E94A35E10928F0510928E052C960FB673
:10986000F894DEBF0FBECDBFDF91CF911F910F9156
:10987000FF90EF90DF90CF90BF90AF909F908F9030
:109880000895DF92EF92FF920F931F93CF93DF9390
:1098900000D000D0CDB7DEB76CE671E186E398E08A
:1098A0000E94A35E05E717E0D12C80E1E82EF12CA1
:1098B000F8018081803130F466E675E086E398E057
:1098C0000E94CA5FF8018081F5E090E0A0E0B0E07E
:1098D00089839A83AB83BC83FE82ED82BE016F5F76
:1098E0007F4F86E398E0DF1639F00E9412246AE683
:1098F00071E10E94A35E04C00E9412240E94C65F10
:10990000D3940F5F1F4F86E0D812D2CF26960FB6A2
:10991000F894DEBF0FBECDBFDF91CF911F910F91A5
:10992000FF90EF90DF900895CF92DF92EF92FF9239
:109930008091E4069091E506892B09F44CC00E94C1
:10994000104A6B017C016CE371E186E398E00E94B0
:10995000A35E2AE0B701A60186E398E00E94DC5EE0
:109960008091E4069091E5060E94713C1092E50614
:109970001092E4061092E7061092E6061092740721
:10998000109273071092FF061092FE061092F506D1
:109990001092F4061092F9061092F8061092F7064B
:1099A0001092F6060E94104A6B017C0167E371E198
:1099B00086E398E00E94A35E2AE0B701A60186E351
:1099C00098E00E94DC5E86E398E0FF90EF90DF90E5
:1099D000CF900C94C65FFF90EF90DF90CF900895EA
:1099E00080E090E008958F929F92AF92BF92DF92B5
:1099F000EF92FF920F931F93CF93DF93CDB7DEB714
:109A0000C854D1090FB6F894DEBF0FBECDBF7C019C
:109A10008B010E94AB23D82E5801AA2488E0B822DB
:109A200013FF10C0B80166277370C7010E942E2370
:109A300064E071E186E398E00E94A35EAA24AA9400
:109A4000BA2CD8C160E073E0C7010E946923082BDB
:109A5000192B1AAA19AAFE01F3968EE0DF011D92B6
:109A60008A95E9F723961FAE1EAE2397709686E07F
:109A7000DF011D928A95E9F711FF45C0C7010E94D9
:109A8000AD22F70140859E012F5C3F4F413038F1F8
:109A9000433020F0473019F597FF13C01F926F93A2
:109AA0001F927F939F779F938F9388E695E09F9374
:109AB0008F931F9280E18F933F932F930E94248175
:109AC0001DC01F926F938EE695E09F938F931F9218
:109AD00080E18F933F932F930E9424810FC09F9327
:109AE0008F937F936F938EE695E09F938F931F9252
:109AF00080E18F933F932F930E9424810FB6F894B7
:109B0000DEBF0FBECDBF10FF1EC08D2D90E0803197
:109B1000910590F4FC018827EF52FF4F8F4F0C9472
:109B2000877C61E071E102C06DEF70E1CE018F5B77
:109B30009F4F0E94D57407C06FEE70E186E398E0F6
:109B40000E94A35E1E7F20E030E043E050E060E32F
:109B5000CE0101960E947F49D7011296ED91FC91AA
:109B600013976081718140E350E0CE0101960E941D
:109B7000EC800E941455882309F438C180918D052A
:109B8000811134C148018824B2E09B2211FF2DC00D
:109B90008D2D90E08230910541F1059731F1BE01A4
:109BA0006F5C7F4FCE0101960E949D5569EE70E17A
:109BB00086E398E00E94A35EBE016F5F7F4F86E35D
:109BC00098E00E94CA5F66EE70E186E398E00E942A
:109BD000A35EBE016F5C7F4F86E398E00E94CA5F80
:109BE00086E398E00E94C65F2AC010FF25C0BE0130
:109BF0006F5B7F4FCE0101960E949D5560EE70E134
:109C000086E398E00E94A35EBE016F5F7F4F86E30C
:109C100098E00E94CA5F6DED70E186E398E00E94D3
:109C2000A35EBE016F5B7F4F86E398E00E94CA5F30
:109C300086E398E00E94C65F892809F457C020E0B7
:109C400030E043E050E060E3CE0101960E947F499E
:109C5000D7011296ED91FC9113976081718140E3D9
:109C600050E0CE0101960E94EC806CEC73E0CE01D6
:109C700001960E94C68040E350E069ED70E1CE019C
:109C800001960E94DC7463ED70E186E398E00E9427
:109C9000A35EBE016F5F7F4F86E398E00E94CA5FBC
:109CA00060ED70E186E398E00E94A35EBE016F5C08
:109CB0007F4F86E398E00E94CA5F86E398E00E94A7
:109CC000C65F0E941455882309F490C080918D05C9
:109CD00081118CC0BE016F5C7F4FCE0101960E9446
:109CE0009D5560E072E0C7010E94F12210FF7AC02A
:109CF000BAE0DB16D1F0BD1538F0E1E0DE1681F0F8
:109D0000F6E0DF1669F018C08BE0D81631F09CE061
:109D1000D91212C06BEC70E10AC061EC70E107C0AF
:109D2000D70118968C91853039F466EC70E1CE013C
:109D30008F5B9F4F0E94D57420E030E043E050E0FD
:109D400060E3CE0101960E947F49D7011296ED9102
:109D5000FC9113976081718140E350E0CE01019640
:109D60000E94EC806CEC73E0CE0101960E94C680EC
:109D700040E350E06DEB70E1CE0101960E94DC748F
:109D800067EB70E186E398E00E94A35EBE016F5F1F
:109D90007F4F86E398E00E94CA5F64EB70E186E340
:109DA00098E00E94A35EBE016F5B7F4F86E398E060
:109DB0000E94CA5F86E398E00E94C65F0E94145525
:109DC0008823A1F080918D05811110C0BE016F5BC9
:109DD0007F4FCE0101960E949D5560E071E0C70162
:109DE0000E94F122AA24A394B12C04C0B801C70197
:109DF0000E942E23C501C85BDF4F0FB6F894DEBF6B
:109E00000FBECDBFDF91CF911F910F91FF90EF90CB
:109E1000DF90BF90AF909F908F900895CF93DF9386
:109E2000EC0162EA70E186E398E00E94A35E60E0E4
:109E300074E0CE01DF91CF910C942E232F923F92AC
:109E40004F925F926F927F928F929F92AF92BF924A
:109E5000CF92DF92EF92FF920F931F93CF93DF93F6
:109E600000D01F92CDB7DEB76C013B010E94AB233F
:109E7000823011F0853011F4612C712CF6010480D0
:109E8000F581E02DFC83EB838085853009F078C077
:109E9000CF010E945F54082F10E0023011050CF42E
:109EA0006FC060E08B819C810E948C67FC014184C3
:109EB000528461E08B819C810E948C67FC018184CB
:109EC0009284A384B48480918E0590918F059A83A7
:109ED00089830230110509F448C062E08B819C81BE
:109EE0000E948C67FC01E184F2840330110509F4BF
:109EF0003FC063E08B819C810E948C67FC012184C0
:109F000032840430110549F064E08B819C810E9409
:109F10008C67FC018185928502C082E090E09C8381
:109F20008B8321143104A1F0E981FA81EF2B21F018
:109F3000C6010E940E4F24C09301D1010E949E7C55
:109F400024E630E040E050E00E94467C890105C0F4
:109F500089819A81892B61F7830197014B815C810B
:109F6000B401C2010E947A4B0BC0EE24EA94FE2C8D
:109F70008FE3282E312CE2E0F0E0FC83EB83D4CF9A
:109F800080E090E00F900F900F900F90DF91CF91B5
:109F90001F910F91FF90EF90DF90CF90BF90AF9007
:109FA0009F908F907F906F905F904F903F902F90F9
:109FB0000895EF92FF920F931F93CF93DF93CDB746
:109FC000DEB72B970FB6F894DEBF0FBECDBF7C0176
:109FD000DC011296ED91FC9113976081718186E30B
:109FE00098E00E94CA5FC7010E94682281110DC0DB
:109FF00069E970E186E398E00E94A35E86E398E059
:10A000000E94C65F8FEF9FEFABC0C7010E94AB23DA
:10A01000F70110851730F1F0853099F028F4813080
:10A0200049F0823071F016C0863021F0E6EFE80F7B
:10A03000E33080F460E970E186E398E00E94A35E7B
:10A0400083C065E870E186E398E00E94A35E80E04B
:10A0500090E086C0D70119968D919C911A97009730
:10A0600041F0DC01ED91FC910688F789E02D19950E
:10A0700077C0C7010E94AD22812F90E08A30910500
:10A0800008F046C0FC018827EF51FF4F8F4F0C941A
:10A09000877CD7011496ED91FC91159780858530CA
:10A0A000D1F56FE770E186E398E00E94A35ED701E7
:10A0B0001496ED91FC9115970681178101151105F4
:10A0C000F9F0F80161857285CE0101960E946D5408
:10A0D000CE0101960E9468228823C1F1CE0101962B
:10A0E0000E94D94F181619068CF566E770E186E3D1
:10A0F00098E00E94A35ECE0101960E942F5124C0D9
:10A100006BE670E1A0CF062F10E007C08B0105C001
:10A1100061E670E198CF00E010E066E570E186E36B
:10A1200098E00E94A35E4AE050E0B80186E398E020
:10A130000E946D5F86E398E00E94C65F81E090E038
:10A14000012B71F480E00CC081E082CFD80112961F
:10A150000D911C911397CE0101960E942F51AECF05
:10A160002B960FB6F894DEBF0FBECDBFDF91CF9117
:10A170001F910F91FF90EF9008950F931F93CF932E
:10A18000DF938B01FC01C681D781209759F0B8017C
:10A19000888199810E94B380892B21F00A80DB811C
:10A1A000C02DF3CFCE01DF91CF911F910F91089574
:10A1B000DC011696ED91FC91179761157105A1F0E0
:10A1C000309729F417967C936E93169708958281A1
:10A1D0009381009711F0FC01FACF73836283DB0156
:10A1E0001596FC93EE9314970895CF92DF92EF9219
:10A1F000FF920F931F93CF93DF938C017B016A0132
:10A200000E946F2AEC01892B09F182E08887A60160
:10A21000DD0C660B770B49875A876B877C878881B3
:10A220009981009711F00E946D72C7010E947A8097
:10A2300099838883BE01C801DF91CF911F910F914F
:10A24000FF90EF90DF90CF900C94D850DF91CF919A
:10A250001F910F91FF90EF90DF90CF90089527ED21
:10A2600032E0DC0111963C932E9319968D919C91CE
:10A270001A97009739F0DC01ED91FC910280F3818F
:10A28000E02D199408958F929F92AF92BF92CF9232
:10A29000DF92EF92FF920F931F93CF93DF93CDB78F
:10A2A000DEB7DA950FB6F894DEBF0FBECDBFC82E6D
:10A2B00080918C098983CA8221E0C216A0F074E0E3
:10A2C0007C1518F487E1C8120EC080918D09909119
:10A2D0008E099B838C8380918F09909190099D8337
:10A2E0008E8386E001C082E08E010F5F1F4F90E1F8
:10A2F0009C1528F0AFE0CA1630F49BEF01C09AEE2F
:10A300009C0D923078F42091110A9091120AF80174
:10A31000E80FF11D908391E0980FF801E90FF11D0E
:10A320008E5F2083BFE0CB1641F1BC1558F0E5E00D
:10A33000CE16A1F0F6E0CF12B6C02091150A90918A
:10A34000160A10C026E1C21609F48EC077E1C716BE
:10A3500009F459C090E1C912A6C055C02091130A52
:10A360009091140AF801E80FF11D908391E0980F85
:10A37000F801E90FF11D8E5F95C02091130A30910D
:10A38000140AF801E80FF11D308342E0480F91E014
:10A39000980FF801E90FF11D2083B9016770772745
:10A3A000A3E036952795AA95E1F7672B19F091E080
:10A3B000920F01C0922FB3E0B80FF801E40FF11D26
:10A3C00090838C5F60E070E0A0E04FEF480F9A133D
:10A3D00003C08B2F890F67C050E09B0135952795EF
:10A3E000400F511F220F331FF901EB5EF54FA0FD07
:10A3F00002C0208101C02181FA012083AF5F6F5F1D
:10A400007F4F8F5FE2CF2091130A3091140AF80139
:10A41000E80FF11D308391E0980FF801E90FF11D6D
:10A42000208392E0980FF801E90FF11D8D5F922FC4
:10A43000990F908390E03327E92FF0E0E217F307BC
:10A4400094F5EE0FFF1FEB5EF54F50814181F8014F
:10A45000E80FF11D408341E0480FF801E40FF11DC2
:10A460008E5F50839F5FE8CF9091150A2091160A66
:10A47000F801E80FF11D208321E0280FF801E20F19
:10A48000F11D90832091170A9091180A32E0380F3D
:10A49000F801E30FF11D908393E0980FF801E90FA5
:10A4A000F11D8C5F20837801F8012FEF3FEFD02E54
:10A4B0009E2F901B9817A0F49191292748E050E017
:10A4C000B9017695679520FF06C09B0191E0292789
:10A4D00090EA392701C09B014150510989F7E8CF23
:10A4E000F801E80FF11D2083B2E0BB2EB80E8F5F9C
:10A4F000F801E80FF11D3083F801EB0DF11D10821A
:10A5000080918A0990918B09DC01ED91FC91028484
:10A51000F385E02D1995019699F7E091A00AF09145
:10A52000A10A309709F0199580918A0990918B09B9
:10A530002E2D2D192B1558F4F70161917F01DC01A7
:10A54000ED91FC910190F081E02D1995EDCFDC01AA
:10A55000ED91FC910680F781E02D1995E091A20A1A
:10A56000F091A30A309709F019950E9412654B01EA
:10A570005C01A8E0EA2EF12CD12C80918A099091FF
:10A580008B09DC01ED91FC910084F185E02D19959A
:10A59000892BC1F080918A0990918B09DC01ED91A2
:10A5A000FC910284F385E02D199590918C0989170F
:10A5B00011F0FF2099F1F801EF0DF11D8083EA946D
:10A5C000F39407C0E0919E0AF0919F0A309709F03A
:10A5D0001995B5E0FB1222C0EA818E2F8F7790E0AB
:10A5E0008C159D0509F0A2C0E7FF04C08B8188236C
:10A5F00081F181C08E2F90E0FC013197E731F105A8
:10A6000068F48827E551FF4F8F4F0C94877CF3E067
:10A61000EF2E04C0EB8002C0E5E0EE2E0E94126532
:10A62000DC01CB0188199909AA09BB09813D974032
:10A63000A105B10538F480E0EE2031F0882309F45B
:10A640009CCF59C082EEF8CF811155C0F4E0FF15C0
:10A65000C0F58FEF9FEF60E0EF2DF0E09F012250FB
:10A660003109462F50E0D80142175307BCF4A40F1C
:10A67000B51F4C91842748E050E0DC01B695A795C2
:10A6800080FF06C0CD0171E0872770EA972701C0DF
:10A69000CD014150510989F76F5FE3CFA20FB31F7E
:10A6A0002C9130E0AC0155274217530709F040C008
:10A6B000892F9927EC0FFD1F208130E08217930727
:10A6C000B9F58A818530B0F58330B0F5813090F0EE
:10A6D0005B81652F70E07595679520919D0A40E03C
:10A6E000842F90E0861797070CF452C020939D0AA0
:10A6F00050FD6CC080E01092970A1092990A109257
:10A70000980A10929C0AD3950FB6F894DEBF0FBE3C
:10A71000CDBFDF91CF911F910F91FF90EF90DF9010
:10A72000CF90BF90AF909F908F90089581EEE3CF30
:10A7300083EEE1CF8731F1F66B8170E07595679517
:10A7400020919D0A40E0842F90E0861797071CF027
:10A7500020939D0ACFCF4034C0F49C012E5F3F4F21
:10A76000220F331F880F991FFC01E657F64FDE01B9
:10A77000A20FB31F8C9190E0982F8827D801A20FC9
:10A78000B31F2C91822B90878783242F4F5FDBCFC1
:10A790004034C8F4880F991FFC01E657F64FA5E036
:10A7A000B0E0AC0FBD1FA80FB91F2C9130E0322FC5
:10A7B0002227A4E0B0E0AC0FBD1FA80FB91F8C91F9
:10A7C000282B30872783242F4F5F8ACF403468F4AB
:10A7D000880F991FFC01E657F64FDE01A80FB91F3D
:10A7E00014968C9190E09087878381E0840F80930A
:10A7F0009D0A80CFCF92DF92EF92FF921F93CF936B
:10A80000DF93EC016A017B01122FE889F98982E06C
:10A8100080834115514E61057105B1F060E079E02A
:10A820008DE390E0A70196010E94247CDA01C90122
:10A830000197A109B109B695A795979587959C01B0
:10A84000211580E13807A8F0E889F989108260E8CD
:10A8500074E88EE190E0A70196010E94247CDA0161
:10A86000C9010197A109B109B695A7959795879553
:10A870009C01EC85FD853083EE85FF852083188E55
:10A88000EC89FD891083EA89FB898081806180835E
:10A89000EA89FB89808188608083EA89FB898081DD
:10A8A00080688083EA89FB8980818F7D8083DF9146
:10A8B000CF911F91FF90EF90DF90CF900895DC0132
:10A8C0001696ED91FC91179780E0309729F08F5FF5
:10A8D0000280F381E02DF9CF0895CF93DF93EC014F
:10A8E00087ED92E0998388831A8619866115710530
:10A8F00059F08091730790917407009729F00E9496
:10A90000BD509B838A8302C01B821A82CE01DF91D5
:10A91000CF910C94B823CF93DF93EC01FA013296D8
:10A92000E60FF71FDC01AD014C1B5D0BCF01861B51
:10A93000970B2D91222311F02193F5CF9C01241B1D
:10A94000350B620F731FFB013297508331964083A2
:10A95000DF91CF910895EF92FF920F931F93CF93C2
:10A96000DF9300D01F92CDB7DEB77B01BA0130E094
:10A97000962F9F77660F672F661F770B719561156E
:10A98000710509F0906821E0230FE1E0F0E0EC0FA1
:10A99000FD1FE30FF11D90836115710511F0322F3A
:10A9A000E7CF30E0B701621B730B6C5F7F4FDB01B9
:10A9B0008C93DE011196F701E21BF30B359685E0CF
:10A9C000E80EF11CEE16FF0619F08D918193FACF77
:10A9D0008091ED089091EE082F5F3F4F8901040FA1
:10A9E000151FDC01ED91FC910280F381E02DA8019F
:10A9F00019957C010E941265609371097093720928
:10AA0000809373099093740981E00E151F0509F076
:10AA100080E00F900F900F900F90DF91CF911F91DA
:10AA20000F91FF90EF900895CF938091ED08909152
:10AA3000EE08009771F1DC01ED91FC910688F78931
:10AA4000E02D1995C1E0811125C0C0E080918809F1
:10AA500090918909892BF1F48DEF9FEF90938909EB
:10AA6000809388098091ED089091EE08DC01ED91CA
:10AA7000FC910680F781E02D19958091ED08909169
:10AA8000EE08DC01ED91FC910488F589E02D199523
:10AA900001C0C0E08C2FCF910895DF92EF92FF921A
:10AAA0000F931F93CF93DF938C01D62EE72EEA01ED
:10AAB000F22E0E9414558823B9F1F801019000206C
:10AAC000E9F73197E01BF10BCE010796E80FF91F6C
:10AAD000E138F10548F545E050E06FEE78E0C80157
:10AAE0000E948B54AC01ED2DFE2DDC01A151B74F1E
:10AAF0009F012C0F3D1FE217F30719F081918D93F1
:10AB0000FACF2597FF2011F081E301C080E34C0FBD
:10AB10005D1F6FEE78E0DF91CF911F910F91FF9055
:10AB2000EF90DF900C94AB5480E0DF91CF911F91B8
:10AB30000F91FF90EF90DF900895FB0101900020AE
:10AB4000E9F73197AF01461B570B21E00C944D55A7
:10AB50007F928F929F92AF92BF92CF92DF92EF92AD
:10AB6000FF920F931F93CF93DF938C016A017B01B8
:10AB7000722E9A01AB01C701B6010E94337F882370
:10AB800019F061E775E027C046015701E894B7F86E
:10AB90002FEF3FEF4FE75FE7C501B4010E94337F1E
:10ABA00081110DC02FEF3FEF4FE75FE7C501B40103
:10ABB0000E94127D18161CF465E775E00CC02FEF9B
:10ABC0003FEF4FE75FE4C701B6010E94717E1816A0
:10ABD00094F469E775E0C801DF91CF911F910F915F
:10ABE000FF90EF90DF90CF90BF90AF909F908F90AD
:10ABF0007F900C94C75E2FEF3FEF4FE75FECC701EC
:10AC0000B6010E94127D87FDE4CF20E030E0A9016B
:10AC1000C701B6010E94127D87FF0AC06DE2C8011C
:10AC20000E949C5EEC01F7FAF094F7F8F09402C0F1
:10AC3000C0E0D0E0B12C60E070E080E09FE37B14E6
:10AC400041F020E030E040E251E40E94177DB394EF
:10AC5000F6CFA70196010E94A67C6B017C010E94A1
:10AC6000907D4B015C012AE0AB01BC01C8010E9450
:10AC7000DC5EC80FD91F7720C1F1C501B4010E9465
:10AC8000BF7D9B01AC01C701B6010E94A57C6B0191
:10AC90007C016EE2C8010E949C5EC80FD91F20E0B3
:10ACA00030E040E251E4C701B6010E94767E4B01DC
:10ACB0005C010E94907D6B01E12CF12C2AE0B70130
:10ACC000A601C8010E94DC5EC80FD91FC701B601EA
:10ACD0000E94BF7D9B01AC01C501B4010E94A57C0F
:10ACE0006B017C017A947110DACFCE01DF91CF91A4
:10ACF0001F910F91FF90EF90DF90CF90BF90AF909A
:10AD00009F908F907F900895CF92DF92EF92FF9265
:10AD1000CF93DF93EC0160E074E00E946923892BFC
:10AD2000B1F0CE010E94AD226B017C0161E771E1BF
:10AD300086E398E00E94A35E60E074E0CE010E948A
:10AD4000F122B601CE010E941E4F81E001C080E0D9
:10AD5000DF91CF91FF90EF90DF90CF900895AF9269
:10AD6000BF92CF92DF92EF92FF920F931F93CF93F8
:10AD7000DF938C01EB0162E070E00E94C7227C014E
:10AD800097FF03C080E090E076C063E070E0C80108
:10AD90000E94C722AC011816190614F04FE350E0C8
:10ADA00081E0E816F10421F4CD2FDD0FDD0B04C0A6
:10ADB00082E0E816F1040CF4DD2724E630E0DE0141
:10ADC0000E949E7C9A01550F440B550B0E94467CB5
:10ADD00069017A015901C8010E94AB23C82FD0E054
:10ADE000C8010E94AD220D2C000CEE08FF086C1566
:10ADF0007D058E059F0549F4AB28E9F1C230D105E8
:10AE000061F0C530D105B9F508C0AB28E1F0C63016
:10AE1000D10539F0C130D10521F061E0C8010E94AF
:10AE20007F23B701A601C8010E947522C230D10557
:10AE300011F0259729F460E071E0C8010E94F34CFD
:10AE400060E072E00BC0C530D105A9F0229799F0FF
:10AE500062E0C8010E947F2360E071E0C801DF91D9
:10AE6000CF911F910F91FF90EF90DF90CF90BF9007
:10AE7000AF900C94F34CDF91CF911F910F91FF9005
:10AE8000EF90DF90CF90BF90AF900895CF93DF9376
:10AE9000EC0160E073E00E946923892B61F060E0BF
:10AEA00073E0CE010E94F34C60E073E0CE01DF91CD
:10AEB000CF910C94F122DF91CF91089520E3FC0112
:10AEC00020833296862F82958F7090E1899F60193A
:10AED00011246A3014F4605D01C0695C6293682FCC
:10AEE0008111F0CF08957F928F929F92AF92BF927F
:10AEF000CF92DF92EF92FF920F931F93CF93DF9346
:10AF0000CDB7DEB7A6970FB6F894DEBF0FBECDBFA4
:10AF10008C01762E942E852E20E2B22ECE01019643
:10AF20007C01FC012B2D11922A95E9F78DE693E027
:10AF30009AA389A38FEF8BA38CA38DA38EA3680103
:10AF40008BE4C80ED11C43E450E0BE016F5D7F4F1F
:10AF5000C6010E941C44019609F4B9C081E08983AE
:10AF60008A8386E0A82EAB821C82F80164817581F9
:10AF7000868197810E948F7C6D837E838F839887E3
:10AF800089869A8680E890E09C878B874CE150E028
:10AF9000B701C6010E94DD41F7012B2D11922A95C0
:10AFA000E9F7480188E0880E911CF401D70101906F
:10AFB0000D92AA94E1F740E150E0B701C6010E946A
:10AFC000DD41F7011192BA94E9F796E0A92EB12C70
:10AFD00040E250E0B701C6010E94DD41F1E0AF1A46
:10AFE000B108B1F783E6898392E89A8393E59B835E
:10AFF0008C8385E38D8381E08E837F829DE39887B8
:10B0000097E099878A8786E0F401DE011B9601901C
:10B010000D928A95E1F78CE0898B8A8B6DE775E05C
:10B02000CE0143960E94E580F8016385CE014996E2
:10B030000E945E57F8016485CE014B960E945E57D0
:10B04000F8016585CE014D960E945E574EE150E0B5
:10B05000B701C6010E94DD41F3E07F121EC082E30A
:10B06000898384E08A83F80196859B8397859C83F6
:10B0700090899D8391899E8396E39F838887868D9F
:10B080008987878D8A8780A18B8781A18C874CE0F7
:10B0900050E0B701C6010E94DD4187E3898386E065
:10B0A0008A8391E09B8393E09C838D838FE08E83E2
:10B0B0008AE38F838BE388878FEF898749E050E0AD
:10B0C000B701C6010E94DD41C6010E94F343A69666
:10B0D0000FB6F894DEBF0FBECDBFDF91CF911F91A9
:10B0E0000F91FF90EF90DF90CF90BF90AF909F9027
:10B0F0008F907F900895AF92BF92CF92DF92FF9290
:10B100000F931F93CF93DF93F82E8B015A016901A0
:10B1100064E270E00E946E45C82F65E270E08F2DFA
:10B120000E946E45D0E0DC2FCC27080F111DC00F08
:10B13000D11F6F2D6295660F607E6C5E9601A50132
:10B14000CE010E94CA42CC0DDD1D4D2F64E270E09D
:10B150008F2D0E9420434C2F65E270E08F2DDF91F0
:10B16000CF911F910F91FF90DF90CF90BF90AF9044
:10B170000C942043FF920F931F93CF93DF93F82EED
:10B1800000E010E08F2D0E948442EC01892B21F019
:10B190008F2D0E9484428C01C017D10799F7CE01F0
:10B1A000DF91CF911F910F91FF9008950F931F93FF
:10B1B000CF93DF93C82FD62F8A010E9429434D2FAA
:10B1C00060E070E08C2F0E9420430115110551F4BE
:10B1D00000917B0710917C070F5F1F4F10937C0736
:10B1E00000937B07412F64E070E08C2F0E94204386
:10B1F000402F65E070E08C2F0E94204361E070E0FA
:10B200008C2F0E94C73C81E0DF91CF911F910F915D
:10B210000895CF93DF93FC0101900020E9F79F018F
:10B22000281B390B285F3F4F2138310570F5EC01A1
:10B230000E941455882349F180916F0990917009FB
:10B24000019611F481E090E09093700980936F096A
:10B2500080916F09909170099093F4088093F5089C
:10B2600047E050E06FEE78E0CE010E948B54FC0185
:10B27000E751F74F1682AC01445051096FEE78E068
:10B2800082E8DF91CF910C94AB5480E0DF91CF91B5
:10B290000895CF92DF92EF92FF920F931F93CF9377
:10B2A000DF936C01EB017A0189018091E8088093BA
:10B2B000DB0880910502882319F00E945B2B06C0F1
:10B2C00069EB73E086E398E00E94D73C26E030E02B
:10B2D00045E757E064E089E090E00E94CA42C60179
:10B2E00002960E94C546C70102960E94D546C80133
:10B2F00002960E94CD468A819B81AC81BD8180935C
:10B30000DE089093DF08A093E008B093E108DF9196
:10B31000CF911F910F91FF90EF90DF90CF90089504
:10B320002F923F924F925F926F927F928F929F9255
:10B33000AF92BF92CF92DF92EF92FF920F931F9343
:10B34000CF93DF93CDB7DEB7E2970FB6F894DEBFA9
:10B350000FBECDBF7C012A013B0169010E9412652D
:10B360004B015C018701055B1F4FC8010E948C41A6
:10B3700018161906A4F00E941265DC01CB01881989
:10B380009909AA09BB09481659066A067B06F0F016
:10B3900062E370E080E090E00E94D864E6CF42E291
:10B3A00050E0BE016F5F7F4FC8010E941D4189813F
:10B3B000823031F4F801858996898334910541F012
:10B3C000D12CC8010E942B408D2D93C18FEF91C1CC
:10B3D0006D817E818F8198850E948F7C4B015C01FD
:10B3E000F601608371838283938346E050E0B70166
:10B3F000685F7F4FCE014D960E949480892B99F40F
:10B40000F70180819181A281B38188169906AA06ED
:10B41000BB0648F084819581A681B781881599057E
:10B42000AA05BB0528F4C8010E942B4080E061C139
:10B4300089899A89AB89BC89F70186879787A08B10
:10B44000B18B8EECC82ED12CC8010E943C41F1E09A
:10B45000CF1AD108C9F7D12CC7014E963C01F7018C
:10B46000E45AFF4FFAA7E9A740969CA78BA7F2974B
:10B47000FEA7EDA7089798AB8FA77097FAABE9AB3B
:10B480001701F2E22F0E311C270186E1480E511CF4
:10B49000F801818D928D181619060CF092CFC80113
:10B4A0000E943C418F30910509F49AC06CF58330BD
:10B4B000910509F45EC064F4009751F3019709F017
:10B4C0000CC1C8010E943C4144E050E0B201B5C04B
:10B4D0008630910509F469C00C9709F0FEC0C801D7
:10B4E0000E943C415C01BB24C50101960E94D571BC
:10B4F000F701958B848BA501BC01C8010E946B40AC
:10B50000F7018489958980C08633910509F481C04B
:10B510007CF48333910509F4C6C0C59709F0DDC0FA
:10B52000C8010E943C41C8010E943C41D82EB0CFC6
:10B530008B33910509F4A1C08F3F910509F4A8CF81
:10B54000CA9709F0CAC0C8010E943C4144E050E0DB
:10B550006DA57EA5C8010E941D41F70162A573A5D6
:10B5600084A595A50E948F7C62A773A784A795A741
:10B570008FCFC8010E943C415C0144E050E069A9C2
:10B580007AA9C8010E941D41812C912CBB24F4E0B2
:10B59000AF1AB1088A149B040CF07ACFC8010E943C
:10B5A0003C418FEF881A980AF5CFC8010E943C41B0
:10B5B0005C0144E050E0B101C8010E941D41812CB2
:10B5C000912CBB2494E0A91AB1088A149B040CF0B6
:10B5D0005FCFC8010E943C41EFEF8E1A9E0AF5CF63
:10B5E000C8010E943C415C01BB24C50101960E9438
:10B5F000D571F701938B828BA501BC01C8010E9414
:10B600006B40F70182899389FC01EA0DFB1D1082D2
:10B610003FCFC8010E943C41C82EF701868D8111A1
:10B6200010C0878D81110DC080A181110AC081A138
:10B63000811107C044E050E0B301C8010E941D41E0
:10B6400027CFE9A5FAA580809180A280B380B301BD
:10B65000CE0183960E94CC5F8DA19EA1AFA1B8A51B
:10B6600088169906AA06BB0629F3CC2009F410CF48
:10B67000C8010E943C41CA94F8CFC8010E943C41D5
:10B6800044E050E06BA57CA5C8010E941D41F70174
:10B6900066A577A580A991A90E948F7C66A777A748
:10B6A00080AB91ABF5CEC8010E943C4144E050E034
:10B6B0006FA578A9C8010E941D41F70166A177A175
:10B6C00080A591A50E948F7C66A377A380A791A7F0
:10B6D00062AB73AB84AB95ABDBCEC8010E943C413F
:10B6E000C82ECC2009F4D4CEC8010E943C41CA9493
:10B6F000F8CFE2960FB6F894DEBF0FBECDBFDF9154
:10B70000CF911F910F91FF90EF90DF90CF90BF905E
:10B71000AF909F908F907F906F905F904F903F90F1
:10B720002F9008952F923F924F925F926F927F9247
:10B730008F929F92AF92BF92CF92DF92EF92FF9241
:10B740000F931F93CF93DF93CDB7DEB729970FB633
:10B75000F894DEBF0FBECDBF8C010E9441732FEC69
:10B7600037E040E050E00E94467CDC01CB010196CE
:10B77000A11DB11DF80184839583A683B7838083BF
:10B780009183A283B3835801FBE4AF0EB11CC501C2
:10B790000E94364364E470E0C5010E940F42882392
:10B7A00009F42EC10E9412652B013C01812C912CC1
:10B7B000C801865B9F4F9E838D83180192E4290EFA
:10B7C000311C48EEC42E43E0D42EE12CF12CD801DC
:10B7D000DE96B987A887ED81FE818081833009F4E8
:10B7E000FEC0811120C0F80184819581A681B781B6
:10B7F0000196A11DB11D84839583A683B7830E9402
:10B8000012656419750986099709A70196010E94B6
:10B81000247CA90161E0C8010E94735781E0AD81D9
:10B82000BE818C93C3C08430E9F4F8018481958192
:10B83000A681B7810196A11DB11D84839583A6833E
:10B84000B7830E9412656419750986099709A701D3
:10B8500096010E94247CA90163E0C8010E947357ED
:10B86000E2E02AC0813061F5D1014D915D916D9189
:10B870007C919E012F5F3F4FC8010E9490598F839A
:10B88000823009F08DC089819A81AB81BC81F80139
:10B8900084839583A683B7830E9412656419750912
:10B8A00086099709A70196010E94247CA90163E0FB
:10B8B000C8010E947357EF81AD81BE81EC9376C0C1
:10B8C000823009F073C0D1014D915D916D917C91F1
:10B8D0009E012F5F3F4FC8010E9490598F83853092
:10B8E00009F057C083E0ED81FE818083F80186A1D5
:10B8F00097A1A0A5B1A5892B8A2B8B2B41F484E8B5
:10B9000093E0A0E0B0E086A397A3A0A7B1A7F801B9
:10B9100082A593A5A4A5B5A5892B8A2B8B2B61F4B1
:10B9200086A197A1A0A5B1A5B695A795979587954E
:10B9300082A793A7A4A7B5A7D8019E964D915D9124
:10B940006D917C91D1979A968D919D910D90BC911E
:10B95000A02D452B462B472B59F4AC01BD01440FBC
:10B96000551F661F771FF80146A757A760AB71AB3D
:10B97000F80182AB93ABA4ABB5AB86A597A5A0A904
:10B98000B1A986AB97ABA0AFB1AF88248394912CBB
:10B990000DC0FF81F63021F4AD81BE811C9206C03E
:10B9A000BF81BF3F19F4ED81FE811082F1E08F1657
:10B9B000910409F410CF0E941265DC01CB018419B7
:10B9C0009509A609B709E885F98520813181428169
:10B9D0005381281739074A075B0708F0FCCEC501D9
:10B9E0000E943643F80184819581A681B781019632
:10B9F000A11DB11D84839583A683B783C40102C0B2
:10BA000080E090E029960FB6F894DEBF0FBECDBF60
:10BA1000DF91CF911F910F91FF90EF90DF90CF902A
:10BA2000BF90AF909F908F907F906F905F904F905E
:10BA30003F902F900895CF92DF92EF92FF920F9355
:10BA40001F93CF93DF936C017A018B01C0E0D0E0AC
:10BA5000CE15DF0581F0D8016D918D01D601ED91F4
:10BA6000FC910190F081E02DC6011995892B11F010
:10BA70002196EECF7E01C701DF91CF911F910F91EB
:10BA8000FF90EF90DF90CF900895FC01538D448D8F
:10BA9000252F30E0842F90E0821B930B541710F079
:10BAA000CF96089501970895FC01918D828D981786
:10BAB00061F0828DDF01A80FB11D5D968C91928D92
:10BAC0009F5F9F73928F90E008958FEF9FEF08958F
:10BAD000FC01918D828D981731F0828DE80FF11D58
:10BAE000858D90E008958FEF9FEF0895FC01918D73
:10BAF000228D892F90E0805C9F4F821B91098F736C
:10BB00009927089589E997E00E94765D21E0892BC5
:10BB100009F420E0822F089586E398E00E94765D84
:10BB200021E0892B09F420E0822F0895FC01848D07
:10BB3000DF01A80FB11DA35ABF4F2C91848D90E057
:10BB400001968F739927848FA689B7892C93A08932
:10BB5000B1898C91837080648C93938D848D9813BC
:10BB600006C00288F389E02D80818F7D808308954F
:10BB7000EF92FF920F931F93CF93DF93EC0181E03D
:10BB8000888F9B8D8C8D981305C0E889F9898081F9
:10BB900085FD26C0F62E0B8D10E00F5F1F4F0F7333
:10BBA0001127E02E8C8DE8120CC00FB607FCFACFDF
:10BBB000E889F989808185FFF5CFCE010E94965DE5
:10BBC000F1CF8B8DFE01E80FF11DE35AFF4FF0829C
:10BBD0009FB7F8940B8FEA89FB89808180620AC045
:10BBE0009FB7F894EE89FF896083E889F98980819D
:10BBF0008370806480839FBF81E090E0DF91CF916C
:10BC00001F910F91FF90EF900895CF93DF93EC0178
:10BC1000888D8823C9F0EA89FB89808185FD05C06C
:10BC2000A889B9898C9186FD0FC00FB607FCF5CFA6
:10BC3000808185FFF2CFA889B9898C9185FFEDCFEE
:10BC4000CE010E94965DE7CFDF91CF91089580E00D
:10BC500090E0892B21F00E948C5D811121C080E051
:10BC600090E0892B41F080E090E0892B21F00E9448
:10BC70000000811118C080E090E0892B21F00E9423
:10BC8000825D811113C080E090E0892BA1F080E0FB
:10BC900090E0892B81F00E94000081110AC0089574
:10BCA0000E940000DCCF0E940000E5CF0E9400004F
:10BCB000EACF0C94000008950E946D80EF92FF92ED
:10BCC0000F931F93CF93DF93EC018B017A010E94B6
:10BCD0001265FE01E857FF4F60837183828393836F
:10BCE0008C819D81DC01ED91FC910280F381E02D3E
:10BCF000A701B801DF91CF911F910F91FF90EF90B5
:10BD000019941F93CF93DF93EC01162F0E941265B5
:10BD1000FE01E857FF4F60837183828393838C8198
:10BD20009D81DC01ED91FC910190F081E02D612F6E
:10BD3000DF91CF911F911994DC01ED91FC9101905D
:10BD4000F081E02D1994EF92FF920F931F93CF9300
:10BD5000DF938C017B01C0E0D0E0F701EC0FFD1F09
:10BD60006491662361F0D801ED91FC910190F0811E
:10BD7000E02DC8011995892B11F02196EECFCE0147
:10BD8000DF91CF911F910F91FF90EF900895611572
:10BD9000710579F0FB0101900020E9F73197AF01BF
:10BDA000461B570BDC01ED91FC910280F381E02DE5
:10BDB000199480E090E008958F929F92AF92BF9285
:10BDC000EF92FF920F931F93CF93DF93CDB7DEB720
:10BDD000A1970FB6F894DEBF0FBECDBF7C01FA016C
:10BDE000CB0119A2223008F42AE08E010F5D1F4F0B
:10BDF000822E912CA12CB12CBF01A50194010E948F
:10BE0000247CF901CA01015011096A3014F4605D03
:10BE100001C0695CD8016C93232B242B252B61F77F
:10BE2000B801C7010E94C75EA1960FB6F894DEBFA5
:10BE30000FBECDBFDF91CF911F910F91FF90EF907B
:10BE4000BF90AF909F908F900895CF92DF92EF9226
:10BE5000FF920F931F93CF93DF932115310581F448
:10BE6000DC01ED91FC910190F081E02D642FDF91D8
:10BE7000CF911F910F91FF90EF90DF90CF90199489
:10BE80002A30310501F577FF1DC06A017B01EC0105
:10BE90006DE20E949C5E8C0144275527BA014C1923
:10BEA0005D096E097F092AE0CE010E94DC5E800FE9
:10BEB000911FDF91CF911F910F91FF90EF90DF9035
:10BEC000CF9008952AE0DF91CF911F910F91FF90BD
:10BED000EF90DF90CF900C94DC5E9A01AB01770F6E
:10BEE000660B770B0C94255F9A01452B39F4DC0126
:10BEF000ED91FC910190F081E02D1994462F50E0D6
:10BF000060E070E00C94DC5E8F929F92AF92BF92E3
:10BF1000CF92DF92EF92FF920F931F93CF93DF9315
:10BF20007C018B014C0182E0880E911C5701E5E0F9
:10BF3000AE0EB11CC0E0D0E0F40161914F014AE0C7
:10BF400050E0C8010E94745F6C016EE2C8010E945B
:10BF50009C5E8C0D9D1DC80FD91F8A149B0461F730
:10BF60004AE050E0F7016581C8010E94745F8C0FC0
:10BF70009D1FDF91CF911F910F91FF90EF90DF9068
:10BF8000CF90BF90AF909F908F90089564E174E040
:10BF90000C94C75E0C94C75EDC018DE693E08D9334
:10BFA0009D9384E0FB0101900D928A95E1F708953D
:10BFB0001F920F920FB60F9211240BB60F922F9370
:10BFC0003F934F935F936F937F938F939F93AF9321
:10BFD000BF93EF93FF9389E997E00E94965DFF91ED
:10BFE000EF91BF91AF919F918F917F916F915F91F1
:10BFF0004F913F912F910F900BBE0F900FBE0F905E
:10C000001F9018951F920F920FB60F9211240BB626
:10C010000F922F938F939F93EF93FF93E091A90734
:10C02000F091AA078081E091AF07F091B00782FDFF
:10C0300012C090818091B2078F5F8F732091B307F8
:10C04000821751F0E091B207F0E0E756F84F958F74
:10C050008093B20701C08081FF91EF919F918F91F2
:10C060002F910F900BBE0F900FBE0F901F90189541
:10C070001F920F920FB60F9211240BB60F922F93AF
:10C080003F934F935F936F937F938F939F93AF9360
:10C09000BF93EF93FF9386E398E00E94965DFF9134
:10C0A000EF91BF91AF919F918F917F916F915F9130
:10C0B0004F913F912F910F900BBE0F900FBE0F909D
:10C0C0001F9018951F920F920FB60F9211240BB666
:10C0D0000F922F938F939F93EF93FF93E0914608D6
:10C0E000F09147088081E0914C08F0914D0882FD65
:10C0F00012C0908180914F088F5F8F7320915008FC
:10C10000821751F0E0914F08F0E0EA5CF74F958F0D
:10C1100080934F0801C08081FF91EF919F918F9193
:10C120002F910F900BBE0F900FBE0F901F90189580
:10C130001F920F920FB60F9211240BB60F922F93EE
:10C140003F934F935F938F939F93EF93FF93209130
:10C150008C0730918D0780918A0790918B07AC01F5
:10C160004F5F5F4F50938B0740938A07F901E80FA9
:10C17000F91F80818093CE00809107029091080280
:10C1800020918A0730918B078217930748F48FEF2D
:10C190009FEF90938B0780938A0788E48093C90070
:10C1A000FF91EF919F918F915F914F913F912F91CF
:10C1B0000F900BBE0F900FBE0F901F9018951F92FF
:10C1C0000F920FB60F9211242F933F938F939F934B
:10C1D000209188073091890780918A0790918B0779
:10C1E00021303105A9F48F3F2FEF920789F4109287
:10C1F000C8001092CD0089E08093CC0086E2809345
:10C20000CA001092CE0010928B0710928A0717C0B6
:10C21000892BA9F41092C8001092CD0083E080937E
:10C22000CC008EE08093CA0088E28093C90010920F
:10C23000CE0081E090E090938B0780938A079F91D6
:10C240008F913F912F910F900FBE0F901F901895D7
:10C250001F920F920FB60F9211240BB60F922F93CD
:10C260003F934F935F936F937F938F939F93AF937E
:10C27000BF93EF93FF939091C8008091CE0094FFFD
:10C2800008C081E08093870780918C0790918D078B
:10C2900057C090918707913099F481110EC082E0C8
:10C2A000809387070E9412656093810770938207CD
:10C2B00080938307909384073EC01092870744C001
:10C2C000923009F041C0E0918507F0918607908196
:10C2D000891721F091E090930602808320918507D1
:10C2E0003091860780917F07909180072817390742
:10C2F00011F510928707809106028823D1F0809172
:10C300007D0790917E07892BA1F01092C900E091E2
:10C310007D07F0917E07199580E98093C9001092FE
:10C32000C8001092CD0083E08093CC008EE0809313
:10C33000CA001092060280918507909186070196A7
:10C340009093860780938507FF91EF91BF91AF91FE
:10C350009F918F917F916F915F914F913F912F911D
:10C360000F900BBE0F900FBE0F901F901895CF929D
:10C37000DF92EF92FF920F931F93CF93DF936C01A5
:10C380008B0186E090E00E94D571EC0190938F07BD
:10C3900080938E07F60101900020E9F7CF018C19F8
:10C3A0009D090E94D5717C01B6010E94E580F601CD
:10C3B00001900020E9F73197EC19FD09EE0DFF1D02
:10C3C0001082F982E8821B830A8380918B05909109
:10C3D0008C059D838C83D0938C05C0938B05DF9156
:10C3E000CF911F910F91FF90EF90DF90CF90089524
:10C3F000CF92DF92EF92FF920F931F93CF93DF9331
:10C40000CDB7DEB7EC970FB6F894DEBF0FBECDBF49
:10C41000DC012C91222309F455C06BE275E00E94E7
:10C4200009759A8389837E01B3E0EB0EF11C01E06C
:10C4300010E0D02EC12E6BE275E080E090E00E940B
:10C440000975F701819391937F010E31110539F43C
:10C4500000918E0710918F07E980FA8008C00F5F66
:10C460001F4F892B31F7F4CFF80104811581011595
:10C470001105A1F0D8016D917C91C7010E94DC806B
:10C48000892B91F7D8011296ED91FC911397BE017B
:10C490006F5F7F4F8D2D9C2D19950AC063E871E168
:10C4A00086E398E00E94A35E86E398E00E94C65F60
:10C4B00086E398E00E94C65F6FE771E186E398E04B
:10C4C0000E94A35EEC960FB6F894DEBF0FBECDBF00
:10C4D000DF91CF911F910F91FF90EF90DF90CF9060
:10C4E0000895FB012481358142815381241735074A
:10C4F00058F440815181DA01A20FB31F8C938481DB
:10C50000958101969583848380E00895FC0140E045
:10C5100050E020E030E08AE09191992301F124304D
:10C5200031055CF59E3271F44F3F510509F02CF551
:10C53000DB01A20FB31F12964C932F5F3F4F40E0D9
:10C5400050E0EACF849FD001859FB00D1124492F80
:10C55000990F550B405351094A0F5B1FDDCF4F3FD9
:10C56000510509F054F4243031053CF4FB01E20F8D
:10C57000F31F428381E090E0089580E090E0089509
:10C580003FB7F8948091940790919507A0919607F2
:10C59000B091970726B5A89B05C02F3F19F00196CB
:10C5A000A11DB11D3FBFBA2FA92F982F8827820F39
:10C5B000911DA11DB11DBC01CD0142E0660F771F89
:10C5C000881F991F4A95D1F70895CF92DF92EF9275
:10C5D000FF92CF93DF93CDB7DEB768970FB6F8948D
:10C5E000DEBF0FBECDBFFA012DE633E03A832983CB
:10C5F0005FEF5B835C835D831E8238872F83C280FD
:10C60000D380E480F580C986DA86EB86FC863E8797
:10C610002D87FB0142815381648175814F87588B3F
:10C62000698B7A8B3C8B2B8BFC0182819381A4815B
:10C63000B5818D8B9E8BAF8BB88F9E012F5F3F4F47
:10C64000AE01495F5F4FBE01635F7F4FCE014396EE
:10C650000E94495968960FB6F894DEBF0FBECDBF51
:10C66000DF91CF91FF90EF90DF90CF9008950F93DF
:10C670001F93CF93DF93CDB7DEB768970FB6F894CB
:10C68000DEBF0FBECDBFFB01DC0112964D915D9167
:10C690006D917C9115974D8B5E8B6F8B788F8DE6AE
:10C6A00093E09A83898321E0288F0D891E892F8941
:10C6B000388D0B831C832D833E8398878F83028163
:10C6C00013812481358109871A872B873C879E87B0
:10C6D0008D874F87588B698B7A8BAE014F5F5F4F89
:10C6E000BE01695F7F4FCE010D960E94E56268969C
:10C6F0000FB6F894DEBF0FBECDBFDF91CF911F9173
:10C700000F910895CF93DF93CDB7DEB762970FB641
:10C71000F894DEBF0FBECDBFFC0182819381A4815E
:10C72000B5818F87988BA98BBA8B2DE633E03A833E
:10C73000298341E04A8B4F85588969897A894B83DF
:10C740005C836D837E8338872F8389879A87AB8745
:10C75000BC87BE016F5F7F4FCE0107960E94376393
:10C7600062960FB6F894DEBF0FBECDBFDF91CF91BA
:10C770000895CF92DF92EF92FF920F931F93CF9382
:10C78000DF936C01EB017B0182E0E80EF11C00E01D
:10C7900010E0C601800F911F0E94FE7BF70181937C
:10C7A0007F010F5F1F4F0430110599F78A8188239D
:10C7B00061F08F3F61F48B818F3F49F48C818F3F13
:10C7C00031F481E09D819F3F19F480E001C081E058
:10C7D00090E0DF91CF911F910F91FF90EF90DF904C
:10C7E000CF900895EF92FF920F931F93CF93DF9313
:10C7F0007C018B010E5F1F4FC0E0D0E0F80161911A
:10C800008F01C7018C0F9D1F0E94067C2196C430AA
:10C81000D105A1F7DF91CF911F910F91FF90EF907C
:10C820000895FC0121912111FDCF0C94866290E0C6
:10C83000FC013197E231F10508F04EC08827EE5F28
:10C84000FE4F8F4F0C94877C809180008F7703C0C0
:10C85000809180008F7D809380000895809180007A
:10C86000877FF9CF84B58F7702C084B58F7D84BD73
:10C8700008958091B0008F7703C08091B0008F7DC4
:10C880008093B0000895809190008F7707C08091C9
:10C8900090008F7D03C080919000877F80939000EF
:10C8A00008958091A0008F7707C08091A0008F7DB0
:10C8B00003C08091A000877F8093A000089580919D
:10C8C00020018F7707C0809120018F7D03C0809168
:10C8D0002001877F8093200108951F93CF93DF93DA
:10C8E000282F30E0F901ED5AFD4E8491F901E35F04
:10C8F000FD4ED491F901E953FE4EC491CC23C1F011
:10C90000162F81110E941764EC2FF0E0EE0FFF1F2D
:10C91000E355FE4EA591B4919FB7F894111104C050
:10C920008C91D095D82302C0EC91DE2BDC939FBF75
:10C93000DF91CF911F910895CF93DF9390E0FC0199
:10C94000E35FFD4E2491FC01E953FE4E8491882360
:10C9500061F190E0880F991FFC01ED56FE4EC591E4
:10C96000D491FC01E355FE4EA591B491611109C02B
:10C970009FB7F8948881209582238883EC912E2399
:10C980000BC0623061F49FB7F8948881322F3095E4
:10C9900083238883EC912E2B2C939FBF06C08FB7E7
:10C9A000F894E8812E2B28838FBFDF91CF910895D3
:10C9B0008F929F92AF92BF92CF92DF92EF92FF92AF
:10C9C0006B017C010E94C0624B015C01C114D10467
:10C9D000E104F104F1F00E94C062DC01CB0188198E
:10C9E0009909AA09BB09883E9340A105B10570F3D6
:10C9F00021E0C21AD108E108F10888EE880E83E030
:10CA0000981EA11CB11CC114D104E104F10419F752
:10CA1000DDCFFF90EF90DF90CF90BF90AF909F90D1
:10CA20008F9008952FB7F8946091900770919107B7
:10CA300080919207909193072FBF08954F925F9234
:10CA40006F927F928F929F92AF92BF92CF92DF921E
:10CA5000EF92FF920F931F93CF93DF93CDB7DEB783
:10CA600063970FB6F894DEBF0FBECDBF7C015B01AC
:10CA70002A01FB0181918111FDCFB201C5010E9404
:10CA80008662892B09F04DC1F7014281538164818F
:10CA900075818091D5089091D608A091D708B09162
:10CAA000D808481759076A077B0709F43DC10E9457
:10CAB00012658701085F1F4F6F7077277C5FC80181
:10CAC0000E940F42813009F017C18DE693E09A83EE
:10CAD0008983F70182819381A481B5818B839C83B3
:10CAE000AD83BE8345E350E0BE016F5F7F4FC80159
:10CAF0000E941C44892B19F4C12CD12CF9C00E942E
:10CB00001265F7017783668342E050E0B7016A5F00
:10CB10007F4FC8010E94DD4181E090E09A838983C4
:10CB200042E050E0BE016F5F7F4FC8010E94DD41CF
:10CB300080E091E09A83898342E050E0BE016F5F1C
:10CB40007F4FC8010E94DD411A82198242E050E005
:10CB5000BE016F5F7F4FC8010E94DD4142E050E09F
:10CB6000BE016F5F7F4FC8010E94DD4142E050E08F
:10CB7000BE016F5F7F4FC8010E94DD414501F50195
:10CB80008081882301F164015601F60181913F0102
:10CB9000882321F08E3211F06301F6CFC818D9082E
:10CBA0001C141D0474F4CD8641E050E0BE01635FA7
:10CBB0007F4FC8010E94DD41A601B401C8010E9457
:10CBC000DD414301DCCF1D8641E050E0BE01635FE3
:10CBD0007F4FC8010E94DD41C12CDD24D394DA824D
:10CBE000C98242E050E0BE016F5F7F4FC8010E94E2
:10CBF000DD41DA82C98242E050E0BE016F5F7F4FC3
:10CC0000C8010E94DD41C8010E94F343892B09F449
:10CC100073CFE3E0AE2EB12C22E0420E511C0E94F5
:10CC200012653B014C01C8010E948C41181619067F
:10CC3000B4F00E941265DC01CB0186199709A8099E
:10CC4000B90989389341A105B105E0F462E370E0C8
:10CC500080E090E00E94D8640E94F22FE4CFF701B8
:10CC60004281538164817581818D928DA38DB48DB4
:10CC7000481759076A077B0749F4858D968DC59734
:10CC800029F409C0CC24CA94DC2C29C09EEFC92EFB
:10CC9000DD24DA9424C0F70181A192A10C970CF451
:10CCA0001FC14CE050E0BE016F5F7F4FC8010E9482
:10CCB0001D418B819C819827892798279A8B898B86
:10CCC000F7014681578129813A814217530779F14B
:10CCD000C8010E942B407CEFC72EDD24DA9481E04E
:10CCE000A81AB10829F0FFEFCF16DF0609F497CF95
:10CCF000C8010E94364302C0C12CD12C64E875E003
:10CD000086E398E00E94CA5F4AE050E0B60186E3FD
:10CD100098E00E946D5F86E398E00E94C65FC601BE
:10CD2000E4C081E090E0E1C08EEF9FEFDEC097FFAE
:10CD3000CFCF8F709270892B41F0C8010E942B4099
:10CD40006BEFC62EDD24DA94CACF6F807884762408
:10CD5000672476246114710419F0C12CD12C25C0EC
:10CD6000C8010E942B405AEFC52EDD24DA94B7CFBC
:10CD700041E050E0BE01635F7F4FC8010E941D414A
:10CD80008D8581111BC08D858111F2CFC8010E9454
:10CD90003C41C8010E943C41C8010E943C41C8017D
:10CDA0000E943C41FFEFCF1ADF0A8D819E819827B8
:10CDB00089279827C816D906D8F20AC08D859FEF13
:10CDC000980F9D878823F9F2C8010E943C41F6CF55
:10CDD000812C912C41E050E0BE016D5E7F4FC80177
:10CDE0000E941D418B89982F907C61F4882389F0E3
:10CDF0008B899FEF980F9B8B882341F0C8010E947D
:10CE00003C41F6CFC8010E943C411B8A8B898111AD
:10CE1000E1CF42E050E0BE01615F7F4FC8010E9458
:10CE20001D4142E050E0BE01635F7F4FC8010E9498
:10CE30001D41C8010E943C41C8010E943C41C801FB
:10CE40000E943C41C8010E943C4142E050E0BE01CA
:10CE50006F5E7F4FC8010E941D418F8598898115A3
:10CE6000914049F4CD84DE84DC24CD24DC2481E0AF
:10CE7000C816D10419F0C12CD12C14C089899A8903
:10CE80008115944041F0C8010E942B4047EFC42E09
:10CE9000DD24DA9424CF44E050E0B201C8010E94BE
:10CEA0001D411DCF89899A89982789279827C816F7
:10CEB000D90638F4C8010E943C41FFEFCF1ADF0ABF
:10CEC000F1CF2FEF821A920A6814790409F082CF09
:10CED000C8010E942B4036EFC32EDD24DA94FFCE2A
:10CEE0008DEFC82EDD24DA94FACE63960FB6F8944F
:10CEF000DEBF0FBECDBFDF91CF911F910F91FF908D
:10CF0000EF90DF90CF90BF90AF909F908F907F90E9
:10CF10006F905F904F900895FC01868197810097F4
:10CF200039F0662329F06150FC0182819381F7CFAB
:10CF300008951F920F920FB60F9211242F933F93D3
:10CF40008F939F93AF93BF93809190079091910798
:10CF5000A0919207B09193073091240B23E0230F07
:10CF60002D3720F40196A11DB11D05C026E8230F21
:10CF70000296A11DB11D2093240B809390079093DE
:10CF80009107A0939207B093930780919407909193
:10CF90009507A0919607B09197070196A11DB11D25
:10CFA0008093940790939507A0939607B093970763
:10CFB000BF91AF919F918F913F912F910F900FBE95
:10CFC0000F901F901895CF93DF93CDB7DEB7C6565D
:10CFD000D1090FB6F894DEBF0FBECDBF789484B5EB
:10CFE000826084BD84B5816084BD85B5826085BD65
:10CFF00085B5816085BD80916E00816080936E00F3
:10D0000010928100809181008260809381008091E4
:10D010008100816080938100809180008160809395
:10D0200080008091B10084608093B1008091B00055
:10D0300081608093B0008091910082608093910024
:10D040008091910081608093910080919000816037
:10D05000809390008091A10082608093A1008091D4
:10D06000A10081608093A1008091A00081608093E5
:10D07000A000809121018260809321018091210193
:10D080008160809321018091200181608093200143
:10D0900080917A00846080937A0080917A00826027
:10D0A00080937A0080917A00816080937A008091E9
:10D0B0007A00806880937A001092C1001092D005A7
:10D0C00010928C0510928B0526E040E052EC61E056
:10D0D00070E086E398E00E94FA5367EF78E086E319
:10D0E00098E00E94A35E6AE575E380EE93E00E94FB
:10D0F000B7616CE974E385EE93E00E94B7616DED72
:10D1000078E38AEE93E00E94B76165E473E38FEE03
:10D1100093E00E94B7616DE673E383EF93E00E94B2
:10D12000B76166E475E387EF93E00E94B7616AED4B
:10D1300074E38CEF93E00E94B76168EE73E380E0E4
:10D1400094E00E94B7616BEC73E383E094E00E948B
:10D15000B76168E573E387E094E00E94B7616FE42C
:10D1600073E38DE094E00E94B7610E94003055E7C0
:10D17000E52E57E0F52E6701B12C00E010E0C80164
:10D180000E94FE7BD6018D936D0181508E3F10F47D
:10D19000BB24B3940F5F1F4F0630110581F7BB20EE
:10D1A000B1F10E94414C0E947A3861E08DE00E940A
:10D1B0009C6426E040E855E260E070E089E997E091
:10D1C0000E94FA5387EE9FE290939F0A80939E0AF3
:10D1D00080E09CE29093A10A8093A00A8CEF9BE2EE
:10D1E0009093A30A8093A20A64E170E080E090E04B
:10D1F0000E94D8648CE99AE490937B0980937A0921
:10D2000064EF71E080E090E00E94D8645BC06BEF57
:10D2100078E086E398E00E94A35E4BE7C42E47E0E7
:10D22000D42E0EEC13E040E150E060E070E0C80165
:10D230000E949873F70161937F016AE370E0C8016F
:10D240000E94D180009709F4ACCFDC012C912223FD
:10D2500009F4A7CF8C010F5F1F4FCE14DF0419F71D
:10D26000A0CF86E398E00E94545D182F8A3061F5C4
:10D27000E091D005F0E0EC56FA4F108264E174E0E2
:10D2800086E398E00E94CA5F84E995E00E94F86115
:10D290001092D00586E398E00E94765D892B09F70D
:10D2A0000E94BA12029714F00E94DF3D0E9483256B
:10D2B0008091730790917407892B49F50E94042C83
:10D2C0000E94275EA895E6CF8D3091F2883069F4F0
:10D2D00068E086E398E00E949C5E8091D0058823F8
:10D2E000C9F281508093D005D5CF682F86E398E0AE
:10D2F0000E949C5EE091D005EB3360F681E08E0FDA
:10D300008093D005F0E0EC56FA4F1083C3CF8091A4
:10D31000920590919305049709F483C00E941265C9
:10D320000091D1051091D2052091D3053091D405FB
:10D33000061717072807390708F073C020E02224D2
:10D340002394312CE0919005F0919105309709F4E8
:10D3500068C0211166C08085853009F04BC027ED7B
:10D3600032E063963FAF2EAF63976596FFAFEEAFA7
:10D3700065976C961FAE1EAE6C97CE018F5A9F4F6D
:10D380000E94B8230E9412652B013C016C968EAD61
:10D390009FAD6C97009709F441C1DC01ED91FC91C0
:10D3A0000484F585E02D1995892B09F437C16C9615
:10D3B0008EAD9FAD6C97DC01ED91FC910480F58101
:10D3C000E02D199584E690E0092E000CAA0BBB0B0A
:10D3D000480E591E6A1E7B1E4092D1055092D205FE
:10D3E0006092D3057092D405CE018F5A9F4F0E9450
:10D3F0002F5121E0E0919005F09191058281938178
:10D400009093910580939005892B09F09BCFE09133
:10D410007307F091740786819781909391058093AB
:10D4200090050E9412650091D5051091D6052091B6
:10D43000D7053091D805601771078207930708F464
:10D440003DCFE0917307F0917407309709F436CF20
:10D450002680378010E02114310479F1D10118962B
:10D460008C91853031F560E0C1010E948C67FC0130
:10D4700081859285A385B4850597A105B105C9F479
:10D48000C1010E945F5490E005979CF064E0C101E7
:10D490000E948C67A3969FAF8EAFA397892B49F00C
:10D4A000A3968EAD9FADA3970E945F54823008F083
:10D4B000EDC4F10122803380CECF0E941265DC01E1
:10D4C000CB01805D9A48AF4FBF4F8093D5059093B5
:10D4D000D605A093D705B093D8050E94104A4B01FA
:10D4E0005C010E9412656B017C010E941455882327
:10D4F00009F462C020E030E041E050E060E4CE0199
:10D5000001960E947F4940E450E063EC79E0CE014F
:10D5100001960E94DC746CEC73E0CE0101960E94CF
:10D52000C68040E450E06AEB79E0CE0101960E94AB
:10D53000DC74B501A401CE018F5B9F4F0E9424498A
:10D54000BE016F5B7F4FCE0101960E949D5520E08A
:10D5500030E041E050E060E4CE0101960E947F4956
:10D5600040E450E063EC79E0CE0101960E94DC7467
:10D570006CEC73E0CE0101960E94C68040E450E05E
:10D5800063EB79E0CE0101960E94DC74C701B6011D
:10D5900028EE33E040E050E00E94247CBA01A9016B
:10D5A000CE018F5B9F4F0E942449BE016F5B7F4F6E
:10D5B000CE0101960E949D551123C1F00E94104A90
:10D5C0006B017C016EEC79E086E398E00E94A35E3B
:10D5D0002AE0B701A60186E398E00E94DC5E6BE2D8
:10D5E00075E086E398E00E94CA5F68CE0E94104A08
:10D5F0006B017C016CEC79E086E398E00E94A35E0D
:10D600002AE0B701A60186E398E00E94DC5E6AEC9E
:10D6100079E086E398E00E94A35E50CE6A968FADD3
:10D620006A97843009F0D6C080918E0590918F055D
:10D63000892B09F0C7C0CE018F5A9F4F0E94845694
:10D640008111C0C06796AEACBFAC6797F50180850D
:10D65000853009F07AC3C5010E945F54C82ED12CD1
:10D66000F2E0CF16D1040CF470C330928F052092F3
:10D670008E0560E070E0CE018F5A9F4F0E94C72256
:10D680004C0161E070E0CE018F5A9F4F0E94C7228B
:10D690007C01B5E0CB16D1040CF4C7C364E0C5012E
:10D6A0000E948C67DC0119960D911C911A9726E255
:10D6B00040E855E260E070E089E997E00E94FA53A3
:10D6C00080928C0989E997E090938B0980938A096D
:10D6D0001092970A1092990A1092980A0130110537
:10D6E00009F453C30CF438C30230110509F040C3E8
:10D6F000F0928E09E0928D093092900920928F0964
:10D7000083E00E944351A1968FAFA197A196BFAD30
:10D71000A197B1116BC3C0909109D0909209C60135
:10D720000D2C000CAA0BBB0B89839A83AB83BC83A3
:10D73000E0E1F0E0FE83ED836596EEADFFAD659729
:10D74000A080B18063E879E086E398E00E94A35E60
:10D75000B50186E398E00E94CA5F6CE779E086E352
:10D7600098E00E94A35EBE016F5F7F4F86E398E062
:10D770000E9412240E94C65FB601CE018F5A9F4FAD
:10D780000E94AF56A0909005B0909105D5011296D9
:10D790008D919C911397E7EDF2E0FA83E9839C83E6
:10D7A0008B831B861A86CE0101960E94B823AB2874
:10D7B00009F0FCC2CE0101960E942F5110928F05F4
:10D7C00010928E05CE018F5A9F4F0E94465780EDD2
:10D7D00097E0FACD893009F0B2C280918E05909120
:10D7E0008F05892B79F7CE018F5A9F4F0E9484565F
:10D7F0008111E8CF30928F0520928E050E946F2A0A
:10D800005C01892B21F086E0D50118968C9320E0ED
:10D8100030E043E050E060E2CE0101960E947F4993
:10D820006596EEADFFAD6597608171814FE150E087
:10D83000CE0101960E94EC8067E174E0CE01019672
:10D840000E94C68026E040E855E260E070E089E989
:10D8500097E00E94FA5360E070E0CE018F5A9F4F2C
:10D860000E94C72280938C0989E997E090938B09E5
:10D8700080938A091092970A1092990A1092980A36
:10D88000E4E3F8E0F0938E09E0938D092AE030E0BC
:10D890003093900920938F0983E00E9443518111B6
:10D8A000CBC06CE579E086E398E00E94A35E01E9D5
:10D8B00019E095EAE92E99E0F92ED8018D919D9114
:10D8C0008D01092E000CAA0BBB0B25968CAF9DAFCA
:10D8D000AEAFBFAF2597E0E1F0E02796FFAFEEAF28
:10D8E0002797BE016F5B7F4F86E398E00E9412246A
:10D8F0006AE579E00E94A35EE016F106F1F686E3A0
:10D9000098E00E94C65F6091950970919609072E74
:10D91000000C880B990B0E94C17D20E030E048ECA0
:10D9200052E40E94177D9B01AC016DE174E0C501DA
:10D930000E94293C0091990910919A09A8016FE170
:10D9400074E0C5010E94F55060919B0970919C099B
:10D95000072E000C880B990B0E94C17D20E030E05F
:10D9600048EC52E40E94177D9B01AC0163E274E035
:10D97000C5010E94293C60919D0970919E09072E66
:10D98000000C880B990B0E94C17D20E030E040E242
:10D9900051E40E94177D9B01AC0161E274E0C50176
:10D9A0000E94293C409191095091920965E274E0EE
:10D9B000C5010E94F550012B09F45CC067968EAD3D
:10D9C0009FAD6797DC0118962C91253009F052C065
:10D9D00061E00E948C67009709F44CC0E4E6F0E037
:10D9E0006E96FFAFEEAF6E97DC0119966D917C914C
:10D9F0001A97CE018F5B9F4F0E946D54CE018F5BB3
:10DA00009F4F0E946822882389F0C12CD12CE12CE1
:10DA1000F12C01E09E01245A3F4F41E050E060E0CC
:10DA200070E0CE018F5B9F4F0E948109CE018F5B1A
:10DA30009F4F0E942F511EC090E0A0E0B0E02596BD
:10DA40008CAF9DAFAEAFBFAF2597E0E1F0E027967A
:10DA5000FFAFEEAF279764E479E086E398E00E9499
:10DA6000A35EBE016F5B7F4F86E398E00E941224A5
:10DA70000E94C65F8091910983FF39C08EE398E0D0
:10DA800090938E0980938D093092900920928F098E
:10DA900083E00E944351811109C040919109509146
:10DAA000920968E274E0C5010E94F55010928F055A
:10DAB00010928E05CE018F5A9F4F0E94D94F181693
:10DAC000190684F4C12CD12CE12CF12C01E020E0CA
:10DAD00030E040E050E062E070E0CE018F5A9F4FAE
:10DAE0000E94810930928F0520928E0507C040E088
:10DAF00050E068E274E0C5010E94F55062E370E016
:10DB000080E090E00E94D86423E130E030938E09F9
:10DB100020938D0944E050E05093900940938F0981
:10DB200083E00E9443518111ABC06AE379E086E350
:10DB300098E00E94A35E01E919E089E9E82E89E0F6
:10DB4000F82ED8016D917D918D014AE050E086E379
:10DB500098E00E946D5F68E379E086E398E00E94B8
:10DB6000A35EE016F10669F786E398E00E94C65FBF
:10DB7000009191091091920901151105D1F0B80198
:10DB8000012E000C880B990B0E94C17D2DEE3EE901
:10DB90004CE35EE30E94767E22E538EB42E152E4FC
:10DBA0000E94A57C9B01AC016CE274E0C5010E945F
:10DBB000293C6091930970919409072E000C880B01
:10DBC000990B0E94C17D2DEE3EE94CE35EE30E947D
:10DBD000767E22E538EB42E152E40E94A57C6B019F
:10DBE0007C019B01AC016BE174E0C5010E94293C02
:10DBF000609197097091980916161706A4F4072EDC
:10DC0000000C880B990B0E94C17D20E030E040E2BF
:10DC100051E40E94177D9B01AC0160E374E0C501F3
:10DC20000E94293C07C040E050E060E374E0C50179
:10DC30000E94F55020E030E040E252E4C701B60116
:10DC40000E94717E1816C4F5012BB1F10E94145583
:10DC5000882329F080918D05882309F406C1C12C01
:10DC6000D12CE12CF12C01E020E030E040E050E04C
:10DC700062E070E0CE018F5A9F4F0E9481091CC064
:10DC800090E0A0E0B0E025968CAF9DAFAEAFBFAF07
:10DC90002597E0E1F0E02796FFAFEEAF279762E22D
:10DCA00079E086E398E00E94A35EBE016F5B7F4F40
:10DCB00086E398E00E94122480E091E00E94D571F2
:10DCC0008C01892B61F125961FAE1EAE25972796F4
:10DCD0001FAE1EAE27978FEF9FEF29969FAF8EAF97
:10DCE00029978EE392E023969FAF8EAF23972B96D2
:10DCF0001FAE1EAE2B972D961FAF0EAF2D9780E057
:10DD000091E061969FAF8EAF61972F961FAE1EAECA
:10DD10002F97B501CE018F5B9F4F0E9478280E94FC
:10DD20001455882329F080918D05882309F4A8C013
:10DD3000C8010E946D72C5010E94713C3FCDCE01A9
:10DD40008F5A9F4F0E9446573DCB60EA79E086E3A9
:10DD500098E00E94A35E36CD012B09F5F0928E0962
:10DD6000E0928D093092900920928F0981E0C9CC10
:10DD700003301105A1F4F0928E09E0928D093092E2
:10DD8000900920928F0984E0BCCCF0928E09E09239
:10DD90008D091093900900938F0982E0B2CC68E856
:10DDA00079E086E398E00E94A35EB0CCCE010196B4
:10DDB0000E946822882309F4FDCC8985843009F00B
:10DDC000F9CC60E070E0CE0101960E94C72288166F
:10DDD000990609F0EFCC61E070E0CE0101960E9457
:10DDE000C722E816F90609F0E5CC22C0A196FFADDE
:10DDF000A1978F2F90E0A0E0B0E089839A83AB8356
:10DE0000BC8320E130E03E832D8366E679E086E343
:10DE100098E00E94A35EBE016F5F7F4F86E398E0AB
:10DE20000E9412240E94C65FC9CC02E010E03FCCE1
:10DE3000B601CE0101960E94AF56E0919005F09197
:10DE40009105828193819093910580939005892B10
:10DE500009F0B0CCE0917307F09174078681978147
:10DE60009093910580939005A5CC6596EEADFFAD9E
:10DE700065976081718180E494E00E94663CEFCEFA
:10DE8000B801CE0101960E94663C52CF61E0C1010B
:10DE90000E948C67FC011185728462E0C1010E94BE
:10DEA0008C67DC0119968D909D90AD90BC901C976D
:10DEB00063E0C1010E948C67DC0119962D913D91B0
:10DEC0004D915C911C97A7962CAF3DAF4EAF5FAFC5
:10DED000A79760E0A3968EAD9FADA3970E948C6735
:10DEE000FC01C184D284E384F48461E0A3968EAD06
:10DEF0009FADA3970E948C67DC0119964D915D91AF
:10DF00006D917C911C97411551056105710571F466
:10DF1000D1016D917C9186E398E00E94CA5F63E035
:10DF20007AE086E398E00E94A35E14C04150510954
:10DF300061097109FC014187528763877487452B0A
:10DF4000462B472B39F4D1016D917C9184E394E009
:10DF50000E94663C20E030E048E152E4C701B6018F
:10DF60000E94717E18163CF4F1016081718180E499
:10DF700094E00E94663C6F961FAF6F97A0967FAEAD
:10DF8000A097C501B4010E94C17D2B013C01A5965B
:10DF90008EAC9FACA597D101AD90BC9086E398E084
:10DFA0000E94C65FB50186E398E00E94CA5F6DEFEC
:10DFB00079E086E398E00E94A35E22E0B301A2012B
:10DFC00086E398E00E94A85567EF79E086E398E041
:10DFD0000E94A35E22E0B701A60186E398E00E94BA
:10DFE000A85561EF79E086E398E00E94A35E4AE0DD
:10DFF00050E0A5966EAD7FADA59786E398E00E94B0
:10E000006D5FA096EEADFFADA09761E0812FF7FDAB
:10E0100081950E949C6461E0A3968EAD9FADA3970D
:10E020000E948C67FC0181859285A385B485892B2C
:10E030008A2B8B2B89F0F6E08F169104F9F024F4EB
:10E040008A94892849F41AC04AE084169104B1F0F0
:10E050005CE08516910491F0A096EEADFFADA0971F
:10E06000F7FF05C060E0812F81950E946D6460E03C
:10E07000812F0E946D646CEE79E021C020E030E0D9
:10E0800040E85FE3C301B2010E94A57C9B01AC01A3
:10E09000C701B6010E94127D87FF17C0A0968EAD02
:10E0A0009FADA09797FF05C060E0812F81950E94EA
:10E0B0006D6461E0812F0E946D6468EE79E086E313
:10E0C00098E00E94A35E11E0F4C9A7019601C30184
:10E0D000B2010E94127D181694F0A096AEADBFADAD
:10E0E000A097B7FF05C061E0812F81950E946D6404
:10E0F00060E0812F0E946D6463EE79E0E0CF64ED13
:10E1000079E0DDCFCF92DF92EF92FF92CF93DF9352
:10E11000E9E9F7E01382128288EEC82E83E0D82E58
:10E12000E12CF12CC482D582E682F7828FED92E059
:10E130009183808325ED30E03587248724ED30E01E
:10E140003787268720ED30E0318B208B21ED30E0C2
:10E15000338B228B22ED30E0358B248B26ED30E0A3
:10E16000378B268B118E128E138E148EE6E3F8E019
:10E1700013821282C482D582E682F78291838083E1
:10E1800085EC90E09587848784EC90E0978786877C
:10E1900080EC90E0918B808B81EC90E0938B828B74
:10E1A00082EC90E0958B848B86EC90E0978B868B4D
:10E1B000118E128E138E148EE1EBFAE0CDE6D3E0D1
:10E1C000D183C0831282138214821582E7EBFAE0B6
:10E1D000D183C0831282138214821582EDEBFAE0A0
:10E1E000D183C0831282138214821582E3EDF8E09A
:10E1F000D183C0831282138214821582E3ECFAE089
:10E20000D183C0831282138214821582E9EDF8E073
:10E2100080E5808381E08183E9ECFAE0D183C083EB
:10E220001282138214821582EFECFAE0D183C0834C
:10E230001282138214821582E5EDFAE0D183C08345
:10E240001282138214821582ECEDF8E0D183C08330
:10E250001282138214821582138612868AE08487C2
:10E2600061E08091DB080E949C64EBEDFAE0138290
:10E270001282C482D582E682F78281EF92E0918396
:10E280008083E7EEFAE0D183C08312821382148286
:10E290001582EDEEFAE0D183C083128213821482DC
:10E2A0001582E4EAFAE013821282C482D582E68201
:10E2B000F7828BE493E09183808388E084871092D7
:10E2C0009F0A10929E0A1092A10A1092A00A109220
:10E2D000A30A1092A20AA9EEB8E013961C921E920D
:10E2E000129783E093E011969C938E93D0937D09CF
:10E2F000C0937C0910927E0910927F0910928009C8
:10E30000109281098FEF9FEF90938909809388097C
:10E310001596FC93EE931497109287091092860934
:10E32000E3EFFAE0D183C083128213821482158254
:10E33000E9EFFAE0D183C08312821382148215823E
:10E34000EFEFFAE0D183C083128213821482158228
:10E35000E5E0FBE0D183C083128213821482158230
:10E36000EBE0FBE0D183C08312821382148215821A
:10E37000E1E1FBE0D183C083128213821482158213
:10E38000E7E1FBE0808312821182148613868FEF0F
:10E390009FEFDC0187839087A187B287DF91CF91C0
:10E3A000FF90EF90DF90CF9008950F931F93CF933E
:10E3B000DF938230910510F482E090E0E091290B28
:10E3C000F0912A0B20E030E0A0E0B0E0309719F1A6
:10E3D000408151810281138148175907C8F0841781
:10E3E000950769F4109731F012960C9312971396D3
:10E3F0001C9327C00093290B10932A0B22C02115D0
:10E40000310519F04217530718F49A01BD01EF01C5
:10E41000DF01F801DBCF21153105F9F0281B390B9D
:10E420002430310580F48A819B816115710521F0CA
:10E43000FB019383828304C090932A0B8093290B62
:10E44000FE01329644C0FE01E20FF31F81939193C7
:10E4500022503109398328833AC02091270B30910B
:10E46000280B232B41F420910B0230910C023093A6
:10E47000280B2093270B2091090230910A022115C5
:10E48000310541F42DB73EB740910D0250910E0277
:10E49000241B350BE091270BF091280BE217F307B3
:10E4A000A0F42E1B3F0B2817390778F0AC014E5F04
:10E4B0005F4F2417350748F04E0F5F1F5093280B0E
:10E4C0004093270B8193919302C0E0E0F0E0CF01ED
:10E4D000DF91CF911F910F910895CF93DF93009714
:10E4E00009F481C0FC01329713821282A091290B9A
:10E4F000B0912A0B109781F420813181820F931FF4
:10E500002091270B3091280B2817390751F5F093EC
:10E51000280BE093270B67C0ED0120E030E0CE1719
:10E52000DF0740F44A815B819E0141155105F1F0FE
:10E53000EA01F5CFD383C28340815181840F951FB7
:10E54000C817D90759F488819981840F951F0296BD
:10E55000918380838A819B819383828321153105F6
:10E5600029F4F0932A0BE093290B3DC0E901FB83CA
:10E57000EA8349915991C40FD51FEC17FD0761F447
:10E5800080819181840F951F0296E9019983888388
:10E59000828193819B838A83E0E0F0E012968D91E3
:10E5A0009C911397009719F0FD01DC01F7CF8D9135
:10E5B0009C9111979D012E5F3F4F820F931F2091D9
:10E5C000270B3091280B2817390769F4309729F465
:10E5D00010922A0B1092290B02C013821282B09360
:10E5E000280BA093270BDF91CF9108958F929F92D4
:10E5F000AF92BF92CF92DF92EF92FF92CF93DF93D1
:10E60000EC01688179818A819B81611571058105A1
:10E61000910521F464E279ED8BE597E02DE133EF8C
:10E6200041E050E00E94467C49015A019B01AC0147
:10E63000A7EAB1E40E94657C6B017C01ACEEB4EF0B
:10E64000A50194010E94737CDC01CB018C0D9D1D02
:10E65000AE1DBF1DB7FF03C00197A109B048888355
:10E660009983AA83BB83BC01CD019F77DF91CF91B2
:10E67000FF90EF90DF90CF90BF90AF909F908F90E2
:10E6800008958F929F92AF92BF92CF92DF92EF92B6
:10E69000FF9260910F02709110028091110290918F
:10E6A0001202611571058105910521F464E279ED8D
:10E6B0008BE597E02DE133EF41E050E00E94467C8E
:10E6C00049015A019B01AC01A7EAB1E40E94657CB3
:10E6D0006B017C01ACEEB4EFA50194010E94737C48
:10E6E000DC01CB018C0D9D1DAE1DBF1DB7FF03C00E
:10E6F0000197A109B04880930F0290931002A09354
:10E700001102B0931202BC01CD019F77FF90EF90F0
:10E71000DF90CF90BF90AF909F908F9008956093BF
:10E720000F027093100280931102909312020895C9
:10E730003F924F925F926F927F928F929F92AF9291
:10E74000BF92CF92DF92EF92FF920F931F93CF93DE
:10E75000DF935C016B017A016115710519F0FB0112
:10E7600091838083E114F10429F0C7010297839714
:10E7700008F0C9C0E5012196F5011081812F90E0D4
:10E780000E94C374892B11F05E01F4CF1D3229F46D
:10E790002196F501118101E007C01B3221F4E5014A
:10E7A0002296F501118100E0E114F104B1F0F0E1ED
:10E7B000EF16F10429F4B0C010E3E114F10401F103
:10E7C0002AE0E216F104B1F180E1E816F10471F0FB
:10E7D000E8E0EE16F104F1F413C0103341F588813E
:10E7E0008F7D883549F7198122960260F0E1EF2E7E
:10E7F000F12C88248A94982CA82CAFE0BA2E20C043
:10E8000078E0E72EF12C88248A94982CA82CEFE14C
:10E81000BE2E16C06FEF7FEFCB0197010F2C000CBF
:10E82000440B550B0E94247C49015A0109C08AE01F
:10E83000E82EF12C69E9862E982CA82C69E1B62ED9
:10E8400040E060E070E0CB0127010F2C000C66086F
:10E850007708FE0150ED352E310E29E0231570F4B6
:10E860002FEB210F2A3118F439EC332E06C02FE993
:10E87000210F2A3130F529EA322E310E232D30E0D6
:10E880002E153F05F4F44F3FC9F086169706A806EB
:10E89000B90688F0A30192010E94147C232D30E078
:10E8A00040E050E0620F731F841F951F62177307CB
:10E8B0008407950710F44FEF01C041E021961081C5
:10E8C000C8CFC114D10451F0442311F0219703C0E3
:10E8D00001FF04C02297F601D183C08300FF07C067
:10E8E00090958095709561957F4F8F4F9F4F4F3FCB
:10E8F00079F482E290E09093320B8093310B3FEFFA
:10E900002FEF9FEF0DC040E030E020E090E008C026
:10E91000462F372F282F04C0103309F067CF5FCF61
:10E92000642F732F822FDF91CF911F910F91FF9052
:10E93000EF90DF90CF90BF90AF909F908F907F909F
:10E940006F905F904F903F900895FC018827992722
:10E95000E89421912032E9F3293010F02E30C8F3E9
:10E960002B3241F02D3239F4689404C00E94347582
:10E97000820F911D219120532A30C0F31EF49095EF
:10E9800081959F4F089591110C94207B803219F04E
:10E9900089508550C8F70895FB01DC018D910590E1
:10E9A00080190110D9F3990B0895FB01DC01059042
:10E9B0000D920020E1F70895FB01DC010D9000208D
:10E9C000E9F711974150504028F0059000200D9232
:10E9D000C9F708951C920895FB01DC014150504095
:10E9E00030F08D910590801919F40020B9F7881B3B
:10E9F000990B0895FB01DC014150504048F005900F
:10EA00000D920020C9F701C01D9241505040E0F71F
:10EA1000089545E25BE00C940D75FA01A191B08177
:10EA2000009719F41097E1F0CD01DC01CD010D90B4
:10EA3000002011F4C00113C0FB012191222319F021
:10EA40002015D9F7F3CFFB012191201519F41E925F
:10EA5000119606C02223C1F70D900020A1F7D00126
:10EA6000FA01A193B08308957AE0979F902D879F34
:10EA7000802D910D11240895FC01238127FF10C0E2
:10EA8000EBE2FBE0208131818217930711F41182C0
:10EA9000108232962BE0E133F207A1F70E946D72EB
:10EAA00080E090E008950F931F93CF93DF9300973A
:10EAB00031F46115710519F480E090E03AC08B01E2
:10EAC000EC016EE070E081E090E00E94047BFC01CC
:10EAD000892B91F380E883830115110571F0138769
:10EAE000028781E8838380912B0B90912C0B892BDB
:10EAF00021F4F0932C0BE0932B0B2097C9F0D187D6
:10EB0000C08783818260838380912D0B90912E0B2F
:10EB1000892B71F4F0932E0BE0932D0B80912F0B2A
:10EB20009091300B892B21F4F093300BE0932F0B55
:10EB3000CF01DF91CF911F910F910895CF93DF9374
:10EB4000EC012B8120FF33C026FF0AC02F7B2B83D3
:10EB50008E819F8101969F838E838A8190E029C058
:10EB600022FF0FC0E881F9818081082E000C990BEB
:10EB7000009719F420622B831AC03196F983E88339
:10EB80000EC0EA85FB85199597FF09C02B81019678
:10EB900011F080E201C080E1822B8B8308C02E81BE
:10EBA0003F812F5F3F4F3F832E83992702C08FEF16
:10EBB0009FEFDF91CF9108950F931F93CF93DF9332
:10EBC000CDB7DEB708851985F80183818860838316
:10EBD000AE01445F5F4F6A857B85C8010E9416764F
:10EBE000F8012381277F2383DF91CF911F910F911C
:10EBF00008950F931F93CF93DF93CDB7DEB70885AA
:10EC00001985F801838188608383AE01445F5F4F7B
:10EC10006A857B85C8010E94DF79F8012381277FFF
:10EC20002383DF91CF911F910F9108952F923F92EF
:10EC30004F925F926F927F928F929F92AF92BF920C
:10EC4000CF92DF92EF92FF920F931F93CF93DF93B8
:10EC5000CDB7DEB72B970FB6F894DEBF0FBECDBF92
:10EC60006C017B018A01FC0117821682838181FF7E
:10EC7000CCC1CE0101963C01F6019381F70193FDD1
:10EC8000859193FF81917F01882309F4BAC1853270
:10EC900039F493FD859193FF81917F01853229F4A9
:10ECA000B60190E00E944B7BE7CF912C212C312CB8
:10ECB000FFE1F315D8F08B3279F038F4803279F037
:10ECC0008332A1F4232D20611DC08D3261F0803389
:10ECD00069F4232D216016C0832D8260382EE32D28
:10ECE000E4603E2E2AC0F32DF8601DC037FC2DC015
:10ECF00020ED280F2A3040F08E32B9F436FC81C165
:10ED0000232D2064322E19C036FE06C08AE0989E5C
:10ED1000200D1124922E11C0EAE02E9E200D112408
:10ED2000222EF32DF0623F2E08C08C3621F4832D65
:10ED30008068382E02C0883641F4F70193FD859132
:10ED400093FF81917F018111B3CF982F9F7D9554BF
:10ED5000933028F40C5F1F4F9FE399830DC08336D7
:10ED600031F0833771F0833509F059C021C0F801C3
:10ED7000808189830E5F1F4F88248394912C5301D7
:10ED800013C02801F2E04F0E511CF801A080B180A1
:10ED900036FE03C0692D70E002C06FEF7FEFC50142
:10EDA0000E94407B4C018201F32DFF773F2E16C05D
:10EDB000280122E0420E511CF801A080B18036FEED
:10EDC00003C0692D70E002C06FEF7FEFC5010E94A4
:10EDD0002E7B4C01F32DF0683F2E820133FC1BC0CB
:10EDE000822D90E088169906B0F4B60180E290E09A
:10EDF0000E944B7B2A94F4CFF50137FC859137FEB6
:10EE000081915F01B60190E00E944B7B21102A9412
:10EE100021E0821A91088114910471F7E8C08436C8
:10EE200011F0893641F5F80137FE07C06081718124
:10EE3000828193810C5F1F4F08C060817181072E12
:10EE4000000C880B990B0E5F1F4FF32DFF763F2EA2
:10EE500097FF09C090958095709561957F4F8F4F72
:10EE60009F4FF0683F2E2AE030E0A3010E94A07B74
:10EE7000882E861845C0853731F4232D2F7EB22E7B
:10EE80002AE030E025C0932D997FB92E8F36C1F04E
:10EE900018F4883579F0B5C0803719F0883721F03B
:10EEA000B0C0E92FE061BE2EB4FE0DC0FB2DF460B2
:10EEB000BF2E09C034FE0AC0292F2660B22E06C01C
:10EEC00028E030E005C020E130E002C020E132E07F
:10EED000F801B7FE07C060817181828193810C5F68
:10EEE0001F4F06C06081718180E090E00E5F1F4F70
:10EEF000A3010E94A07B882E8618FB2DFF773F2E52
:10EF000036FE0DC0232D2E7FA22E891458F434FE18
:10EF10000BC032FC09C0832D8E7EA82E05C0B82CF4
:10EF2000A32C03C0B82C01C0B92CA4FE0FC0FE0155
:10EF3000E80DF11D8081803321F49A2D997EA92E50
:10EF400009C0A2FE06C0B394B39404C08A2D86788B
:10EF500009F0B394A3FC11C0A0FE06C0B21488F45B
:10EF6000280C922C9B180EC0B21460F4B60180E2FB
:10EF700090E00E944B7BB394F7CFB21418F42B1897
:10EF800002C0982C212CA4FE10C0B60180E390E0B2
:10EF90000E944B7BA2FE17C0A1FC03C088E790E053
:10EFA00002C088E590E0B6010CC08A2D867859F041
:10EFB000A1FE02C08BE201C080E2A7FC8DE2B60197
:10EFC00090E00E944B7B891438F4B60180E390E016
:10EFD0000E944B7B9A94F7CF8A94F301E80DF11DC0
:10EFE0008081B60190E00E944B7B8110F5CF2220FA
:10EFF00009F442CEB60180E290E00E944B7B2A9455
:10F00000F6CFF6018681978102C08FEF9FEF2B9696
:10F010000FB6F894DEBF0FBECDBFDF91CF911F9129
:10F020000F91FF90EF90DF90CF90BF90AF909F90A7
:10F030008F907F906F905F904F903F902F900895AA
:10F0400020FD09C0FC0123FD05C022FF02C073831F
:10F05000628351834083089544FD17C046FD17C065
:10F06000AB01BC01DA01FB01AA0FBB1FEE1FFF1FA2
:10F070001094D1F74A0F5B1F6E1F7F1FCB01BA019F
:10F08000660F771F881F991F09C033E001C034E065
:10F09000660F771F881F991F3150D1F7620F711DBE
:10F0A000811D911D08950F931F93CF93DF938C01C2
:10F0B000C8010E949E75EC0197FD08C00E94C374B0
:10F0C000892BB1F7B801CE010E94877BCE01DF9179
:10F0D000CF911F910F9108958F929F92AF92BF92FF
:10F0E000EF92FF920F931F93CF93DF938C01D62F54
:10F0F0007A01B22E0E949E759C0133272B32310576
:10F1000031F02D32310561F48B2D8068B82ED1504D
:10F1100011F480E068C0C8010E949E7597FDF9CF88
:10F12000CB2DCD7F2B2D207309F58033F9F4AA2444
:10F13000AA94AD0E09F443C0C8010E949E7597FDC4
:10F140003EC09C012F7D33272835310549F4C26428
:10F15000D250A9F1C8010E949E7597FF07C02FC029
:10F16000B6FE02C0C26001C0C261DA2D812C912CB2
:10F17000540120ED280F283080F0C4FF04C0B801EE
:10F180000E94877B19C02A3040F0C6FFF8CF2F7D40
:10F190003FEE320F363098F727504C2FC501B4019F
:10F1A0000E942C784B015C01C260D15059F0C8011B
:10F1B0000E949E7597FFDDCFC1FD04C0AACF812CB0
:10F1C000912C5401C7FF08C0B094A09490948094EF
:10F1D000811C911CA11CB11C2C2FB501A401C701DD
:10F1E0000E94207881E0DF91CF911F910F91FF90D5
:10F1F000EF90BF90AF909F908F9008955F926F9225
:10F200007F928F929F92AF92BF92CF92DF92EF92B6
:10F21000FF920F931F93CF93DF93CDB7DEB7A097E5
:10F220000FB6F894DEBF0FBECDBF5C01962E7A01FB
:10F23000F9018E010F5F1F4F680180E2D8011D9216
:10F240008A95E9F7D50113968C9080E090E0612CC7
:10F25000712C30E061E070E083FC259183FE219108
:10F260008F01522E211103C080E090E092C02E3514
:10F2700011F4009751F1432F50E0481759073CF41F
:10F280002D3559F12D3219F4772009F103C077207B
:10F2900009F46AC0452D469546954695D601A40FBA
:10F2A000B11D452D47708B0102C0000F111F4A95FB
:10F2B000E2F7A8015C91452B4C93651459F0561464
:10F2C00010F45394E7CF5A94E5CF31E004C077248B
:10F2D000739401C0712C0196BFCF772019F08E81F5
:10F2E00080628E83311103C08824839417C0F60195
:10F2F0009E012F5D3F4F8081809581932E173F07A0
:10F30000D1F7F2CFE114F10429F0D7018C93F70182
:10F3100031967F019A94812C9920F9F0C5010E94C1
:10F320009E7597FD18C0FC01FF2723E0F595E79532
:10F330002A95E1F7EC0DFD1D208130E0AC0147700E
:10F34000552702C0359527954A95E2F720FDDACF7B
:10F35000B5010E94877B811087CFE114F10411F081
:10F36000D7011C92C80115C0422F46954695469577
:10F37000D601A40FB11D422F47708B0102C0000FB0
:10F38000111F4A95E2F7A8015C91452B4C93622E20
:10F39000A2CFA0960FB6F894DEBF0FBECDBFDF910F
:10F3A000CF911F910F91FF90EF90DF90CF90BF9082
:10F3B000AF909F908F907F906F905F9008955F9235
:10F3C0006F927F928F929F92AF92BF92CF92DF9275
:10F3D000EF92FF920F931F93CF93DF936C01EB019A
:10F3E0005A01FC0117821682512CF601E380FE01BE
:10F3F000E3FC8591E3FE8191182FEF01882309F446
:10F40000EEC090E00E94C374892B21F0C6010E94D7
:10F410005378EBCF153241F4FE01E3FC1591E3FE86
:10F420001191EF01153281F4C6010E949E7597FD7E
:10F43000D4C0412F50E09C01332724173507A9F28F
:10F44000B6010E94877BCBC01A3239F4E3FC1591D8
:10F45000E3FE1191EF0101E001C000E0F12C20ED8D
:10F46000210F2A3080F402606F2D70E080E090E080
:10F4700040E20E942C78F62EFE01E3FC1591E3FE9B
:10F480001191EF01ECCF01FF03C0F11003C0A7C041
:10F49000FF24FA94183619F01C3651F010C0FE0102
:10F4A000E3FC1591E3FE1191EF01183641F4086079
:10F4B0000460FE01E3FC1591E3FE1191EF011123BD
:10F4C00009F48DC0612F70E08EE495E00E94237BEB
:10F4D000892B09F484C000FD07C0F501808091806C
:10F4E000C50102965C0102C0812C912C1E3651F49C
:10F4F000F6014681578160E070E0202FC4010E9430
:10F50000207873CF1336A9F401FD02C0FF24F394D1
:10F51000C6010E949E7597FD60C08114910429F078
:10F52000F4018083C40101964C01FA94F110F0CFEC
:10F5300050C01B3559F49E01A4016F2DC6010E94D5
:10F54000FE78EC01892B09F044C03EC0C6010E9440
:10F55000537897FD42C01F3661F128F4143639F113
:10F56000193651F128C0133771F0153701F123C056
:10F570008114910429F0F4016082C40101964C01C8
:10F58000FA94FF2071F0C6010E949E753C0197FD20
:10F5900008C00E94C374892B59F3B601C3010E94AD
:10F5A000877B81149104A9F0F401108212C00062DB
:10F5B00003C0006101C00064202FA4016F2DC601AB
:10F5C0000E946C78811105C0F6018381807329F453
:10F5D00006C000FD0ACF539408CF552019F0852DA1
:10F5E00090E002C08FEF9FEFDF91CF911F910F91BD
:10F5F000FF90EF90DF90CF90BF90AF909F908F9053
:10F600007F906F905F9008950F931F93CF93DF9338
:10F61000869F8001879F100D969F100D1124C801B1
:10F620000E94D571EC01009729F0A80160E070E01C
:10F630000E94397BCE01DF91CF911F910F910895E8
:10F64000992788270895FC010590061621F00020CF
:10F65000D9F7C00108953197CF010895FC010590B5
:10F66000615070400110D8F7809590958E0F9F1FC4
:10F670000895DC0101C06D9341505040E0F70895BA
:10F68000FC016150704001900110D8F78095909571
:10F690008E0F9F1F08950F931F93CF93DF93FB014E
:10F6A000238121FD03C08FEF9FEF2CC022FF16C0E6
:10F6B00046815781248135814217530744F4A08144
:10F6C000B1819D012F5F3F4F318320838C93268131
:10F6D00037812F5F3F4F3783268314C08B01EC01A6
:10F6E000FB010084F185E02D1995892BE1F6D80105
:10F6F00016968D919C911797019617969C938E93D1
:10F700001697CE01DF91CF911F910F910895FB01C4
:10F71000238120FF12C026FD10C08F3F3FEF9307CB
:10F7200061F082832F7D20642383268137812150DD
:10F73000310937832683992708958FEF9FEF089526
:10F74000FA01AA27283051F1203181F1E8946F9312
:10F750006E7F6E5F7F4F8F4F9F4FAF4FB1E03ED0B8
:10F76000B4E03CD0670F781F891F9A1FA11D680F56
:10F77000791F8A1F911DA11D6A0F711D811D911D89
:10F78000A11D20D009F468943F912AE0269F1124FE
:10F790003019305D3193DEF6CF010895462F477062
:10F7A000405D4193B3E00FD0C9F7F6CF462F4F70BD
:10F7B000405D4A3318F0495D31FD4052419302D01B
:10F7C000A9F7EACFB4E0A6959795879577956795C1
:10F7D000BA95C9F700976105710508959B01AC01C1
:10F7E0000A2E06945795479537952795BA95C9F7E8
:10F7F000620F731F841F951FA01D0895F999FECFF6
:10F8000092BD81BDF89A992780B50895262FF99960
:10F81000FECF1FBA92BD81BD20BD0FB6F894FA9AF3
:10F82000F99A0FBE01960895DB018F939F930E9472
:10F83000657CBF91AF91A29F800D911DA39F900DFC
:10F84000B29F900D11240895A1E21A2EAA1BBB1B92
:10F85000FD010DC0AA1FBB1FEE1FFF1FA217B3079C
:10F86000E407F50720F0A21BB30BE40BF50B661FB2
:10F87000771F881F991F1A9469F760957095809576
:10F8800090959B01AC01BD01CF010895052E97FB1A
:10F890001EF400940E945D7C57FD07D00E94247CDA
:10F8A00007FC03D04EF40C945D7C50954095309548
:10F8B00021953F4F4F4F5F4F0895909580957095DC
:10F8C00061957F4F8F4F9F4F08950E94787CA59F31
:10F8D000900DB49F900DA49F800D911D112408954B
:10F8E000B7FF0C94657C0E94657C821B930B089586
:10F8F000A29FB001B39FC001A39F700D811D112471
:10F90000911DB29F700D811D1124911D0895EE0F60
:10F91000FF1F881F8BBF0790F691E02D1994692770
:10F920009627692778278727782708950E94787C6B
:10F93000332312F48A1B9B0B0C94A07C0E94787CCE
:10F94000B7FF0895821B930B08955058BB27AA2731
:10F950000E94BD7C0C94377E0E94297E38F00E9464
:10F96000307E20F039F49F3F19F426F40C94267E63
:10F970000EF4E095E7FB0C94207EE92F0E94487E70
:10F9800058F3BA17620773078407950720F079F4D4
:10F99000A6F50C946A7E0EF4E0950B2EBA2FA02DDE
:10F9A0000B01B90190010C01CA01A0011124FF272C
:10F9B000591B99F0593F50F4503E68F11A16F04027
:10F9C000A22F232F342F4427585FF3CF4695379526
:10F9D0002795A795F0405395C9F77EF41F16BA0BEB
:10F9E000620B730B840BBAF09150A1F0FF0FBB1F99
:10F9F000661F771F881FC2F70EC0BA0F621F731FE2
:10FA0000841F48F4879577956795B795F7959E3F3E
:10FA100008F0B0CF9395880F08F09927EE0F9795CF
:10FA2000879508950E94FC7D08F481E008950E9466
:10FA30002B7D0C94377E0E94307E58F00E94297EE8
:10FA400040F029F45F3F29F00C94207E51110C9472
:10FA50006B7E0C94267E0E94487E68F39923B1F356
:10FA6000552391F3951B550BBB27AA2762177307E4
:10FA7000840738F09F5F5F4F220F331F441FAA1F78
:10FA8000A9F335D00E2E3AF0E0E832D09150504034
:10FA9000E695001CCAF72BD0FE2F29D0660F771FE2
:10FAA000881FBB1F261737074807AB07B0E809F0C8
:10FAB000BB0B802DBF01FF2793585F4F3AF09E3F4D
:10FAC000510578F00C94207E0C946B7E5F3FE4F33C
:10FAD000983ED4F3869577956795B795F7959F5F90
:10FAE000C9F7880F911D9695879597F90895E1E0DC
:10FAF000660F771F881FBB1F621773078407BA073B
:10FB000020F0621B730B840BBA0BEE1F88F7E09595
:10FB100008950E94907D6894B1110C946B7E0895B5
:10FB20000E94507E88F09F5798F0B92F9927B751BF
:10FB3000B0F0E1F0660F771F881F991F1AF0BA9591
:10FB4000C9F714C0B13091F00E946A7EB1E0089507
:10FB50000C946A7E672F782F8827B85F39F0B93FF9
:10FB6000CCF3869577956795B395D9F73EF4909544
:10FB70008095709561957F4F8F4F9F4F0895E894C2
:10FB800009C097FB3EF490958095709561957F4FE5
:10FB90008F4F9F4F9923A9F0F92F96E9BB27939593
:10FBA000F695879577956795B795F111F8CFFAF4A3
:10FBB000BB0F11F460FF1BC06F5F7F4F8F4F9F4FD4
:10FBC00016C0882311F096E911C0772321F09EE832
:10FBD000872F762F05C0662371F096E8862F70E098
:10FBE00060E02AF09A95660F771F881FDAF7880F72
:10FBF0009695879597F90895990F0008550FAA0BC8
:10FC0000E0E8FEEF16161706E807F907C0F012162F
:10FC10001306E407F50798F0621B730B840B950B32
:10FC200039F40A2661F0232B242B252B21F4089587
:10FC30000A2609F4A140A6958FEF811D811D089524
:10FC400097F99F6780E870E060E008959FEF80EC8F
:10FC5000089500240A941616170618060906089532
:10FC600000240A9412161306140605060895092E98
:10FC70000394000C11F4882352F0BB0F40F4BF2B07
:10FC800011F460FF04C06F5F7F4F8F4F9F4F089547
:10FC900057FD9058440F551F59F05F3F71F047953D
:10FCA000880F97FB991F61F09F3F79F08795089522
:10FCB000121613061406551FF2CF4695F1DF08C041
:10FCC000161617061806991FF1CF8695710561055E
:10FCD00008940895E894BB2766277727CB0197F906
:10FCE00008950E94FC7D08F48FEF08950E94897E9C
:10FCF0000C94377E0E94297E38F00E94307E20F0DE
:10FD0000952311F00C94207E0C94267E11240C94E3
:10FD10006B7E0E94487E70F3959FC1F3950F50E073
:10FD2000551F629FF001729FBB27F00DB11D639FAD
:10FD3000AA27F00DB11DAA1F649F6627B00DA11D53
:10FD4000661F829F2227B00DA11D621F739FB00DF9
:10FD5000A11D621F839FA00D611D221F749F332769
:10FD6000A00D611D231F849F600D211D822F762F02
:10FD70006A2F11249F5750409AF0F1F088234AF0DF
:10FD8000EE0FFF1FBB1F661F771F881F915050404B
:10FD9000A9F79E3F510580F00C94207E0C946B7E59
:10FDA0005F3FE4F3983ED4F3869577956795B795D2
:10FDB000F795E7959F5FC1F7FE2B880F911D9695EC
:10FDC000879597F90895FA01EE0FFF1F30962105E8
:10FDD0003105A1F16115710561F48038BFE39B071E
:10FDE00049F168949038810561F08038BFEF9B0736
:10FDF00041F099234AF5FF3FE1053105210519F14D
:10FE0000E8940894E795D901AA2329F4AB2FBE2FD3
:10FE1000F85FD0F310C0FF5F70F4A695E0F7F739F4
:10FE200050F019F0FF3A38F49F779F930DD00F9060
:10FE300007FC9058089546F00C94267E60E070E030
:10FE400080E89FE308954FE79F775F934F933F9339
:10FE50002F930E94E37F2F913F914F915F910E94DA
:10FE6000767E0C94407F0E94FC7D880B990B089550
:10FE700029F416F00C94207E0C946A7E0C94267E55
:10FE80000E94507EA8F39638A0F707F80F92E894E6
:10FE90002BE33AEA48EB5FE70E948C7E0F920F92C9
:10FEA0000F924DB75EB70F920E942B80E8E2F2E00E
:10FEB0000E94727F4F915F91EF91FF91E595EE1F48
:10FEC000FF1F49F0FE57E0684427EE0F441FFA95E4
:10FED000E1F74195550B0E94A57F0F9007FE0C940A
:10FEE000997F0895DF93CF931F930F93FF92EF9223
:10FEF000DF927B018C01689406C0DA2EEF010E942C
:10FF0000897EFE01E894A591259135914591559101
:10FF1000A6F3EF010E94BD7CFE019701A801DA94CF
:10FF200069F7DF90EF90FF900F911F91CF91DF91D4
:10FF300008959B01AC0160E070E080E89FE30C94C1
:10FF4000177D0C94207E0C945F800E94507ED8F325
:10FF50009923C9F3940F511DA3F39150504094F08D
:10FF600059F0882332F0660F771F881F9150504058
:10FF7000C1F79E3F51052CF7880F911D96958795E7
:10FF800097F908955F3FACF0983E9CF0BB278695AB
:10FF900077956795B79508F4B1609395C1F7BB0F56
:10FFA00058F711F460FFE8CF6F5F7F4F8F4F9F4F7F
:10FFB000E3CF0C946B7E16F00C945F800C94267E3D
:10FFC00068940C94207E0E94507EA8F39923C1F37C
:10FFD000AEF3DF93CF931F930F93FF92C92FDD27CB
:10FFE00088232AF02197660F771F881FDAF720E011
:10FFF00030E040E85FEB9FE3883920F0803E38F046
:020000021000EC
:1000000021968F770E94A67CE0E5F2E004C00E9472
:10001000A67CEDE7F2E00E94727F8B01BE01EC014D
:10002000FB2E6F5771097595771F880B990B0E94EE
:10003000C17D28E132E741E35FE30E94897EAF2D75
:100040009801AE01FF900F911F91CF91DF910E9417
:10005000BD7C0C94377EFA01DC01AA0FBB1F9B010B
:10006000AC01BF5728F4222733274427507820C0FB
:10007000B75190F4AB2F0024469537952795011C76
:10008000A395D2F3002071F0220F331F441FB395C4
:10009000DAF30ED00C94A57C61307105A0E88A07D4
:1000A000B94630F49B01AC01662777278827907802
:1000B000309621F0208331834283538308959F3FFC
:1000C00031F0915020F4879577956795B795880F13
:1000D000911D9695879597F9089581E090E0F894A1
:1000E0000C94BB819111089581568A5108F4805275
:1000F000855808950F931F93CF93DF938C01FC01D4
:1001000001900020E9F7CF01801B910B0E94D5716F
:10011000EC01009719F0B8010E94E580CE01DF9153
:10012000CF911F910F910895FB01DC0104C08D91C7
:100130000190801921F441505040C8F7881B990B59
:1001400008956817790768F4FB01DC01E40FF51FD7
:10015000A40FB51F02C002900E9241505040D8F734
:1001600008950C94B281FB01DC018D9181341CF067
:100170008B350CF4805E619161341CF06B350CF4AE
:10018000605E861B611189F3990B0895FB01DC0108
:100190000D900020E9F7119701900D920020E1F7F2
:1001A0000895FC018191861721F08823D9F79927BA
:1001B00008953197CF010895FB01DC018D910190E5
:1001C00080190110D9F3990B0895FB01DC0101900E
:1001D0000D920020E1F70895FB01DC010D90002055
:1001E000E9F711974150504028F0019000200D92FE
:1001F000C9F708951C920895FB01DC01415050405D
:1002000030F08D910190801919F40020B9F7881B06
:10021000990B0895FB01DC014150504048F00190DA
:100220000D920020C9F701C01D9241505040E0F7E7
:100230000895FC0181E090E00190061609F4CF01D9
:100240000020D1F7019708950F931F93CF93DF9369
:10025000CDB7DEB72E970FB6F894DEBF0FBECDBF79
:100260000E891F89888D998D26E02C831A83098336
:1002700097FF02C080E090E801979E838D83AE01D6
:10028000445E5F4F6A8D7B8DCE0101960E9416768B
:100290004D815E8157FD0AC02F8138854217530773
:1002A0000CF49A01F801E20FF31F10822E960FB69C
:1002B000F894DEBF0FBECDBFDF91CF911F910F919C
:1002C00008950F931F93CF93DF93CDB7DEB72E978B
:1002D0000FB6F894DEBF0FBECDBF0E891F8986E032
:1002E0008C831A8309838FEF9FE79E838D83AE01F2
:1002F000465E5F4F688D798DCE0101960E9416761D
:10030000EF81F885E00FF11F10822E960FB6F8945A
:10031000DEBF0FBECDBFDF91CF911F910F9108952A
:10032000CF93DF93CDB7DEB72E970FB6F894DEBF2D
:100330000FBECDBF85E08C838C899D899A8389838C
:10034000AE01485E5F4F6E897F89CE0101960E94A3
:10035000DF792E960FB6F894DEBF0FBECDBFDF91CA
:10036000CF910895FB01DC0102C001900D92415034
:0A0370005040D8F70895F894FFCF2D
:10037A000310000004010120000000330B8000017B
:10038A0000000000044D5154540400000000000015
:10039A000000000000000000000000000000000053
:1003AA0000000000000000000000000000002226FB
:1003BA001B5DF04C132661263F266F26D426974AEA
:1003CA00000000009A261B5DF04C1326DB269727B7
:1003DA006F26D426974A00000000000000000000A3
:1003EA0000009A261B5DF04C1326DB2687276F2612
:1003FA00D426974A30313233343536373839414288
:10040A0043444546000000000059271B5DF04C1389
:10041A0026AC266A276F26D426974A000000003D9C
:10042A0040DD41F04C2B4053403C41C4400F4272E6
:10043A004036431C447544F3438C411D416B405B79
:10044A004057400000000081097C1D00000000B8F0
:10045A005D1B5D455D055E765D545D685D0000006F
:10046A00005D455245F04C23494B454845454500FA
:10047A00000000815E5E5EF04C9B4A000000005C5A
:10048A005E1B5DF04C9B4A5C5E5C5E5C5E0000003D
:10049A00005C5E1B5DF04C9B4A000000005C5E5CE9
:1004AA005EF04C5C5E5C5E5C5E5C5E5C5E5C5E5CF0
:1004BA005E5C5E5C5E5C5E0000000088408C43F01F
:1004CA004C8740834169419E4077452C4A654144A7
:1004DA00433D427F407440E04400000000845F00D6
:1004EA000000005C5E4C6F616465642066726F6D2B
:1004FA0020666C6173682049503A0020444E533A92
:10050A00002047573A00204D41534B3A000A4E6F9C
:10051A00204950206461746120666F756E64206999
:10052A006E20666C6173680A00496E697420736B89
:10053A006970706564002B2F2B2F23002F006465D0
:10054A003A61643A62653A65663A66653A65640094
:10055A0068656C700073617665006C6F6164006732
:10056A006574006D6163006B696C6C007265710083
:10057A0069700070776400636C656172007265620D
:10058A006F6F74000D0A005F737461740056005235
:10059A00504D004900737700666C740073657400EF
:1005AA00707772002F616C61726D2F736E737200B7
:1005BA002F616C61726D2F6F767268740023253219
:1005CA0058253258253258006974656D0073636D79
:1005DA00640072636D6400656D6974004F4E004F6C
:1005EA00464600540053003B0022006E756C6C00B6
:1005FA00747275650066616C7365002D002E0025A6
:10060A0025253278006D6170002F636E662F2530C4
:10061A0032782D253032782D253032782D2530321A
:10062A00782D253032782D253032782E636F6E661C
:10063A0069672E6A736F6E0025783A25783A2578AD
:10064A003A25783A25783A25782563002F7265731A
:10065A00702F23002F7265712F636F6E6600310051
:10066A00646D78696E00646D78006D6F646275738D
:10067A00006974656D7300746F70696373006D71DE
:10068A00747400436C6F73656400202D20436C6999
:10069A00656E74206275737900533A200020536E98
:1006AA005352743A2000536F636B65743A200045C5
:1006BA00737461626C69736865640054696D656F0F
:1006CA00757400726F6F7400626373740024636FD1
:1006DA006D6D616E6400300025642C25642C2564E0
:1006EA00006E616E00696E66006F76660057495A41
:0A06FA006E6574005265733D000048
:00000001FF
